:100000000C94EC190C941D1A0C941D1A0C941D1AC6
:100010000C941D1A0C941D1A0C941D1A0C941D1A84
:100020000C941D1A0C941D1A0C941D1A0C941D1A74
:100030000C941D1A0C9461E30C941D1A0C941D1A57
:100040000C941D1A0C949BBA0C941D1A0C941D1A36
:100050000C941D1A0C941D1A0C9488F30D94FB102B
:100060000C941D1A0C947B600C941D1A0C941D1A90
:100070000C941D1A0C941D1A0C941D1A0C941D1A24
:100080000C941D1A0C941D1A0C941D1A0C941D1A14
:100090000C941D1A0C941D1A0C941D1A0C941D1A04
:1000A0000C941D1A0C941D1A0C941D1A0C941D1AF4
:1000B0000C941D1A0C941D1A0C941D1A0C941D1AE4
:1000C0000C941D1A0C941D1A0C941D1A0C941D1AD4
:1000D0000C941D1A0C941D1A0C941D1A0C941D1AC4
:1000E0000C941D1A53AB3AAB56AB3DAB40AB4CAB8B
:1000F00043AB51AB46AB49ABF0000401CA000A0167
:10010000DA001401D4001E01E200F600C600060168
:10011000EC00D600140128012001E600E0000E01E9
:100120001201CC002601D200C8002A0102012401DC
:100130001601EA00F4002201D20008011C01180196
:10014000084AD73B3BCE016E84BCBFFDC12F3D6C3E
:1001500074319ABD56833DDA3D00C77F11BED9E4A4
:10016000BB4C3E916BAAAABE000000803F05A84C84
:10017000CDB2D44EB93836A9020C50B99186880850
:100180003CA6AAAA2ABE000000803F000D94910F51
:100190000D943F100D946A0F0D942B100D94C917F8
:1001A0000D94AC190D94AE100D947F0F0D949F0F0C
:1001B0000D9405080D94740F0D94BA090D94A317AE
:1001C0000D9417100D94890F0D94BD160D94AD0F5D
:1001D0000D9483280D946D100D949B0F0D94200C9D
:1001E0000D94780F0D941E0C0D947C100D948D0FB2
:1001F0000D941A0F0D941C0F0D941F0F0D94C22116
:100200000D94A6170D944F100D947B0F0D94970F1E
:100210000D9490100D946E0F0D94E0160D941C101B
:100220000D94C1110D9421100D94B20F0D94631013
:100230000D94A4100D94763D0D949A100D94830F97
:100240000D94A90F0D9486100D9459100D9435102E
:100250000D94A50F0D9447100D9492364E414E49C2
:100260004E495459494E46CDCCCC3D0AD7233C1774
:10027000B7D13877CC2B329595E6241FB14F0A00C1
:100280000020410000C84200401C4620BCBE4CCAB1
:100290001B0E5AAEC59D74434F4D4D554E494341BB
:1002A00054494F4E0044525952554E004552524FF8
:1002B000525300494E464F004543484F00536C652A
:1002C00065702E2E2E00205A3A200020593A200028
:1002D00042656420583A2000436C69636B20746F58
:1002E00020726573756D652E2E2E004E6F206D6F1A
:1002F00076652E00456E642066696C65206C6973B6
:10030000740A00426567696E2066696C65206C69D5
:1003100073740A004D31323500286E6F2066696CA7
:100320006529005344207072696E74696E6720629B
:1003300079746520004E6F74205344207072696E8A
:1003400074696E670A0043757272656E742066691F
:100350006C653A200046696C652064656C6574655F
:10036000643A0044656C6574696F6E206661696CFF
:1003700065642C2046696C653A2000256973002568
:10038000696D20256973002569682025696D202520
:10039000697300256964202569682025696D202519
:1003A00069730025697920256964202569682025FD
:1003B000696D20256973005072696E742074696DCF
:1003C000653A2000B802B302AC02A50297026F663C
:1003D000660044454255473A004B494C4C45442E33
:1003E00020004D3131332053006F6B00416E796333
:1003F0007562696320504C5553204F66662E005439
:100400004845524D414C5F50524F54454354494F1B
:100410004E004155544F5245504F52545F53445F24
:1004200053544154555300454D455247454E435949
:100430005F50415253455200434153455F4C494739
:1004400048545F4252494748544E45535300544F15
:1004500047474C455F4C494748545300534F465417
:10046000574152455F504F574552004255494C4401
:100470005F50455243454E54004C4556454C494EFD
:10048000475F44415441005A5F50524F424500413A
:1004900055544F4C4556454C005052494E545F4AB6
:1004A0004F420050524F4752455353004155544F0D
:1004B0005245504F52545F54454D5000564F4C5585
:1004C0004D455452494300454550524F4D00534508
:1004D0005249414C5F584F4E5F584F46460046497F
:1004E000524D574152455F4E414D453A4D61726CF8
:1004F000696E20312E312E39202847697468756263
:100500002920534F555243455F434F44455F555251
:100510004C3A68747470733A2F2F67697468756207
:100520002E636F6D2F4D61726C696E4669726D77C7
:100530006172652F4D61726C696E2050524F544F3D
:10054000434F4C5F56455253494F4E3A312E30205F
:100550004D414348494E455F545950453A416E79A3
:10056000637562696320504C555320455854525569
:100570004445525F434F554E543A312055554944F6
:100580003A63656465326132662D343161322D34EF
:100590003734382D396231322D6335356336326662
:1005A00033363766660A002F2F20004D3134352050
:1005B000533C696E6465783E206F7574206F6620C9
:1005C00072616E67652028302D31290A00205400A1
:1005D000205200416363656C65726174696F6E3AA5
:1005E000205000205A00205900580020204D6178EA
:1005F0003A2000205A00205900580020204D696EF2
:100600003A20004F6E20004F666600536F667420DC
:10061000656E6473746F70733A200020466C6F7758
:100620003A20000001363726FF02FFFF353C3D38F7
:10063000FF0FFFFF312E303E1213FFFFFF28FF0C8C
:100640000809FFFF071A1C18FFFF2A08440A2C4359
:1006500020643A0020693A0020703A00496E7661C1
:100660006C69642065787472756465720A00432948
:100670000A0061626C656420286D696E2074656D86
:10068000702000436F6C64206578747275646573C4
:1006900020617265200020643A0020693A002070D1
:1006A0003A004E6F2063617365206C696768740A55
:1006B00000426564204C6576656C696E6720004673
:1006C00061696C656420746F20656E61626C652081
:1006D000426564204C6576656C696E670A00426508
:1006E00064204C6576656C20436F72726563746933
:1006F0006F6E204D61747269783A00454550524FD3
:100700004D204F4B0A003F5A206F7574206F6620B2
:1007100072616E676520282D333020746F2033306E
:10072000290A003A200050726F6265205A204F66F5
:1007300066736574004163746976652045787472E8
:10074000756465723A2000496E76616C6964206553
:10075000787472756465720A007879007A78007925
:100760007A00207A0020790020780063002E202073
:10077000202000253033692E7800302E2530336953
:10078000002073643A00737464206465763A0073E1
:100790007464206465763A004E6F20636F6E7665F0
:1007A0007267656E636500497465726174696F6E26
:1007B000203A2025303269005361766520776974CC
:1007C00068204D35303020616E642F6F7220636F6A
:1007D000707920746F20436F6E66696775726174FB
:1007E000696F6E2E6800253033692E7800302E2513
:1007F0003033690043616C6962726174696F6E20A5
:1008000073643A00726F6C6C696E67206261636B2F
:100810002E00737464206465763A0043616C6962EB
:10082000726174696F6E204F4B00456E64204452B4
:10083000592D52554E00436F727265637420646582
:100840006C74612073657474696E67732077697462
:1008500068204D36363520616E64204D3636360AB6
:10086000002020285345542D55502900202844525B
:10087000592D52554E29003F284D363635204229F4
:1008800065642072616469757320697320696D7095
:100890006C61757369626C652E0A00436865636BF1
:1008A000696E672E2E2E2041430047333320417559
:1008B000746F2043616C6962726174650A003F283D
:1008C00056296572626F7365206C6576656C206968
:1008D0007320696D706C61757369626C6520283076
:1008E000202D2033292E0A003F2846296F72636588
:1008F00020697465726174696F6E20697320696D17
:10090000706C61757369626C65202830202D20330E
:1009100030292E0A003F284329616C696272617494
:10092000696F6E20707265636973696F6E20697399
:1009300020696D706C61757369626C6520283E3D3D
:1009400030292E0A003F2850296F696E7473206980
:100950007320696D706C61757369626C6520282DF8
:1009600031202D203130292E0A0020496E76616C0D
:10097000696420657874727564657220000000E80F
:10098000C20000E8C2000000000000E8420000E8E9
:10099000420000A043486F6D6520257325732573C1
:1009A000206669727374002066697273740A005A53
:1009B0000059005800486F6D65200050726F6269E1
:1009C0006E67206661696C65640A0050726F6269C7
:1009D0006E67206661696C656400205A3A200020C9
:1009E000593A200042656420583A200047322F4788
:1009F000332062616420706172616D657465727329
:100A00000A004B494C4C45442E200053544F505043
:100A100045442E20005072696E7465722073746FA5
:100A2000707065642064756520746F206572726FE4
:100A300072732E2046697820746865206572726F23
:100A40007220616E6420757365204D3939392074C8
:100A50006F20726573746172742E202854656D70F6
:100A6000657261747572652069732072657365744F
:100A70002E2053657420697420616674657220723B
:100A8000657374617274696E67290A004E6F204342
:100A90006865636B73756D2077697468206C696E27
:100AA00065206E756D6265722C204C617374204CEC
:100AB000696E653A20004E6F20436865636B7375FD
:100AC0006D2077697468206C696E65206E756D6243
:100AD00065722C204C617374204C696E653A20005D
:100AE000636865636B73756D206D69736D617463A5
:100AF000682C204C617374204C696E653A20004C60
:100B0000696E65204E756D626572206973206E6F27
:100B100074204C617374204C696E65204E756D6253
:100B200065722B312C204C617374204C696E653AD0
:100B300020004D313130004D333100534420726577
:100B40006164206572726F720A00446F6E65207076
:100B500072696E74696E672066696C650A00526519
:100B600073656E643A20006F6B0020746F6F206CA9
:100B70006F6E6720657874727573696F6E2070721E
:100B80006576656E7465640A0020636F6C64206529
:100B90007874727573696F6E2070726576656E74A5
:100BA00065640A00627573793A20706175736564D3
:100BB00020666F7220696E7075740A0062757379B1
:100BC0003A2070617573656420666F722075736575
:100BD000720A00627573793A2070726F636573737D
:100BE000696E670A004B494C4C45442E20004B4926
:100BF0004C4C20636175736564206279204B494CCD
:100C00004C20627574746F6E2F70696E0A004B49C8
:100C10004C4C45442E20004B494C4C20636175736D
:100C2000656420627920746F6F206D756368206938
:100C30006E6163746976652074696D65202D20632B
:100C4000757272656E7420636F6D6D616E643A20AB
:100C500000506C6561736520726573657400505255
:100C6000494E5445522048414C5445440050726905
:100C70006E7465722068616C7465642E206B696C9B
:100C80006C28292063616C6C6564210A00656E71B3
:100C900075657565696E6720220000004842000096
:100CA000484200004842000000005761726E696EC1
:100CB000673A20486F6D696E672042756D702044F9
:100CC000697669736F72203C20310A000A0A0A00B3
:100CD00000A0400000A0400000A0400000684300C9
:100CE0000068430000A043010101000021104220E0
:100CF00063308440A550C660E770088129914AA1FD
:100D00006BB18CC1ADD1CEE1EFF131121002733273
:100D10005222B5529442F772D662399318837BB34C
:100D20005AA3BDD39CC3FFF3DEE362244334200403
:100D30000114E664C774A44485546AA54BB528859C
:100D40000995EEE5CFF5ACC58DD553367226111653
:100D50003006D776F6669556B4465BB77AA71997EC
:100D60003887DFF7FEE79DD7BCC7C448E5588668DB
:100D7000A7784008611802282338CCC9EDD98EE93C
:100D8000AFF9488969990AA92BB9F55AD44AB77AB3
:100D9000966A711A500A333A122AFDDBDCCBBFFB8C
:100DA0009EEB799B588B3BBB1AABA66C877CE44CC3
:100DB000C55C222C033C600C411CAEED8FFDECCDDC
:100DC000CDDD2AAD0BBD688D499D977EB66ED55E93
:100DD000F44E133E322E511E700E9FFFBEEFDDDF2C
:100DE000FCCF1BBF3AAF599F788F8891A981CAB1B8
:100DF000EBA10CD12DC14EF16FE18010A100C230EA
:100E0000E3200450254046706760B9839893FBA3A4
:100E1000DAB33DC31CD37FE35EF3B1029012F32239
:100E2000D2323542145277625672EAB5CBA5A895F4
:100E300089856EF54FE52CD50DC5E234C324A01489
:100E400081046674476424540544DBA7FAB7998784
:100E5000B8975FE77EF71DC73CD7D326F2369106D9
:100E6000B01657667676154634564CD96DC90EF9CC
:100E70002FE9C899E9898AB9ABA944586548067829
:100E80002768C018E1088238A3287DCB5CDB3FEBE4
:100E90001EFBF98BD89BBBAB9ABB754A545A376A79
:100EA000167AF10AD01AB32A923A2EFD0FED6CDDB4
:100EB0004DCDAABD8BADE89DC98D267C076C645CC9
:100EC000454CA23C832CE01CC10C1FEF3EFF5DCFC4
:100ED0007CDF9BAFBABFD98FF89F176E367E554E19
:100EE000745E932EB23ED10EF01E7C3C3E5E2B3DD6
:100EF0003F2F5B5D3B2C2A225C00454550524F4DF5
:100F0000206461746173697A65206572726F722EF4
:100F10000A00290A002062797465733B20637263BA
:100F2000200053657474696E67732053746F726523
:100F300064202800290A002062797465733B2063CD
:100F4000726320002073746F72656420736574741B
:100F5000696E6773207265747269657665642028AE
:100F600000202863616C63756C6174656429210AD3
:100F70000020213D2000454550524F4D2043524313
:100F8000206D69736D61746368202D202873746F00
:100F90007265642920002053697A653A2000496E01
:100FA0006465783A2000204D61726C696E3D56355B
:100FB00035290A0028454550524F4D3D00454550C2
:100FC000524F4D2076657273696F6E206D69736D37
:100FD000617463682000436172642072656D6F768E
:100FE0006564004361726420696E73657274656440
:100FF000004D3234004D323320257300556E6B6E38
:101000006F776E20636F6D6D616E643A20220049C8
:101010006E736572742066696C616D656E742061B3
:101020006E6420707265737320627574746F6E20C5
:10103000286F72204D313038290A005344206361F3
:101040007264206F6B0A006F70656E526F6F742050
:101050006661696C65640A00766F6C756D652E69F2
:101060006E6974206661696C65640A005344206986
:101070006E6974206661696C0A0057726974696EE2
:101080006720746F2066696C653A20006F70656E2A
:10109000206661696C65642C2046696C653A2000A5
:1010A0006F70656E206661696C65642C2046696CA2
:1010B000653A200046696C652073656C65637465EC
:1010C000640A002053697A653A200046696C6520FD
:1010D0006F70656E65643A20002066696C653A2021
:1010E00000646F696E67006672657368004E6F77A3
:1010F0002000454E4420535542524F5554494E45C9
:101100000A002220706F73002220706172656E7475
:101110003A2200535542524F5554494E45204341BF
:101120004C4C207461726765743A22004B494C4CF8
:1011300045442E2000747279696E6720746F2063B5
:10114000616C6C207375622D67636F6465206669DE
:101150006C6573207769746820746F6F206D616EA1
:1011600079206C6576656C732E204D4158206C6536
:1011700076656C2069733A004572726F723A0000AE
:10118000000000000000000000A0430A0A4265645D
:10119000204C6576656C20436F7272656374696F6D
:1011A0006E204D61747269783A00202B000A436FFB
:1011B000727265637465642042656420486569677E
:1011C00068742076732E2042656420546F706F6CB3
:1011D0006F67793A0A00202B000A4265642048654F
:1011E0006967687420546F706F6772617068793ACC
:1011F0000A2020202B2D2D2D204241434B202D2D28
:101200002B0A2020207C202020202020202020208D
:10121000207C0A204C207C20202020282B292020E4
:1012200020207C20520A2045207C202020202020C5
:1012300020202020207C20490A2046207C20282DA8
:1012400029204E20282B29207C20470A2054207C4E
:1012500020202020202020202020207C20480A2020
:1012600020207C20202020282D29202020207C20A8
:10127000540A2020207C20202020202020202020F4
:10128000207C0A2020204F2D2D2046524F4E5420E6
:101290002D2D2B0A2028302C30290A004D65616E37
:1012A000206F662073616D706C656420706F696E6D
:1012B00074733A200020643A200020623A200045EE
:1012C000716E20636F656666696369656E74733AF3
:1012D00020613A2000202844525952554E29004797
:1012E0003239204175746F20426564204C65766503
:1012F0006C696E67003F20284C2C522C462C4229EA
:10130000206F7574206F6620626F756E64732E0A8D
:10131000003F50726F626520706F696E7473202891
:10132000592920697320696D706C61757369626CED
:10133000652028322D39292E0A003F50726F6265D0
:1013400020706F696E747320285829206973206992
:101350006D706C61757369626C652028322D392956
:101360002E0A003F2856296572626F7365206C65EE
:1013700076656C20697320696D706C617573696244
:101380006C652028302D34292E0A004C696E656169
:1013900072204C6576656C696E670045787472756D
:1013A000646572733A203100687474703A2F2F6D3F
:1013B00061726C696E66772E6F726700416E796339
:1013C0007562696320504C555300323031382D30EE
:1013D000382D303100312E312E39004D61726C695B
:1013E0006E00546865726D6973746F727300426F3A
:1013F00061726420496E666F005072696E74657226
:1014000020496E666F004D61696E004D37303220A5
:10141000542564004D36303020423020542564007D
:101420004D373032203B2564004D37303120542574
:101430006400556E6C6F61642066696C616D656EE9
:101440007400556E6C6F61642066696C616D656EC9
:1014500074004D373032004D373031004C6F6164CD
:101460002066696C616D656E74004D3630302042C7
:1014700030004368616E67652066696C616D656EFA
:10148000740050726570617265005052494E54206C
:1014900050415553454400554E4C4F414420464918
:1014A0004C414D454E54004C4F41442046494C411F
:1014B0004D454E54005075726765206D6F72650022
:1014C000436F6E74696E756500524553554D4520E6
:1014D0004F5054494F4E533A0020204E6F7A7A6C49
:1014E000653A20006368616E6765006F6620746806
:1014F000652066696C616D656E7400576169742062
:10150000666F722073746172740020204E6F7A7A55
:101510006C653A200066696C616D656E7420756E4D
:101520006C6F6164005761697420666F72002020DF
:101530004E6F7A7A6C653A2000506C656173652055
:10154000776169742E2E2E0048656174696E67207C
:101550006E6F7A7A6C650020204E6F7A7A6C653AED
:10156000200068656174206E6F7A7A6C652E005079
:101570007265737320627574746F6E20746F0020CF
:10158000204E6F7A7A6C653A2000746F20636F6E1C
:1015900074696E75652E2E2E00616E642070726502
:1015A000737320627574746F6E00496E7365727424
:1015B0002066696C616D656E740020204E6F7A7ACA
:1015C0006C653A200066696C616D656E74206C6FA5
:1015D0006164005761697420666F720020204E6F4D
:1015E0007A7A6C653A200066696C616D656E74206C
:1015F0007075726765005761697420666F72007458
:101600006F20726573756D65005761697420666F30
:1016100072207072696E740020746F6F206C6F6E30
:101620006720657874727573696F6E207072657665
:10163000656E7465640A0020636F6C64206578745D
:10164000727573696F6E2070726576656E7465640D
:101650000A0024F4D43050C38E20C2A24017828BDB
:101660007011127A910D816CD90AA861E108C758EE
:101670006607615143061E4B5D05C145A7041A412B
:101680001104093D9803713931034036DB0265339B
:101690009102D4305402802E1D02632CEE01752A73
:1016A000C501B028A001102781018F2564012B24DA
:1016B0004B01E0223401AC211F018D200D01801F60
:1016C000FC00841EED00971DDF00B81CD200E61B55
:1016D000C600201BBC00641AB200B219A8000A1987
:1016E000A0006A189900D117910040178B00B51619
:1016F000840031167E00B31579003A157300C714C3
:101700006F0058146A00EE136600881363002513F7
:101710005E00C7125B006C12570015125400C11115
:10172000510070114F0021114B00D61049008D104F
:1017300047004610440002104200C00F4000800FD6
:101740003E00420F3C00060F3B00CB0E3800930ECC
:1017500037005C0E3500270E3400F30D3200C10D4A
:101760003100900D3000600D2E00320D2D00050D62
:101770002C00D90C2B00AE0C2900850C29005C0C28
:101780002700350C27000E0C2600E80B2400C40BA4
:101790002400A00B23007D0B23005A0B2100390BE2
:1017A0002100180B2000F80A1F00D90A1E00BB0AEE
:1017B0001E009D0A1D00800A1D00630A1C00470AC6
:1017C0001B002C0A1B00110A1A00F7091A00DD0978
:1017D0001900C4091900AB091900920917007B0907
:1017E0001800630917004C09160036091600200975
:1017F00016000A091500F5081500E0081400CC08C9
:101800001400B8081400A4081400900813007D0800
:1018100012006B0813005808120046081200340822
:101820001100230811001208110001081100F0072F
:101830001000E0071000D0071000C0071000B0072C
:101840000F00A107100091070E0083070F00740717
:101850000F0065070E0057070E0049070E003B07F3
:101860000D002E070E0020070D0013070D000607C0
:101870000D00F9060C00ED060D00E0060C00D40684
:101880000C00C8060C00BC060C00B0060C00A40638
:101890000B0099060C008D060B0082060B007706E4
:1018A0000B006C060B0061060A0057060B004C0685
:1018B0000A0042060A0038060A002E060A0024061C
:1018C0000A001A060A001006090007060A00FD05AC
:1018D0000900F4050900EB050900E2050900D90536
:1018E0000900D0050900C7050900BE050900B505B6
:1018F0000800AD050800A50509009C050800940531
:1019000008008C050800840508007C0508007405A3
:1019100008006C050700650508005D050700560511
:1019200008004E0507004705070040050800380578
:101930000700310507002A050700230507001C05DD
:101940000600160507000F0507000805060002053A
:101950000700FB040600F5040700EE040600E80497
:101960000600E2040700DB040600D5040600CF04ED
:101970000600C9040600C3040600BD040600B7043F
:101980000600B1040500AC040600A6040600A0048D
:1019900005009B04060095040500900406008A04D7
:1019A000050085040500800406007A04050075041E
:1019B0000500700405006B04050066040500610461
:1019C00005005C04050057040500520405004D04A1
:1019D000050048040500430405003E0404003A04E1
:1019E000050035040500300404002C04050027041C
:1019F0000400230405001E0404001A040400160455
:101A00000500110404000D04040009040500040489
:101A1000040000040400FC030400F8030400F403C1
:101A20000400F0030400EC030400E8030400E403F2
:101A30000400E0030400DC030400D8030400D40322
:101A40000400D0030400CC030400C8030300C50352
:101A5000030024F404D9201BC40C5C0E9804C409B0
:101A60005F0265077101F405F900FB04B300480447
:101A70008700C10369005803550003034500BE02F7
:101A80003A008402310053022A0029022500040290
:101A90002000E4011C00C8011900AF0117009801E3
:101AA0001400840113007101100061011000510144
:101AB0000E0043010D0036010B002B010B0020012D
:101AC0000B00150109000C01090003010800FB00CF
:101AD0000800F3000800EB000700E4000600DE0049
:101AE0000600D8000600D2000600CC000500C700A2
:101AF0000500C2000500BD000400B9000400B500E7
:101B00000400B1000400AD000400A9000400A50019
:101B10000300A20003009F0004009B000300980044
:101B200003009500020093000300900003008D0065
:101B300002008B000300880002008600020084007F
:101B40000300810002007F0002007D0002007B0094
:101B500002007900020077000100760002007400A4
:101B6000020072000100710002006F0002006D00AF
:101B700001006C0002006A000100690002006700B9
:101B800001006600010065000100640002006200BF
:101B9000010061000100600001005F0002005D00C3
:101BA00001005C0001005B0001005A0001005900C7
:101BB00001005800010057000100560001005500C7
:101BC00001005400010053000000530001005200C6
:101BD000010051000100500001004F0001004E00C3
:101BE00000004E0001004D0001004C0001004B00C0
:101BF00000004B0001004A000100490001004800BC
:101C000000004800010047000100460000004600B7
:101C100001004500000045000100440001004300B0
:101C200000004300010042000000420001004100AA
:101C3000000041000100400001003F0000003F00A3
:101C400001003E0000003E0001003D0000003D009C
:101C500001003C0000003C0000003C0001003B0093
:101C600000003B0001003A0000003A00010039008A
:101C70000000390001003800000038000000380082
:101C80000100370000003700010036000000360078
:101C9000000036000100350000003500000035006E
:101CA0000100340000003400000034000100330063
:101CB0000000330000003300010032000000320059
:101CC000000032000100310000003100000031004E
:101CD00001003000000030000000300001002F0043
:101CE00000002F0000002F0000002F0001002E0038
:101CF00000002E0000002E0001002D0000002D002D
:101D000000002D0000002D0001002C0000002C0020
:101D100000002C0000002C0001002B0000002B0014
:101D200000002B0000002B0001002A0000002A0008
:101D300000002A0000002A000100290000002900FC
:101D400000002900000029000000290001002800EF
:101D500000002800000028000000280000002800E3
:101D600001002700000027000000270000002700D6
:101D700000002700010026000000260000002600C9
:101D800000002600000026000100250000002500BC
:101D900000002500000025000000250000002500AF
:101DA00001002400000024000000240000002400A2
:101DB0000000240001002300000023000000230095
:101DC0000000230000002300000023000000230087
:101DD000010022000000220000002200000022007A
:101DE000000022000000220001002100000021006C
:101DF000000021000000210000002100000021005F
:101E00000000210001002000000020000000200050
:101E10000000200000002000000020000000200042
:101E20000000200001001F0000001F0000001F0034
:101E300000001F0000001F0000001F0000001F0026
:101E400001001E0000001E0000001E0000001E0019
:101E50000000043700001E290000511B000058102C
:101E6000000010090000CC040000780200004101CD
:101E700000001000C90210012C0140012201700174
:101E80001801B0010E01F00104015002FA00B00285
:101E9000F0003003E600D003DC009004D2007005AF
:101EA000C800A006BE000008B400B009AA00D00B0C
:101EB000A000600E960060118C00001582002019B1
:101EC0007800C01D6E00A0226400B0275A00902C3C
:101ED000500000314600E0343C0010383200903AA7
:101EE0002800603C1E00A03D1400803E0A00203FF8
:101EF0000000202F002042403A0020403A00257583
:101F00003A2530327500253032753A253032750069
:101F10002D2D2D00534400202020202020002020A3
:101F2000202000205A3A0020593A0020436F756E55
:101F30007420583A0020453A00205A3A0020593A75
:101F400000583A003A004361703A004B6420002385
:101F5000646566696E652044454641554C545F0092
:101F60004B69200023646566696E652044454641DF
:101F7000554C545F004B70200023646566696E65A4
:101F80002044454641554C545F005049442041751A
:101F9000746F74756E652066696E69736865642117
:101FA0002050757420746865206C617374204B70C8
:101FB0002C204B6920616E64204B6420636F6E732C
:101FC00074616E74732066726F6D2062656C6F77DA
:101FD00020696E746F20436F6E66696775726174F5
:101FE000696F6E2E680A00504944204175746F7401
:101FF000756E65206661696C6564212074696D6524
:102000006F75740A00453120544845524D414C20AB
:1020100052554E415741590042454420544845527B
:102020004D414C2052554E415741590054686572FC
:102030006D616C2052756E61776179004531204881
:10204000656174696E67206661696C6564004265EC
:10205000642068656174696E67206661696C656497
:102060000048656174696E67206661696C6564002B
:10207000504944204175746F74756E6520666169BE
:102080006C6564212054656D70657261747572654C
:1020900020746F6F20686967680A00204B643A20DB
:1020A00000204B693A2000204B703A20000A204360
:1020B0006C617373696320504944200A0020547591
:1020C0003A2000204B753A2000206D61783A2000BC
:1020D000206D696E3A200020643A20002062696118
:1020E000733A2000504944204175746F74756E65D1
:1020F000206661696C6564212042616420657874A2
:102100007275646572206E756D6265720A00504961
:1021100044204175746F74756E65207374617274B8
:102120000A00496E736572742066696C616D656E34
:102130007420616E642070726573732062757474AC
:102140006F6E0A00507265737320627574746F6EDF
:1021500020746F2068656174206E6F7A7A6C650AEE
:1021600000496E736572742066696C616D656E748A
:1021700020616E6420707265737320627574746F71
:102180006E20286F72204D313038290A0050726558
:10219000686561742041425320456E640050726549
:1021A0006865617420414253204265640050726545
:1021B00068656174204142530050726570617265B8
:1021C0000050726568656174204142530050726529
:1021D0006865617420504C4100436F6F6C646F7789
:1021E0006E004368616E67652066696C616D656E3F
:1021F000740044697361626C652073746570706506
:102200007273004D3834004F6666004F6E200042F6
:102210006564204C6576656C696E670044656C7416
:10222000612043616C6962726174696F6E004C6514
:1022300076656C20626564004732380A473239009F
:102240004175746F20686F6D6500473238004D6FBF
:1022500076652061786973004D61696E00486F6D25
:10226000696E672058595A004732380044696167DF
:1022700020526F64004469616720526F6400547A91
:1022800000547A005479005479005478005478004E
:102290005261646975730052616469757300457AAF
:1022A00000457A0045790045790045780045780079
:1022B00048656967687400486569676874004465C3
:1022C0006C74612043616C6962726174696F6E0045
:1022D0004573746570732F6D6D004573746570730D
:1022E0002F6D6D004373746570732F6D6D004373B4
:1022F000746570732F6D6D004273746570732F6D0C
:102300006D004273746570732F6D6D004173746559
:1023100070732F6D6D004173746570732F6D6D0058
:102320004D6F74696F6E0053746570732F6D6D001F
:102330004A65726B00416363656C65726174696FB5
:102340006E0056656C6F636974790050726F6265D8
:10235000205A204F66667365740050726F62652064
:102360005A204F666673657400436F6E74726F6CAB
:10237000004C6F6164206D6D004C6F6164206D6D69
:10238000004C6F6164206D6D00556E6C6F61642050
:102390006D6D00556E6C6F6164206D6D00556E6CD7
:1023A0006F6164206D6D0046696C2E204469612E5A
:1023B0000046696C2E204469612E004F6666004F0E
:1023C0006E20004520696E206D6D3300436F6E7482
:1023D000726F6C0043616E6E6F7420656E7465720F
:1023E000207375626469723A2000052E2E004D61DB
:1023F000696E004D61782054656D703A203132303D
:10240000004D696E2054656D703A20350054426568
:10241000643A4154432031303447542D32004D61E9
:10242000782054656D703A20323735004D696E2042
:1024300054656D703A20350054303A2041544320A1
:1024400031303447542D32005053553A2047656E91
:10245000657269630050726F746F636F6C3A2031FC
:102460002E3000426175643A203235303030300011
:1024700052414D505320312E3400000022002500DF
:1024800028002B002E00310034000201000005015D
:1024900008010B01000020002300260029002C0069
:1024A0002F003200000100000301060109010505AB
:1024B0000505070508080808020202020A0A0808BA
:1024C00004040404010101010101010103030303E8
:1024D00003030303040707070C0C0C0C0C0C0C0C77
:1024E0000202020206060606060606060B0B0B0B88
:1024F0000B0B0B0B010210202008081020401020AD
:1025000040800201020108040201010204081020B7
:1025100040808040201008040201800402018040B5
:10252000201008040201080402010102040810201E
:102530004080010204081020408000000A0B0209BC
:102540000C0D0E080703040100000000000000004D
:10255000000000000000000000000000000000007B
:102560000000000000001211100000000000000038
:10257000000000000000000000000000000000005B
:102580000200000000010204040000001C1C0C04F6
:102590000404020100000000000408100000000014
:1025A000002D2D2D2D2D2D007C4D61726C696E7CC2
:1025B000002D2D2D2D2D2D0020312E312E390020D6
:1025C00020506C616E6E6572427566666572427906
:1025D0007465733A20002046726565204D656D6F05
:1025E00072793A2000436F6D70696C65643A204AD5
:1025F000616E20323620323031390A00207C204191
:102600007574686F723A2028547269616C6F6E2C11
:1026100020323031382F31322F3130290A00323018
:1026200031382D30382D303100204C6173742055F5
:102630007064617465643A2000312E312E390A00CD
:102640004D61726C696E0020536F667477617265BC
:102650002052657365740A00205761746368646F63
:10266000672052657365740A002042726F776E208E
:102670006F75742052657365740A0020457874651F
:10268000726E616C2052657365740A00506F7765D5
:102690007255700A0073746172740A006175746F08
:1026A00025692E67006572726F722077726974698E
:1026B0006E6720746F2066696C650A00456E6473EE
:1026C000746F7073202563202563202563202563A4
:1026D00000205A3A0020593A0020583A00656E64AA
:1026E00073746F7073206869743A2000446F6E656C
:1026F00020736176696E672066696C652E0A004DED
:1027000032390043616C696272617465205A00431A
:10271000616C69627261746520590043616C696221
:10272000726174652058004175746F20686F6D6523
:102730000044656C74612053657474696E6773003E
:102740004C6F61642073657474696E6773004361D4
:102750006C6962726174652043656E7465720053C2
:10276000746F72652073657474696E67730050725C
:102770006F6265205A2D6F66667365740047333348
:1027800020502D31005365742044656C74612048DD
:1027900065696768740047333320503100417574B0
:1027A0006F2043616C6962726174696F6E004733B8
:1027B00033004D61696E004D6F76652058004D6F96
:1027C00076652059004D6F7665205A004578747201
:1027D00075646572004D6F766520302E316D6D0029
:1027E0004D6F766520316D6D004D6F76652031300F
:1027F0006D6D004D6F766520617869730045787462
:102800007275646572004D6F7665205A004D6F7663
:10281000652059004D6F76652058004D6F76696EC2
:10282000672E2E2E004578747275646572004175AE
:10283000746F20686F6D6500473238004D6F7665A4
:10284000205A0046726565205859004D6F76652004
:1028500059004D6F76652058004F6666004F6E2018
:1028600000536F667420456E6473746F707300500C
:1028700072657061726500496E697469616C697A2C
:102880006520454550524F4D00436F6E74726F6C1A
:1028900000526573746F7265206661696C7361665E
:1028A00065004C6F61642073657474696E677300B2
:1028B000496E697469616C697A6520454550524F6B
:1028C0004D0053746F72652073657474696E67731D
:1028D0000046696C616D656E74004D6F74696F6E52
:1028E0000054656D7065726174757265004D616943
:1028F0006E004D3330332055312045256920532556
:102900006900507265686561742041425320636FAD
:102910006E66005072656865617420504C4120639A
:102920006F6E6600504944204175746F74756E6512
:1029300000504944204175746F74756E65005049AC
:1029400044204175746F74756E65005049442D4480
:10295000005049442D44005049442D4900504944F9
:102960002D49005049442D50005049442D5000201D
:1029700002204661637400200220466163740020D7
:1029800002204D6178002002204D61780020022055
:102990004D6178002002204D696E002002204D69B3
:1029A0006E002002204D696E004F6666004F6E205B
:1029B000004175746F74656D700046616E207370B0
:1029C0006565640046616E207370656564004661EC
:1029D0006E20737065656400426564004265640042
:1029E000426564004E6F7A7A6C65004E6F7A7A6C3D
:1029F00065004E6F7A7A6C6500436F6E74726F6C0F
:102A00000053746F72652073657474696E67730028
:102A10004265640042656400426564004E6F7A7AE4
:102A20006C65004E6F7A7A6C65004E6F7A7A6C65D1
:102A30000046616E2073706565640046616E2073A8
:102A4000706565640046616E20737065656400544E
:102A5000656D7065726174757265002CFFFFFFFF14
:102A6000FF0001010101016265640A002C207379F5
:102A70007374656D2073746F707065642120486590
:102A8000617465725F49443A20004265642068655C
:102A90006174696E67206661696C65640048656190
:102AA00074696E67206661696C6564004531204811
:102AB000656174696E67206661696C65640048656C
:102AC0006174696E67206661696C656400453120D8
:102AD000544845524D414C2052554E4157415900A2
:102AE00042454420544845524D414C2052554E4198
:102AF00057415900546865726D616C2052756E6162
:102B0000776179004531204572723A204D41585421
:102B1000454D50004572723A204D415854454D5034
:102B200020424544004D415854454D50207472692F
:102B3000676765726564004531204572723A204DC1
:102B4000494E54454D50004572723A204D494E54FD
:102B5000454D5020424544004D494E54454D50206E
:102B6000747269676765726564004D383420582057
:102B700059205A20450048617264636F646564207F
:102B800044656661756C742053657474696E67730F
:102B9000204C6F616465640A00E8030000E80300EC
:102BA00000E8030000E8030000000048430000487C
:102BB0004300004843000048420000A0420000A03B
:102BC000420000A0420000C0423A0A0020286D6D79
:102BD000290020204D36303320002055004C00467F
:102BE000696C616D656E74206C6F61642F756E6CBD
:102BF0006F6164206C656E677468733A0A00202008
:102C00004D383531205A005A2D50726F6265204F71
:102C100066667365740020440020490020204D330F
:102C2000303420500020440020490020204D333013
:102C3000312050005049442073657474696E677385
:102C40003A0A0020460020420020480020204D3152
:102C500034352053004D6174657269616C2068657C
:102C60006174757020706172616D65746572733A1C
:102C70000A00205A0020590020580020420020530A
:102C80000020480020520020204D363635204C00D0
:102C900044656C74612073657474696E67733A205F
:102CA0004C3C646961676F6E616C5F726F643E205B
:102CB000523C7261646975733E20483C686569677F
:102CC00068743E20533C7365676D656E74735F7006
:102CD00065725F733E20423C63616C69627261742D
:102CE000696F6E207261646975733E2058595A3C51
:102CF000746F77657220616E676C6520636F7272A6
:102D0000656374696F6E733E0A00205A0020590093
:102D100020204D363636205800456E6473746F702F
:102D20002061646A7573746D656E743A0A002020C0
:102D30004D3432302053004175746F204265642059
:102D40004C6576656C696E673A0A00204500205A2A
:102D50000020590020580020540020530020204D0E
:102D600032303520420020453C6D61785F655F6AF6
:102D700065726B3E0020583C6D61785F785F6A65D4
:102D8000726B3E20593C6D61785F795F6A65726B4A
:102D90003E205A3C6D61785F7A5F6A65726B3E00D7
:102DA000416476616E6365643A20423C6D696E5F92
:102DB0007365676D656E745F74696D655F75733E8D
:102DC00020533C6D696E5F66656564726174653E33
:102DD00020543C6D696E5F74726176656C5F6665E8
:102DE0006564726174653E0020540020520020200A
:102DF0004D323034205000416363656C65726174FC
:102E0000696F6E2028756E6974732F7332293A20AA
:102E1000503C7072696E745F616363656C3E2052F2
:102E20003C726574726163745F616363656C3E20BC
:102E3000543C74726176656C5F616363656C3E0AD5
:102E400000204500205A0020590020204D3230310A
:102E50002058004D6178696D756D20416363656C24
:102E600065726174696F6E2028756E6974732F7353
:102E700032293A0A00204500205A0020590020201B
:102E80004D3230332058004D6178696D756D206684
:102E900065656472617465732028756E6974732F3B
:102EA00073293A0A00204500205A002059002020AA
:102EB0004D3932205800537465707320706572204C
:102EC000756E69743A0A0020204D3230302044304B
:102ED0000A0020204D3230302044002044697361C4
:102EE000626C65640A0046696C616D656E7420737E
:102EF000657474696E67733A0020204D313439204F
:102F000043203B20556E69747320696E2043656CC5
:102F1000736975730A002020473231202020203B3E
:102F2000006F70656E206661696C65642C2046696F
:102F30006C653A200043616E6E6F74206F70656E31
:102F40002073756264697220006563686F3A0000DF
:102F50001C1F11111F00000006191803130C000498
:102F60000E1F041C000000000E1315110E00001CA3
:102F700010181705060500040A0A0A0A11110E0C9A
:102F800012120C00000000001F1511151F00005642
:102F900054726176206D696E005654726176206DB0
:102FA000696E005654726176206D696E00566D69C7
:102FB0006E00566D696E00566D696E00566D6178D3
:102FC000204500566D6178204500566D617820459A
:102FD00000566D6178204300566D6178204300569D
:102FE0006D6178204300566D6178204200566D6116
:102FF00078204200566D6178204200566D6178203D
:103000004100566D6178204100566D617820410085
:103010004D6F74696F6E00416D6178204500416DA0
:103020006178204500416D6178204300416D6178F1
:10303000204300416D6178204200416D617820425B
:1030400000416D6178204100416D6178204100416F
:103050002D74726176656C00412D74726176656CB9
:1030600000412D7265747261637400412D72657444
:103070007261637400416363656C00416363656CF6
:10308000004D6F74696F6E0056652D6A65726B0036
:1030900056652D6A65726B0056652D6A65726B0008
:1030A00056632D6A65726B0056632D6A65726B00FC
:1030B00056632D6A65726B0056622D6A65726B00ED
:1030C00056622D6A65726B0056622D6A65726B00DE
:1030D00056612D6A65726B0056612D6A65726B00D0
:1030E00056612D6A65726B004D6F74696F6E0000DA
:1030F000002100240027002A002D003000330001A9
:10310000010000040107010A01416E7963756269DB
:103110006320504C55532052656164792E005072E3
:10312000696E74696E672E2E2E005072696E74205F
:10313000706175736564004D313235004D32340075
:103140005072696E742061626F72746564004E6FB4
:103150002053442063617264005072696E7420666B
:10316000726F6D2053440053746F70207072696EDB
:103170007400526573756D65207072696E740041DC
:10318000626F7574205072696E746572005061755B
:103190007365207072696E7400436F6E74726F6C29
:1031A00000507265706172650054756E6500496EFD
:1031B000666F2073637265656E004368616E676554
:1031C0002066696C616D656E7400466C6F770046B1
:1031D0006C6F7700466C6F770046616E2073706588
:1031E00065640046616E2073706565640046616EBB
:1031F0002073706565640042656400426564004246
:103200006564004E6F7A7A6C65004E6F7A7A6C65F1
:10321000004E6F7A7A6C6500537065656400537078
:10322000656564005370656564004D61696E0050AA
:1032300072656865617420504C4120456E64005091
:1032400072656865617420504C412042656400508D
:1032500072656865617420504C4100507265706100
:103260007265004572726F722077726974696E6759
:1032700020746F20454550524F4D210A00486F740D
:10328000656E6420746F6F20636F6C640A004D3646
:1032900030303A20546F6F20636F6C6400486F7455
:1032A000656E6420746F6F20636F6C640A005072E7
:1032B0006F7465637465642050696E0A0020573A24
:1032C000004520436F6F6C696E672E2E2E004520DF
:1032D00048656174696E672E2E2E0020573A0042B1
:1032E000656420636F6F6C696E672E2E2E004265D9
:1032F000642068656174696E672E2E2E00486F6DBC
:10330000696E67206661696C6564007A5F6D6178DB
:103310003A20007A5F6D696E3A2000795F6D6178BE
:103320003A2000785F6D61783A20005265706F72C4
:1033300074696E6720656E6473746F702073746156
:103340007475730A004368616E67652066696C6115
:103350006D656E7400556E6C6F61642066696C619A
:103360006D656E74004C6F61642066696C616D659B
:103370006E7400507265686561742041425300505C
:1033800072656865617420504C41004368616E67E6
:10339000652066696C616D656E74002020004F6663
:1033A000667365740020205261646975733A005435
:1033B0007A00547900547800202052616469757352
:1033C0003A00457A004579004578002E48656967DE
:1033D00068743A001A012C0111241FBECFEFD1E20C
:1033E000DEBFCDBF00E00CBF13E0A0E0B2E0ECE137
:1033F000FBE902E00BBF02C007900D92A035B107B8
:10340000D9F723E1A0E5B3E001C01D92AB3AB207C2
:10341000E1F719E1CBEED9E100E006C021970109FF
:10342000802FFE010F94EC4CCA3ED10780E00807C4
:10343000A9F70F947F380D947D4D0C9400002F92C6
:103440003F924F925F926F927F928F929F92AF9234
:10345000BF92CF92DF92EF92FF920F931F93CF9381
:10346000DF93CDB7DEB7A7970FB6F894DEBF0FBED8
:10347000CDBF41E040932E058091A4138D3409F413
:10348000C6C1843511F40C949D2D873411F00C9431
:10349000E92D2091A2133091A3132C31310509F4A9
:1034A000C7C09CF4243031053CF4223031050CF0C7
:1034B00044C037FF28C0A7C12430310509F446C0F5
:1034C0002B31310509F481C09EC12132310509F447
:1034D0001FC14CF42D31310509F4AEC02E31310538
:1034E00009F4AEC090C12B35310509F415C12C3556
:1034F000310509F415C12A35310509F084C110924E
:1035000054030C94EB2D80914802882311F40C9401
:10351000EB2D8AE50E947B5C082F89E50E947B5C8D
:10352000182F88E50E947B5C402F612F0E94474B3B
:1035300081110C94EB2D0C94F02D81E0223031059B
:1035400009F080E00E94F94B0C94EB2D80E50E947D
:10355000C45C882329F00E94085C6B017C0103C0D5
:10356000C12CD12C760183E50E94C45C882361F0D4
:103570000E94485C20E030E04AE754E40F94C245E2
:103580000F94D04A6B017C010E94C6B9809131052D
:10359000811105C060E08DEB92E00E94CD890F940F
:1035A000EF10C60ED71EE81EF91E0F94EF10DC01B7
:1035B000CB018C199D09AE09BF09B7FD02C00C945F
:1035C000EB2D80E00E941561F0CF41E061E081E0E9
:1035D0000E94474B81110C94EB2D80E090E0A4ED0C
:1035E000B2EC89839A83AB83BC8380E090E0A4ED46
:1035F000B2E48D839E83AF83B88780E090E0A0EF34
:10360000B1E489879A87AB87BC8780E50E94C45C58
:10361000882319F00E94185C01C060E068A3BE0115
:103620006F5F7F4FCE0180960F94592C0C94EB2D39
:103630000E94D1750C94EB2D0E94AB950C94EB2D50
:10364000C0909505D0909605E0909705F09098056C
:1036500088E50E94C45C811108C020E030E0A90127
:10366000C701B6010F94874902C00E94485C68A355
:1036700079A38AA39BA3C0909905D0909A05E09066
:103680009B05F0909C0589E50E94C45C811108C0EF
:1036900020E030E0A901C701B6010F94874902C0BC
:1036A0000E94485C6B017C0169837A838B839C83D5
:1036B00068A179A18AA19BA19B01AC010F94C2458D
:1036C0004B015C01A7019601C701B6010F94C245E9
:1036D0009B01AC01C501B4010F9487496B017C01CA
:1036E00020E030E442E556E40F945D45181614F4EA
:1036F0000C94EB2D20E030E94FE256E4C701B6010F
:103700000F945D45181614F40C94EB2D0C94F52DC4
:103710000E942B2F0C94EB2D409354030C94EB2D13
:10372000F7E52F2EF2E03F2EADE0EA2EAFE0FA2EC5
:10373000B5E9CB2EB5E0DB2E00E010E0F101819180
:103740001F010E94C45C882309F449C00E94485CA0
:103750002B013C01133049F0F70120813181428176
:1037600053810F9486492B013C01F6012081318160
:1037700042815381C301B2010F9486494B015C0120
:103780002DEB37E346E855EB0F94FB4B87FD0AC062
:103790002DEB37E346E855E3C501B4010F945D45D1
:1037A0001816ECF4133051F44092A1055092A20582
:1037B0006092A3057092A40501E011C0A5019401D7
:1037C000F70160817181828193810F948749F701AC
:1037D0006083718382839383812F0E9410561F5FC1
:1037E000F4E0EF0EF11C24E0C20ED11C143009F0FD
:1037F000A5CF002321F081EA95E00E948B920E94E0
:1038000080D40C94EB2D0E9432950C94EB2D80917A
:10381000A2139091A3138737910511F40C943D25C1
:103820000CF0EBC08D34910509F4ADC50CF058C017
:103830008931910509F41DC31CF58431910509F402
:1038400006C27CF48131910509F47CC22CF4029704
:1038500008F400C20C949A2D429709F48BC70C947B
:103860009A2D8631910509F4BEC20CF4B8C2873195
:10387000910509F4BEC2489709F4D1C20C949A2D5F
:103880008E31910509F4B3C384F48B31910509F4A9
:103890000CC30CF4FCC28C31910509F49EC34D9706
:1038A00011F40C94EB2D0C949A2D8A32910509F4A5
:1038B00032C54CF48F31910509F477C4809709F42F
:1038C00028C40C949A2D8B34910509F458C58C3476
:1038D000910511F00C949A2D0E94EFF50C94EB2DAC
:1038E0008B36910509F4A3C60CF04CC085359105C3
:1038F00009F475C74CF58235910509F432C7D4F443
:103900008135910511F00C949A2D0E9419F60E94B0
:1039100004BA1092801310927F1368EE73E080E077
:1039200090E00E944A8960E08CEE93E00E94CD898D
:103930000C94EB2D8335910509F417C78435910557
:1039400009F418C70C949A2D8836910509F41FC5FF
:103950007CF48C35910511F00C949A2D47E5C42E1A
:1039600042E0D42E55E8E52E55E0F52E10E052C782
:103970008936910509F4D5C58A36910509F439C609
:103980000C949A2D8037910509F496C584F48D36F0
:10399000910509F408C60CF48BC58E36910509F41F
:1039A00021C58F36910509F430C50C949A2D8337C3
:1039B000910509F449C17CF48137910509F484C566
:1039C0008237910511F00C949A2D0E94C6B90E947D
:1039D00080D40C94EB2D8537910509F4F7C7863711
:1039E000910511F00C949A2D0091A0131091A11340
:1039F00083E0D12C40E00C94FD24803331E0930728
:103A000011F40C94CD290CF07AC08B3C910511F483
:103A10000C943226CCF58139910511F40C944E2585
:103A200094F48937910511F40C94482514F40C94FE
:103A300041258D37910509F40CC68C38910509F4A0
:103A4000B6C50C949A2D8E3B910509F4CEC534F47D
:103A50008B39910509F480C50C949A2D883C910509
:103A600011F40C94C925893C910511F00C949A2D00
:103A700017E5E12E12E0F12E0DE113E18DE2C82EE3
:103A800083E1D82E0C941A268D3D910511F40C94E7
:103A900019289CF48D3C910511F40C94C22614F461
:103AA0000C944D26833D910509F4CAC08C3D9105C7
:103AB00011F40C940C280C949A2D8D32F1E09F0790
:103AC00011F40C94D92864F4823E910511F40C94FD
:103AD00087288C32914011F40C94B0280C949A2DC4
:103AE0008E32E1E09E0711F40C9479298F329140D7
:103AF00011F00C949A2D0E94FBCE0C94EB2D883F74
:103B000021E0920711F40C94052B0CF04BC08A397C
:103B1000E1E09E0709F4D4C414F5803921E092074E
:103B200011F40C94602A4CF48336914011F00C94FB
:103B30009A2DE8E7F1E10C944D2A8139F1E09F07D5
:103B400011F40C94632A8239914011F00C949A2D4F
:103B500080E00E94DC520E9480D40C94EB2D853FC3
:103B600031E0930711F40C94F32A7CF4843AF1E0E9
:103B70009F0711F40C94692A843F914011F00C9432
:103B80009A2D0E94C47E0C94EB2D863F31E0930762
:103B900011F40C94F62A873F914011F40C94F92A01
:103BA0000C949A2D8D3BF2E09F0711F40C944A2C53
:103BB0003CF58B3532E0930711F40C94282B4CF430
:103BC0008835924011F00C949A2D0E94D0CC0C9420
:103BD000EB2D893922E0920711F40C94B12B8A392C
:103BE000924011F00C949A2D27E5E22E22E0F22E5D
:103BF00000E51DE03CE5C32E3DE0D32E0C94422CA5
:103C00008B38E3E09E0711F40C94EB2D6CF48E3BA3
:103C100022E0920711F40C944D2C8335934011F45B
:103C20000C94202D0C949A2D803AE3E09E0709F421
:103C3000AFC2873E934011F40C94852D0C949A2DBD
:103C4000E9E4FFE20C942D27EEEDF4E063C6E3E037
:103C5000F3E087C0A090A013B090A11380E50E946C
:103C6000C45C882359F00E94085C6B017C0111E060
:103C7000672B682B692B31F410E004C010E0C12CD5
:103C8000D12C760183E50E94C45C882311F40C9446
:103C9000862E0E94485C20E030E04AE754E40F940E
:103CA000C2450F94D04A6B017C0111110BC0672BE8
:103CB000682B692B39F4A114B10421F0F50180813E
:103CC000811102C010E001C011E00E94C6B91123A9
:103CD00029F061E0C5010E94098A05C060E088ED15
:103CE00092E00E94CD8983E080932E0581E080934D
:103CF0002D05C114D104E104F104B1F00F94EF10CB
:103D0000C60ED71EE81EF91E0F94EF10DC01CB0182
:103D10008C199D09AE09BF09B7FF0EC080912D0512
:103D200081110C948B2E08C080912D05882321F0E1
:103D300080E00E941561F8CF0F94A81710922D050E
:103D40000C94EB2D60E08BEE92E00E94CD895F98A1
:103D50008A988091080181708093060112980C94D2
:103D6000EB2D84918F010F5F1F4F882321F00E945C
:103D7000EA5CF801F6CF1092FE1281EB90E10E940E
:103D800031718BE1E1EBF0E1DE01159601900D92CE
:103D90008A95E1F78091AF109091B0109C838B834E
:103DA00081E093E09A83898340E050E0BE016F5F39
:103DB0007F4F80E090E00F944205CE0101960E9473
:103DC000A560E4EFF2E084918F010F5F1F4F88231D
:103DD00011F40C94EB2D0E94EA5CF801F4CF0E94E0
:103DE000CF900C94EB2D10925A1010925B100C9403
:103DF000EB2DE091A013F091A1138081882329F08D
:103E0000803209F410823196F8CF40E061E0809171
:103E1000A0139091A1130E94EC8E0C94EB2D80E0E6
:103E200090E0A0E2B1E489839A83AB83BC8318A2BB
:103E300019A21AA21BA21CA21DA21EA21FA280913F
:103E4000C40F882359F020E0AE014F5F5F4FBE01E1
:103E5000605E7F4FCE0184960E941E9480915B101D
:103E6000882319F081E080935A100E94CDF50C94BC
:103E7000EB2D10925A100E94EFF584E193E090939D
:103E8000FA048093F9040E946A5B0C94EB2D8091F4
:103E90005B10882311F40C94EB2D83E50E94C45C25
:103EA00081110C94902E0C94EB2D83E40E947B5C8A
:103EB000882309F450C0E6E4F3E084918F010F5F9A
:103EC0001F4F882321F00E94EA5CF801F6CF809111
:103ED0004C12811103C0E9E1F3E012C0BE016F5F33
:103EE0007F4F89E492E10E94F96F8E010F5F1F4FAF
:103EF000F80181918F01882349F10E94EA5CF8CF93
:103F000084918F010F5F1F4F882301F10E94EA5CAB
:103F1000F801F6CF74ECC72E73E0D72EE12CF12C0C
:103F200020E08091C40790E00E2C02C09595879503
:103F30000A94E2F780FD99C29FEFE91AF90AE2E0DC
:103F4000CE0ED11CF5E0EF16F10459F78AE00E947D
:103F5000EA5C0C94EB2D80915B10882339F0809102
:103F60005A10882319F0E3E2F3E003C0E5E3F3E03D
:103F700028C084918F010F5F1F4F882321F00E947A
:103F8000EA5CF801F6CF6091FA127091FB12809111
:103F9000FC129091FD124AE00E94855F8FE20E9420
:103FA000EA5C6091F6127091F7128091F81290918C
:103FB000F9124AE00E94855F8AE00E94EA5C0C9454
:103FC000EB2D84918F010F5F1F4F882311F40C9408
:103FD000EB2D0E94EA5CF801F4CF40E060E08091B4
:103FE000A0139091A1130E94EC8E0C94EB2D809164
:103FF0005B10882311F40C94EB2D89E492E10F946B
:104000007D1F89E492E10E94D46F109259101092A2
:10401000581080915B10882311F40C94EB2D0091C3
:10402000A0131091A1130F943505B801CE0180960D
:104030000F9449078C01892B11F40C94EB2D68A186
:1040400079A16115710511F06C5F7F4F19821C8297
:1040500022E0A801CE0101960E949677811102C04C
:10406000F12C14C0CE0101960F94A3048823C1F350
:1040700061E0CE0101960E94DD6F009789F325EE85
:10408000FC0120831C820F94261DF82ECE01019680
:104090000E94D05CF11003C0E3E6F3E022C0E5E546
:1040A000F3E084917F012FEFE21AF20A882321F0D6
:1040B0000E94EA5CF701F5CFF80181918F01882316
:1040C00019F00E94EA5CF8CF8AE00E94EA5C109244
:1040D000FA121092FB121092FC121092FD120C9424
:1040E000EB2D84917F012FEFE21AF20A882321F051
:1040F0000E94EA5CF701F5CFF80181918F018823D6
:1041000019F00E94EA5CF8CF8EE20E94EA5C0C94FF
:10411000EB2D80915A1081110E94C6B980915B10DD
:10412000882311F40C94EB2D80E50E94C45C882355
:1041300019F00E94395C03C080E50E947B5C182F57
:10414000482F61E08091A0139091A1130E94EC8E02
:1041500083E50E94C45C882381F00E94185CAB0157
:10416000BC014093FA125093FB126093FC127093BF
:10417000FD1289E492E10F94AF1F80915B108823B8
:1041800019F081E080935A1011110C94EB2D6DCE33
:104190008091A0139091A11321E02093591040E049
:1041A00060E00E94EC8E0C94EB2D0E947EF57B016A
:1041B0008C0120E831E541E050E00F944B49C90102
:1041C0006DE671E00F94A94C4B015C01C801B70189
:1041D00020E13EE040E050E00F944B49CA01B901B4
:1041E00028E130E040E050E00F944B49762E672EF6
:1041F000C62ED72EECE32E2E312C412C512CC8018B
:10420000B701A20191010F944B49F62EE72ECA0186
:10421000B901A20191010F944B49CB018E010F5FAF
:104220001F4F8114910499F0EF92FF927F936F9347
:104230006F927F92BF92AF929F928F9283EA93E0A8
:104240009F938F931F930F930F94F74413C0A11460
:10425000B104B1F0EF92FF927F936F936F927F92D0
:10426000BF92AF9283E993E09F938F931F930F9335
:104270000F94F7440FB6F894DEBF0FBECDBF30C029
:10428000CD2879F0EF92FF927F936F936F927F9298
:1042900087E893E09F938F931F930F930F94F744B6
:1042A000E9CF892B69F0EF92FF927F936F938FE7AD
:1042B00093E09F938F931F930F930F94F744DACF5C
:1042C000EF92FF928BE793E09F938F931F930F934F
:1042D0000F94F7440F900F900F900F900F900F9046
:1042E00060E0C8010E94098AE9E4FFE284917F014D
:1042F0003FEFE31AF30A882321F00E94EA5CF701FA
:10430000F5CFB80187EB93E00E9421C28AE00E94BA
:10431000EA5C0C94EB2D83E50E94C45C882311F4C5
:104320000C94EB2D0E94285CE82E80E50E94C45C72
:10433000882339F00E94285C182F87FF03C00C9453
:10434000EB2D1DE089E40E94C45C882341F00E94AB
:10435000395C81110C94FD2EE3E2F6E00BC089E498
:104360000E947B5CF6CF319686E0E035F80711F4C9
:104370000C94FD2E84911813F6CF0C94FA2E0E9403
:10438000CDF50C94EB2D0E9404F60C94EB2D88E6F1
:1043900090E00E94255781110C94EB2D8091C40769
:1043A00083FF02C00C94EB2D83E50E94C45C88233C
:1043B000A9F00E94485C0F94CB4ACB010E946E8901
:1043C0000E94485C20E030E04AEA52E40F945D45E8
:1043D000181624F00E9404F60F94A8170E943CC2FD
:1043E0000C94EB2D8EE40E94C45C882311F40C9491
:1043F000EB2D0E94185C6093BE077093BF078093FB
:10440000C0079093C1070C94EB2D83E50E947B5C61
:10441000882359F083E50E94C45C882319F00E9428
:10442000285C01C080E08093C407E9E4FFE2849146
:104430008F010F5F1F4F811103C0E2EDF3E004C055
:104440000E94EA5CF801F3CF84918F010F5F1F4F48
:10445000882321F00E94EA5CF801F6CF8091C4071E
:10446000811158CDEEECF3E018C0BB24B394B20E2A
:10447000222319F08CE20E94EA5CF6018591949166
:10448000FC0184918F010F5F1F4F882321F00E9450
:10449000EA5CF801F6CF2B2D4FCD84918F010F5F91
:1044A0001F4F882309F452CD0E94EA5CF801F5CF32
:1044B00010921A020C94EB2D89ED93E00E94C560D6
:1044C0000E94C5CE0C94EB2D83E50E94C45C811143
:1044D00003C0E9E4FFE20DC00E94285C8D3320F4A4
:1044E000809300020C94EB2D8CE3809300020C94DB
:1044F000EB2D84918F010F5F1F4F882321F00E94C5
:10450000EA5CF801F6CF4091000250E060E070E014
:1045100082EE93E00E94CEC18AE00E94EA5C0C9495
:10452000EB2D89E690E00E942557811111C0E9EE3C
:10453000F3E084918F010F5F1F4F882321F00E94C9
:10454000EA5CF801F6CF0E9408CB8AE00E94EA5CA0
:1045500010922E050C94122F83E50E94C45C8823D0
:1045600011F40C94EB2D0E94285C182F8D3308F069
:104570001CE310936F040F94EF106B017C01212F4B
:1045800030E0A8EEB3E00F947749C60ED71EE81EC0
:10459000F91EC0926B04D0926C04E0926D04F0920C
:1045A0006E040C94EB2D0F94AD230C94EB2D8091A5
:1045B000C40783FF02C00C94EB2D83E50E94C45C0A
:1045C000882311F40C94EB2D0E94485C0F94CB4A85
:1045D0006837710514F068E770E070937E1360939C
:1045E0007D130E94BFF30C94EB2D0F94D3210C94F8
:1045F000EB2D80E50E94C45C811106C083E50E941A
:10460000C45C882361F006C00E94285C81110C9470
:10461000EB2DF4CF0E94185C6F3F710510F06FEF27
:1046200070E07093801360937F130C94EB2D80E502
:104630000E94C45C811106C01092801310927F13F7
:104640000C94EB2D0E94185C672B11F00C94EB2D51
:10465000F3CF8CE40E947B5C882361F00E94485C6D
:104660006B017C0120E030E0A9010F94FB4B87FF38
:104670000BC006C0C12CD12C60E8E62E61ECF62EF2
:10468000F7FAF094F7F8F094F7FAF094F7F8F0945A
:10469000CCA2DDA2EEA2FFA280E090E0A4EDB2ECFD
:1046A00089839A83AB83BC8380E090E0A4EDB2E47D
:1046B0008D839E83AF83B88780E090E0A0EFB1E464
:1046C00089879A87AB87BC8788E50E94C45C88236A
:1046D00079F088E50E94C45C882319F00E94485C48
:1046E00003C060E070E0CB0169837A838B839C8395
:1046F00089E50E94C45C882379F089E50E94C45C46
:10470000882319F00E94485C03C060E070E0CB0190
:104710006D837E838F8398878AE50E94C45C88239B
:1047200079F08AE50E94C45C882319F00E94485CF5
:1047300003C060E070E0CB0169877A878B879C8734
:1047400018A219A21AA21BA220E0AE01405E5F4F80
:10475000BE016F5F7F4FCE0184960F94AE270C94FD
:10476000EB2D109253030C94EB2D81E080935303B7
:104770000C94EB2D83E50E94C45C8823A1F00E9479
:10478000485C20E030E04AE754E40F94C2450F94BF
:10479000D04A60935F0470936004809361049093A7
:1047A00062040C94EB2D88E50E947B5C81110C94D3
:1047B000A12E89E50E947B5C81110C94A12E8AE5D3
:1047C0000E947B5C81110C94A12E85E40E947B5C8D
:1047D00081110C94A12E0E9404BA0C94EB2D83E558
:1047E0000E947B5C882311F40C94EB2D0E94485CA2
:1047F00020E030E04AE754E40F94C2450F94D04AD9
:1048000060936704709368048093690490936A04CA
:104810000C94EB2DF60181916F010E947B5C882343
:1048200009F46DC0133009F063C00E94485C4B016D
:104830005C0120E030E040EA51E40F945D4587FFE1
:104840004EC0A501940160919105709192058091EF
:104850009305909194050F94634A2B013C019B01B1
:10486000AC01609141137091421380914313909178
:1048700044130F94C2456093411370934213809385
:10488000431390934413A301920160911913709103
:104890001A1380911B1390911C130F94C2456093BF
:1048A000191370931A1380931B1390931C13609128
:1048B000DA077091DB078091DC079091DD070F9498
:1048C0006145A30192010F94C2450F94D04A6093B1
:1048D000DA077093DB078093DC079093DD07809203
:1048E000910590929205A0929305B092940507C00D
:1048F0000E94485CF70160837183828393831F5F0A
:10490000F4E0EF0EF11C143009F084CF0E94C7C20E
:104910000C94EB2D84918F010F5F1F4F882321F0A2
:104920000E94EA5CF801F6CF60E08EEC94E00E9411
:1049300049D461E087EC94E00E9449D461E08CEBBB
:1049400094E00E9449D461E08CEA94E00E9449D44A
:1049500060E083EA94E00E9449D461E089E994E050
:104960000E9449D461E08FE894E00E9449D461E05C
:1049700087E894E00E9449D461E089E794E00E94CE
:1049800049D460E08BE694E00E9449D460E08CE575
:1049900094E00E9449D460E08EE494E00E9449D4FF
:1049A00060E088E394E00E9449D460E087E294E00C
:1049B0000E9449D460E082E194E00E9449D461E021
:1049C0008FEF93E00E9449D40C94EB2D8091A013BB
:1049D0009091A113FC012081222329F060E00E9424
:1049E000098A0C94EB2D0F94A8170C94EB2DF80169
:1049F0009081292F2B7F213419F08150C1F716C0E7
:104A000021812133D1F7913421F0953421F441E013
:104A100002C0DD24D39498012E5F3F4F89012F5FA0
:104A20003F4FF80190819032C9F3E7CF442369F0FA
:104A3000E9E4FFE284917F012FEFE21AF20A882372
:104A400021F00E94EA5CF701F5CFDD2069F0E7EA8A
:104A5000F5E084917F013FEFE31AF30A882321F008
:104A60000E94EA5CF701F5CFF80181918F0188235C
:104A700009F46CCA0E94EA5CF7CF0F94632D0C9482
:104A8000EB2D81E08093800D80937F0D0C94EB2DB6
:104A90001092800D10927F0D0C94EB2D83E50E94F7
:104AA000C45C882319F00E94185C02C060E070E0CA
:104AB0008B01112702301105DCF0E8E7F1E1849168
:104AC0008F010F5F1F4F811103C0EBEAF5E004C0B7
:104AD0000E94EA5CF801F3CF84918F010F5F1F4FB2
:104AE000882311F40C94EB2D0E94EA5CF801F4CFBA
:104AF00088E40E94C45C8823A9F00E94185C6A3A8A
:104B000071053CF06530F1E07F072CF064E071E066
:104B100002C06AEA70E0F801EE0FFF1FEF5CF04F91
:104B20007183608386E40E94C45C8823A9F00E949C
:104B3000185CF801EE0FFF1FEB5CF04F7183608390
:104B40006F3F710519F014F06FEF70E077FF02C04E
:104B500060E070E07183608382E40E94C45C88231B
:104B600011F40C94EB2D0E94185C6530710534F043
:104B70006A3671052CF069E670E002C065E070E00D
:104B8000000F111FF801E35DF04F718360830C94F7
:104B9000EB2D88EC90E00E94255781110C94EB2DB1
:104BA00084E40E947B5C882309F441C00E94485C35
:104BB0006B017C0111E020E030E0A9010F945D451C
:104BC000811101C010E01093700D20E030E0A901C8
:104BD000C701B6010F945D45882349F10E94485CE6
:104BE000E0910B0D24E0E29FF0011124E459F24F13
:104BF000608371838283938320E030E0A901609118
:104C00006C0D70916D0D80916E0D90916F0D0F94E4
:104C10005D4581110CC080E090E0A0EEBFE3809381
:104C20006C0D90936D0DA0936E0DB0936F0D0F945E
:104C30008328D1C7F70181917F010E947B5C882383
:104C400049F00E94485C0F94D04AF8016083718358
:104C5000828393830C5F1F4FC016D10659F70E94C1
:104C60006CC2B9C7B7E5EB2EB2E0FB2E0DE013E145
:104C7000F70181917F010E947B5C882339F00E94BB
:104C8000485CF80160837183828393830C5F1F4FBC
:104C9000F3E10D311F0761F79EC783E50E94C45CF5
:104CA0008823A1F00E94485C609331137093321303
:104CB000809333139093341360932D1370932E13BA
:104CC00080932F139093301310E001C011E080E522
:104CD0000E94C45C882359F00E94485C60933113A1
:104CE00070933213809333139093341310E082E562
:104CF0000E94C45C882359F00E94485C6093290597
:104D000070932A0580932B0590932C0510E084E581
:104D10000E94C45C882359F00E94485C60932D1364
:104D200070932E1380932F139093301354C7112335
:104D300009F451C7409131135091321360913313EC
:104D40007091341383ED95E00E94EBC140912905E9
:104D500050912A0560912B0570912C0580ED95E00E
:104D60000E94EBC140912D1350912E1360912F138F
:104D7000709130138DEC95E00E94EBC18AE00E94A7
:104D8000EA5C29C782E40E947B5C882351F00E9480
:104D9000085C6093C00F7093C10F8093C20F909313
:104DA000C30F83E50E947B5C882351F00E94485C1E
:104DB0006093091370930A1380930B1390930C1351
:104DC00084E50E947B5C882351F00E94485C6093DC
:104DD000051370930613809307139093081388E5C7
:104DE0000E947B5C882351F00E94485C60933513DD
:104DF00070933613809337139093381389E50E948C
:104E00007B5C882351F00E94485C60933913709357
:104E10003A1380933B1390933C138AE50E947B5C8A
:104E2000882351F00E94485C60933D1370933E13B9
:104E300080933F139093401385E40E947B5C88230A
:104E400009F4C9C60E94485C6093411370934213F1
:104E50008093431390934413BEC684918F010F5FD8
:104E60001F4F882321F00E94EA5CF801F6CF83E50A
:104E70000E947B5C882321F00E94395C8093390278
:104E8000EBE0F6E084918F010F5F1F4F882321F044
:104E90000E94EA5CF801F6CF80913902882319F06C
:104EA000E3E0F6E002C0E7E0F6E084918F010F5FF7
:104EB0001F4F811103C0EBEFF5E004C00E94EA5CD4
:104EC000F801F3CF84918F010F5F1F4F882321F0EA
:104ED0000E94EA5CF801F6CF20910D0F30910E0F81
:104EE00040910F0F5091100F60912702709128028E
:104EF0008091290290912A020F948749AB01BC014D
:104F000089EF95E00E94EBC12091110F3091120FB3
:104F10004091130F5091140F60912B0270912C024D
:104F200080912D0290912E020F948749AB01BC0114
:104F300086EF95E00E94EBC12091150F3091160F7E
:104F40004091170F5091180F60912F02709130020D
:104F500080913102909132020F948749AB01BC01DC
:104F600083EF95E00E94EBC1EBEEF5E084918F01B9
:104F70000F5F1F4F882321F00E94EA5CF801F6CFF3
:104F800020910D0F30910E0F40910F0F5091100F87
:104F900060911B0270911C0280911D0290911E0273
:104FA0000F948749AB01BC0189EE95E00E94EBC1EB
:104FB0002091110F3091120F4091130F5091140F47
:104FC00060911F0270912002809121029091220233
:104FD0000F948749AB01BC0186EE95E00E94EBC1BE
:104FE0002091150F3091160F4091170F5091180F07
:104FF00060912302709124028091250290912602F3
:105000000F948749AB01BC0183EE95E00E94EBC190
:105010008AE00E94EA5CDFC583E50E94C45C8823C5
:1050200009F4D9C50E94185C709353026093520230
:10503000D2C58DED90E00E9425578111CCC583E546
:105040000E94C45C811103C0E9E4FFE23AC0009110
:105050000B0D10E00E94185C000F111FF801E05BBF
:10506000FD4F7183608380910B0D90E08C01000FE8
:10507000111F000F111F9801245B3D4F7901880F0C
:10508000991FFC01E05BFD4F60817181072E000CD0
:10509000880B990B0F9463452AE037ED43E25CE3FC
:1050A0000F94C245F801E15BFC4E208131814281C1
:1050B00053810F94C245F701608371838283938388
:1050C0008AC584918F010F5F1F4F882321F00E94B2
:1050D000EA5CF801F6CF85E40E94EA5C80910B0D52
:1050E000805D0E94EA5CE0910B0DF0E0EE0FFF1F87
:1050F000E05BFD4F608171818BE196E00E9408C208
:1051000085E20E94EA5C8AE00E94EA5C64C580E570
:105110000E947B5C882309F45EC50E94185C6B01C9
:105120007C0183E50E94C45C882321F00E94185C06
:105130008B0102C00FEF1FEFC8010196039708F023
:105140004AC5D7FC48C58C2DE3E2F6E09491891757
:1051500009F450C6319626E0E035F207B9F721C6CA
:1051600083E50E94C45C882319F00E94185C02C089
:1051700064E071E079A368A380E50E94C45C8823A1
:1051800039F00E94185C693833E1730730F402C0CB
:1051900068EE73E07A83698304C088E893E19A83B8
:1051A0008983BE01605E7F4FCE0101960E941292FC
:1051B00012C585E40E94C45C811110C080E50E9484
:1051C0007B5C882391F00E94485C6093200F709371
:1051D000210F8093220F9093230F07C00E94285C19
:1051E000882361F3E8E7F1E171C089E40E947B5C08
:1051F000882381F00E94485C2CEA35EC47E25EE3AC
:105200000F94C2456093280F7093290F80932A0F43
:1052100090932B0F84E40E947B5C882381F00E9492
:10522000485C2CEA35EC47E25EE30F94634A6093F6
:10523000240F7093250F8093260F9093270FE9E496
:10524000FFE284918F010F5F1F4F882321F00E949E
:10525000EA5CF801F6CF4091200F5091210F609148
:10526000220F7091230F88E596E00E94EBC12CEA93
:1052700035EC47E25EE36091280F7091290F809131
:105280002A0F90912B0F0F94634AAB01BC0184E568
:1052900096E00E94EBC12CEA35EC47E25EE36091B8
:1052A000240F7091250F8091260F9091270F0F9456
:1052B000C245AB01BC0180E596E00E94EBC18AE0EB
:1052C0000E94EA5C88C40E94EA5CF80184918F0124
:1052D0000F5F1F4F8111F7CFECE5F6E084918F014E
:1052E0000F5F1F4F882309F476C40E94EA5CF8011F
:1052F000F5CF83E50E947B5C182F882371F00E9414
:10530000485C0F94CB4A709308026093070221E037
:10531000672B09F020E02093220580E50E947B5C4A
:10532000882359F02091070230910802232B11F0B5
:105330000E94395C809322054EC411114CC4E9E4EB
:10534000FFE284918F010F5F1F4F882321F00E949D
:10535000EA5CF801F6CF80912205882319F062E417
:1053600073E002C065E173E083E896E00E9421C229
:10537000609107027091080282E796E00E9408C2DD
:10538000EEE6F6E084918F010F5F1F4F882309F44A
:1053900022C40E94EA5CF801F5CF80E50E947B5CA4
:1053A000882351F00E94485C6093580F7093590F06
:1053B00080935A0F90935B0F89E40E947B5C882353
:1053C00081F00E94485C2CEA35EC47E25EE30F94E2
:1053D000C2456093540F7093550F8093560F90936E
:1053E000570F84E40E947B5C882381F00E94485C14
:1053F0002CEA35EC47E25EE30F94634A6093500F6A
:105400007093510F8093520F9093530FE9E4FFE292
:1054100084918F010F5F1F4F882321F00E94EA5C67
:10542000F801F6CF4091580F5091590F60915A0FE3
:1054300070915B0F8EE996E00E94EBC12CEA35EC8F
:1054400047E25EE36091540F7091550F8091560FC3
:105450009091570F0F94634AAB01BC018AE996E023
:105460000E94EBC12CEA35EC47E25EE36091500FFD
:105470007091510F8091520F9091530F0F94C2452C
:10548000AB01BC0186E996E00E94EBC18AE00E9474
:10549000EA5CA1C30E94EA5CF80184918F010F5F6E
:1054A0001F4F8111F7CFE2EAF6E084918F010F5F81
:1054B0001F4F882309F48FC30E94EA5CF801F5CFDF
:1054C0000E94C6B988C381E00E94DC520E9480D449
:1054D00082C383E50E947B5C882349F00E94395C8B
:1054E000182F811106C080E00E94FC4A02C0109172
:1054F000370D8091950590919605A0919705B091F3
:10550000980589839A83AB83BC8380919905909198
:105510009A05A0919B05B0919C058D839E83AF83D6
:10552000B88780919D0590919E05A0919F05B091AF
:10553000A00589879A87AB87BC8786E50E947B5C3C
:10554000882321F08EED96E00F945A37812F0E9428
:10555000FC4A111103C0E9E4FFE21DC08091370D40
:105560008111F9CFE8E7F1E184918F010F5F1F4FBF
:10557000811103C0EFEBF6E004C00E94EA5CF80181
:10558000F3CF84918F010F5F1F4F882321F30E9477
:10559000EA5CF801F6CF84918F010F5F1F4F8823DB
:1055A00021F00E94EA5CF801F6CF8091370D882344
:1055B00019F069E173E002C06DE173E081EB96E000
:1055C0000E9421C28AE00E94EA5C4CE050E065E95A
:1055D00075E0CE0101960F94064D892B09F4FBC2AC
:1055E0000E9480D4F8C20F949C03F5C20F94E60188
:1055F000F2C283E50E947B5C882321F00E94395C23
:1056000091E089270E948FFCE6C24093BB0F0E9465
:10561000A6781092BB0F882309F4DDC2E9E4FFE20B
:1056200084918F010F5F1F4F811103C0EBEFF6E0F4
:1056300004C00E94EA5CF801F3CF84918F010F5FF0
:105640001F4F882309F4C7C20E94EA5CF801F5CF16
:105650008BE592E00E9425578111BDC285E50E942D
:105660007B5C8823D9F100910B0D10E00E94485C0F
:105670006B017C0120E030E0A9010F94FB4B87FF18
:1056800004C0F7FAF094F7F8F094000F111F000F20
:10569000111FF801E859F24FC082D182E282F382F1
:1056A00000910B0D84E0089F800111240859124FCE
:1056B00020E030E046E154E4F801608171818281AC
:1056C00093810F94FB4B18164CF480E090E0A6E118
:1056D000B4E4F80180839183A283B3838CE40E94B5
:1056E0007B5C882309F477C200910B0D10E00E94C7
:1056F000485C6B017C0120E030E0A9010F94FB4B7A
:1057000087FF04C0F7FAF094F7F8F094000F111F28
:10571000000F111FF801EC59F24FC082D182E282D2
:10572000F38200910B0DF4E00F9F800111240C59BE
:10573000124F20E030E046E154E4F80160817181CD
:10574000828193810F94FB4B18160CF044C280E0C9
:1057500090E0A6E1B4E4F80180839183A283B3834F
:105760003AC288E40E947B5C882351F00E94485C26
:1057700060935C0D70935D0D80935E0D90935F0D53
:105780008CE40E947B5C882351F00E94485C60930B
:105790003C0D70933D0D80933E0D90933F0D82E53F
:1057A0000E947B5C882351F00E94485C60934C0D02
:1057B00070934D0D80934E0D90934F0D83E50E9495
:1057C0007B5C882351F00E94485C6093BC0F70930F
:1057D000BD0F8093BE0F9093BF0F82E40E947B5C4D
:1057E000882351F00E94485C6093380D7093390D06
:1057F00080933A0D90933B0D88E50E947B5C882353
:1058000051F00E94485C6093400D7093410D80936D
:10581000420D9093430D89E50E947B5C882351F0F3
:105820000E94485C6093440D7093450D8093460D33
:105830009093470D8AE50E947B5C882351F00E947B
:10584000485C6093480D7093490D80934A0D909386
:105850004B0D0E944A6EBFC10E94485C20E030E0C0
:10586000A9010F945D4518163CF00E94485CF801B0
:1058700060837183828393830C5F1F4FC016D106B0
:1058800009F4A9C1F70181917F010E947B5C882303
:1058900099F3E2CF0E948BCB9EC141E061E081E0B1
:1058A0000E94474B811107C0812C912C90EFA92EAB
:1058B00091E4B92E03C0812C912C54018EEB92E01F
:1058C0000E942557811187C18AE50E94C45C882304
:1058D00069F08AE50E94C45C882329F00E94485C34
:1058E0004B015C0103C0812C912C540140910B0DA4
:1058F00062E081E00E9427AB20E030E0A901C50111
:10590000B4010F94FB4B18167CF580E090E0A8ECF6
:10591000B2E489839A83AB83BC8320919D05309147
:105920009E0540919F055091A005C501B4010F94BB
:1059300087496B017C0120E030E040EA53E40F949A
:105940005D4587FD06C0C12CD12C80EAE82E83E49A
:10595000F82EC8A2D9A2EAA2FBA2BE016F5F7F4FB8
:10596000CE0180960E94BD5285E50E947B5C882313
:1059700029F00E94485C6B017C010CC0E0910B0D8A
:1059800024E0E29FF0011124E859F24FC080D18059
:10599000E280F38020E030E0A901C701B6010F9456
:1059A000FB4B87FF04C0F7FAF094F7F8F094F7FA8E
:1059B000F094F7F8F094C982DA82EB82FC8242E03C
:1059C00061E0CE0101960F941D2720E030E0A9018F
:1059D000C501B4010F94FB4B18165CF580E090E014
:1059E000A8ECB2E489839A83AB83BC83A5019401BC
:1059F00060919D0570919E0580919F059091A005F5
:105A00000F9486496B017C0120E030E0A9010F94DE
:105A1000FB4B18161CF0C12CD12C7601C8A2D9A2C0
:105A2000EAA2FBA2BE016F5F7F4FCE0180960E946B
:105A3000BD5240912F0560E087E00E9427ABCBC0AC
:105A40008AE50E94C45C811103C0E9E4FFE23BC027
:105A50000E94485C6B017C0120E030E040EF51EC9B
:105A60000F94FB4B87FD0AC020E030E040EF51E48B
:105A7000C701B6010F945D4518161CF4E8E7F1E183
:105A80000CC0C092600DD092610DE092620DF09258
:105A9000630DA1C00E94EA5CF80184918F010F5F41
:105AA0001F4F8111F7CFE6E0F7E084918F010F5F80
:105AB0001F4F882309F48FC00E94EA5CF801F5CFDC
:105AC0000E94EA5CF80184918F010F5F1F4F8111E2
:105AD000F7CFE6E2F7E084918F010F5F1F4F882335
:105AE00021F00E94EA5CF801F6CF4091600D5091E0
:105AF000610D6091620D7091630D83E297E00E94E9
:105B0000EBC18AE00E94EA5C66C081E080934802B3
:105B10001092740583E50E94C45C882339F00E94CA
:105B2000395C811158C00E945A6F55C083E50E94AC
:105B30007B5CF7CF0E9432954EC0F090A2130E947A
:105B4000C6B91091370D80E00E94FC4AFF2029F170
:105B5000E9E4FFE284918F010F5F1F4F882321F05A
:105B60000E94EA5CF801F6CF84E50E94EA5C6F2DA2
:105B700070E080E090E04AE00E94855F80E20E9451
:105B8000EA5CE7E4F7E084918F010F5F1F4F882301
:105B900011F10E94EA5CF801F6CF10922F05812FD7
:105BA0000E94FC4AE9E4FFE284918F010F5F1F4FDE
:105BB000882321F00E94EA5CF801F6CF60912F055E
:105BC00070E085E397E00E9408C28AE00E94EA5CE8
:105BD00002C00E94329510922E050E943D6F22C194
:105BE0000E94BD490E940A69F6CF80E00E94FC4AEB
:105BF0000E947C5285E40E94C45C882321F00E94AC
:105C0000395C182F04C085E40E947B5C11E086E5B6
:105C10000E94C45C882321F00E94185C262F01C0DA
:105C200021E001E0412FBE016F5F7F4FCE018096E2
:105C30000E947D536B017C019B01AC010F94814C50
:105C400081115FC088A099A0AAA0BBA020E030E08D
:105C5000A901C501B4010F945D4587FF05C027E187
:105C600037EB41E558EB04C027E137EB41E558E35A
:105C7000C501B4010F948749AB01BC0180ED92E0EE
:105C80000E94EBC189809A80AB80BC8020E030E02C
:105C9000A901C501B4010F945D4587FF05C027E147
:105CA00037EB41E558EB04C027E137EB41E558E31A
:105CB000C501B4010F948749AB01BC018BEC92E0A4
:105CC0000E94EBC120E030E0A901C701B6010F94AA
:105CD0005D4587FF05C027E137EB41E558EB04C080
:105CE00027E137EB41E558E3C701B6010F94874937
:105CF000AB01BC0186EC92E00E94EBC18AE00E94FD
:105D0000EA5C0E9463520E9480D465CF11110C940A
:105D1000621E0C945B1E80E00E9415610C94841E30
:105D20000E94185CAB01BC014093FA125093FB1225
:105D30006093FC127093FD1289E492E10F94AF1FFF
:105D40004ACF0E94C6B988E50E947B5C882331F067
:105D50005F9A8091810D8E7F8093810D89E50E94ED
:105D60007B5C882331F08A9A8091810D8D7F8093AE
:105D7000810D8AE50E947B5C882359F0809108019F
:105D800080958170809306018091810D8B7F809337
:105D9000810D85E40E947B5C882309F41CCF129A54
:105DA0001ACF0E94C6B9BC2C60E08C2D0F94B30FA3
:105DB0000F3F3FEF130759F48C2D0E9409E331E0A8
:105DC00020E0892B09F030E0032F122F05C00130AD
:105DD000110569F401E010E08B2D0E9409E38017A2
:105DE000910709F4F8CE80E00E941561F5CF00E03C
:105DF00010E0F2CF0F94483FEECE61E0812F0F9478
:105E0000B30F6E2D812F0E9432E3F12CB701812F49
:105E10000F94EF0F193009F0DECEF0928013E0926C
:105E20007F13D9CEA7960FB6F894DEBF0FBECDBFB5
:105E3000DF91CF911F910F91FF90EF90DF90CF9066
:105E4000BF90AF909F908F907F906F905F904F909A
:105E50003F902F9008952F923F924F925F926F92B2
:105E60007F928F929F92AF92BF92CF92DF92EF92EA
:105E7000FF920F931F93CF93DF93CDB7DEB7C4503C
:105E8000D1400FB6F894DEBF0FBECDBF83E50E94B0
:105E90007B5CC556DF4F8883CB59D04081110DC044
:105EA00080E50E94C45C882319F00E94185C01C040
:105EB00064E0AE966FAFAE9704C022E0AE962FAF0F
:105EC000AE97AE968FADAE978F5F8C3070F0E5E4F5
:105ED000F9E084918F010F5F1F4F882311F40C9418
:105EE00051470E94EA5CF801F4CF84E50E947B5C94
:105EF000C456DF4F8883CC59D040C556DF4F8881C8
:105F0000CB59D040811126C083E40E94C45C882311
:105F100011F40C9414470E94485CC555DF4F688308
:105F200079838A839B83CB5AD04020E030E0A9015B
:105F30000F945D4587FF1AC0E5E1F9E084918F0178
:105F40000F5F1F4F882311F40C9451470E94EA5CA5
:105F5000F801F4CF80E090E0A0E8BFE3C555DF4F43
:105F600088839983AA83BB83CB5AD04086E40E945E
:105F7000C45C882361F00E94185CC654DF4F6883BC
:105F8000CA5BD0406F31A8F0E8EEF8E006C0C65416
:105F9000DF4F1882CA5BD0400CC084918F010F5F25
:105FA0001F4F882311F40C9451470E94EA5CF801BA
:105FB000F4CF86E50E94C45C8823B9F00E94285C77
:105FC000C756DF4F8883C959D0408430A0F0EEEB2C
:105FD000F8E084918F010F5F1F4F882311F40C9418
:105FE00051470E94EA5CF801F4CF91E0C756DF4FB9
:105FF0009883C959D04085E40E947B5CC154DF4F2F
:106000008883CF5BD040C556DF4FA881CB59D040A5
:10601000AA2341F18CE59FEFA9E7B4E480935C0DDE
:1060200090935D0DA0935E0DB0935F0D80E090E0C6
:10603000A8EEB2E480934C0D90934D0DA0934E0DBD
:10604000B0934F0D8CE0E0E5FDE0DF01282F1D92BD
:106050002A95E9F7E0E4FDE0DF011D928A95E9F772
:106060000E944A6E81E0C456DF4FB881CC59D040BF
:10607000B827C854DF4FB883C85BD040AE96EFADA9
:10608000AE97E13009F469C0F1E0C155DF4FF88304
:10609000CF5AD040EF3FE1F0C155DF4F1882CF5AC1
:1060A000D040E23011F00C941E47C456DF4F2881D7
:1060B000CC59D04021111DC0C656DF4F1882CA5995
:1060C000D040C356DF4FB883CD59D04010E02AC02E
:1060D000C656DF4F1882CA59D040C356DF4F1882C8
:1060E000CD59D04010E0AE969FADAE979F3FD1F412
:1060F00045C0C854DF4FA881C85BD040AA2311F423
:106100000C944647C456DF4FA881CC59D040C656A0
:10611000DF4FA883CA59D040C356DF4FA883CD595B
:10612000D0401A2FB1E0C754DF4FB883C95BD040CD
:10613000AE96EFADAE97EE2309F1AE96FFADAE97FA
:10614000F3300CF1C854DF4F2881C85BD040C655EE
:10615000DF4F2883CA5AD0401BC0C656DF4F188273
:10616000CA59D040C356DF4F1882CD59D04010E0F5
:10617000B1E0C155DF4FB883CF5AD040C754DF4F8D
:106180001882C95BD040C655DF4F1882CA5AD0402A
:10619000C756DF4F8881C959D040C256DF4F188299
:1061A000CE59D040882399F090ECC156DF4F9883A8
:1061B000CF59D040A9E7C056DF4FA883C05AD0407E
:1061C000B4E4CF55DF4FB883C15AD0400FC0C15699
:1061D000DF4F1882CF59D040C056DF4F1882C05AC7
:1061E000D040CF55DF4F1882C15AD0408091500D1A
:1061F0009091510DA091520DB091530DC352DF4FAC
:1062000088839983AA83BB83CD5DD0408091540D50
:106210009091550DA091560DB091570DCB52DF4F77
:1062200088839983AA83BB83C55DD0408091580D34
:106230009091590DA0915A0DB0915B0DC353DF4F52
:1062400088839983AA83BB83CD5CD04080914C0D19
:1062500090914D0DA0914E0DB0914F0DCF53DF4F4A
:1062600088839983AA83BB83C15CD04080915C0DF5
:1062700090915D0DA0915E0DB0915F0DCB53DF4FFE
:1062800088839983AA83BB83C55CD0408091400DED
:106290009091410DA091420DB091430DC753DF4F36
:1062A00088839983AA83BB83C95CD0408091440DC5
:1062B0009091450DA091460DB091470DC752DF4F0B
:1062C00088839983AA83BB83C95DD0408091480DA0
:1062D0009091490DA0914A0DB0914B0DCF52DF4FD7
:1062E00088839983AA83BB83C15DD040EAEAF8E042
:1062F00084917F019FEFE91AF90A882321F00E9417
:10630000EA5CF701F5CFC155DF4FA881CF5AD040E5
:10631000A11173C0AE96BFADAE97BB2309F46DC09B
:106320008090380D9090390DA0903A0DB0903B0DB3
:10633000A2ED2A2E312CB101032C000C880B990BF5
:106340000F9463452BED3FE049E450E40F94C245C0
:1063500020E030E044E353E40F94634A6B017C0196
:106360000F94364C9B01AC01C501B4010F94C2459A
:106370002B013C01C701B6010F94604A9B01AC019F
:10638000C501B4010F94C2459B01AC010F94C245F5
:10639000E2966CAF7DAF8EAF9FAFE297A301920103
:1063A000C301B2010F94C2459B01AC01E2966CADF2
:1063B0007DAD8EAD9FADE2970F94874920E030E42C
:1063C00042E556E40F945D45181674F4E7E7F8E0EB
:1063D00084918F010F5F1F4F882311F40C94514754
:1063E0000E94EA5CF801F4CFECE32E0E311CFAE3D4
:1063F0002F16F2E03F0609F09ECFEBE9F8E084911A
:106400007F012FEFE21AF20A882321F00E94EA5C52
:10641000F701F5CFC756DF4F8881C959D0408111A8
:106420000DC0ECE6F8E084917F019FEFE91AF90ACC
:10643000882321F00E94EA5CF701F5CFC556DF4FB3
:10644000A881CB59D040AA2369F0E1E6F8E0849115
:106450007F01BFEFEB1AFB0A882321F00E94EA5C60
:10646000F701F5CF8AE00E94EA5C60E08BE998E0F2
:106470000E94CD89C655DF4F6881CA5AD040C754A3
:10648000DF4F8881C95BD0400F949C34AE96EFAD4E
:10649000AE97EE2341F001E0C155DF4FF881CF5AAE
:1064A000D0400F2701C000E00E94C6B90E947C5274
:1064B00001110E941A4BAE962FADAE972223A9F080
:1064C00081E08093800D0E9456A480917F0D80937F
:1064D000800DAE968FADAE9788303CF092E0C05400
:1064E000DF4F9883C05CD04005C0C054DF4F188296
:1064F000C05CD040112339F0A2E0CF51DF4FA88318
:10650000C15ED04006C0B1E0CF51DF4FB883C15E5D
:10651000D040AE96EFADAE97E23039F4F2E0CE5116
:10652000DF4FF883C25ED04006C021E0CE51DF4F7E
:106530002883C25ED040C256DF4FE880CE59D0409B
:10654000C156DF4FF880CF59D040C056DF4F088189
:10655000C05AD040CF55DF4F1881C15AD040CE55D8
:10656000DF4FE882C25AD040CD55DF4FF882C35A80
:10657000D040CC55DF4F0883C45AD040CB55DF4FB5
:106580001883C55AD040CC56DF4F1882C459D0402A
:10659000CE014D96AB969FAF8EAFAB97DE01D996ED
:1065A000AD96BFAFAEAFAD97C054DF4FE881C05CD2
:1065B000D0400E2E000CFF0BC150DF4FF983E88353
:1065C000CF5FD0404C971C01AE968FADAE97082E92
:1065D000000C990BAA0BBB0BCF5FDE4F888399830E
:1065E000AA83BB83C150D1408CE1AB96AEADBFADA9
:1065F000AB971D928A95E9F720E030EC49E754E427
:10660000B701C8010F945D45882399F19701A8014E
:10661000C256DF4F6881CE59D040C156DF4F7881D6
:10662000CF59D040C056DF4F8881C05AD040CF5597
:10663000DF4F9881C15AD0400F94874920E030E065
:1066400040E05FE30F94C245CB56DF4F6883C559E6
:10665000D040CA56DF4F7883C659D040C956DF4F65
:106660008883C759D040C856DF4F9883C859D04057
:1066700028C0C256DF4FB881CE59D040CB56DF4F2D
:10668000B883C559D040C156DF4FE881CF59D040BB
:10669000CA56DF4FE883C659D040C056DF4FF88155
:1066A000C05AD040C956DF4FF883C759D040CF55A4
:1066B000DF4F2881C15AD040C856DF4F2883C859C0
:1066C000D040CC56DF4F8881C459D0408F5FCC5624
:1066D000DF4F8883C459D040AE969FADAE9711E08E
:1066E000913071F09F3F61F010E0923049F4C45650
:1066F000DF4FA881CC59D040AF96AFAFAF9703C062
:10670000AF961FAEAF97FE017D9611921192119236
:106710001192AD968EAD9FADAD97E817F907A9F729
:10672000AE969FADAE97911111C0ACEAAF96AFAFE8
:10673000AF97B5ECE396BFAFE397E7E2E796EFAF2D
:10674000E797F7E3E896FFAFE8974DC4AE962FAD15
:10675000AE972330A1F4AE968FADAE9785508330BF
:1067600008F057C0C12CD12CE0ECEE2EE0E4FE2E58
:10677000812C912CF0E8AF2EFFE3BF2E66C0AE96C1
:106780008FADAE97863039F3AE96AFADAE97A930E8
:1067900009F44BC019821A821B821C8219AE1AAEF0
:1067A0001BAE1CAEC556DF4FB881CB59D040B111DE
:1067B00009C0C154DF4FE881CF5BD040EE2321F008
:1067C00041E003C043E001C042E000E020E0B1014D
:1067D000CE01C9960E947D532D8D3E8D4F8D58A1BF
:1067E0000F9487496D8F7E8F8F8F98A39B01AC018B
:1067F0000F94814C81110C940847AE96FFADAE9773
:10680000F3300CF4DDC0AE969FADAE9798306CF4CB
:10681000A2CFC12CD12C60EAE62E60E4F62E812CAA
:10682000912CA12C70E4B72E10C04BEAC42E4AEA7A
:10683000D42E4AECE42E40E4F42E5BEA852E5AEA8C
:10684000952E5AE2A52E5FE3B52E22E739EF4FE7EA
:106850005FE3C701B6010F94FB4B18160CF08EC016
:1068600020E030E040E85FE3C701B6010F948649BD
:1068700020E030E040E752E40F94C24520E030E0F1
:1068800042E553E40F9487492BED3FE049E450E49F
:106890000F94C24520E030E044E353E40F94634A90
:1068A0002B013C012DEC3CEC4CEC5DE36091380D90
:1068B0007091390D80913A0D90913B0D0F94C24526
:1068C000E6966CAF7DAF8EAF9FAFE697C301B20186
:1068D0000F94364C9B01AC01E6966CAD7DAD8EAD50
:1068E0009FADE6970F94C24569837A838B839C831F
:1068F000C301B2010F94604A9B01AC01E6966CADF6
:106900007DAD8EAD9FADE6970F94C24569AF7AAF6E
:106910008BAF9CAFC556DF4F2881CB59D04021119A
:1069200009C0C154DF4F8881CF5BD040882321F05C
:1069300041E003C043E001C042E000E020E0B101DB
:10694000CE01C9960E947D532D8D3E8D4F8D58A14D
:106950000F9487496D8F7E8F8F8F98A39B01AC0119
:106960000F94814C81110C940847A5019401C70133
:10697000B6010F9486496B017C0167CFCD8CDE8C0C
:10698000EF8CF8A0AE969FADAE97953069F0CF5FD3
:10699000DE4F688179818A819B81C150D1400F94FB
:1069A00063459B01AC0104C020E030E040EE50E4C0
:1069B000C701B6010F94634A6D8F7E8F8F8F98A3A6
:1069C0001111A5C2AF96AFADAF97AA2311F062E047
:1069D00001C061E0AE96BFADAE97BA3011F1B930EB
:1069E00071F1B830E9F1B73009F448C0B63009F4B4
:1069F00056C0B53009F464C0AF961FAEAF97E396AA
:106A00001FAEE397B43009F46CC0B33009F071C025
:106A1000E0E8E796EFAFE797FFE3E896FFAFE89788
:106A20006FC029E8AF962FAFAF9788E8E3968FAF96
:106A3000E39798E8E7969FAFE797ADE356C0BBEAC8
:106A4000AF96BFAFAF97EAEAE396EFAFE397FAEA04
:106A5000E796FFAFE7972DE3E8962FAFE89750C092
:106A600089E3AF968FAFAF979EE8E3969FAFE3972A
:106A7000A3EEE796AFAFE797BDE33FC0E5E2AF9681
:106A8000EFAFAF97F9E4E396FFAFE39722E1E79624
:106A90002FAFE7978EE3E8968FAFE89731C09DEC74
:106AA000AF969FAFAF97ACECE396AFAFE397BCE484
:106AB000E796BFAFE797EEE3E896EFAFE89720C021
:106AC000FBEAAF96FFAFAF972AEAE3962FAFE397C3
:106AD0008AEAE7968FAFE7979EE3E8969FAFE8973D
:106AE0000FC0E7961FAEE797AFE3E896AFAFE89722
:106AF00007C0E7961FAEE797B0E4E896BFAFE89708
:106B0000062E000C770B880B990B0F9463454B01F5
:106B10005C01E1E0E996EFAFE9972EE23FEF4FED40
:106B200050E4C501B4010F945D4587FFA5C120E085
:106B300030E040E85FE3C501B4010F94864920E0EE
:106B400030E040E752E40F94C24520E030E042E5F7
:106B500053E40F9487492BED3FE049E450E40F9450
:106B6000C24520E030E044E353E40F94634A6B01F4
:106B70007C0120E030E040E85FE3C501B4010F9400
:106B8000164BC058DF4F688379838A839B83C05834
:106B9000D040C701B6010F94364CC857DF4F688309
:106BA00079838A839B83C858D040C701B6010F946C
:106BB000604AC457DF4F688379838A839B83CC58AC
:106BC000D040ED961FAEED97E996FFADE997FF2314
:106BD00091F0C150DF4F68817981CF5FD040ED9651
:106BE0002FADED97621B710927FD7395072E000CE1
:106BF000880B990B08C0ED96AFADED976A2FAA0FE1
:106C0000770B880B990B0F9463452DEC3CEC4CEC07
:106C10005DE30F94C2459B01AC0160E070E080E849
:106C20009FE30F9486492091380D3091390D4091A2
:106C30003A0D50913B0D0F94C2456B017C01C85732
:106C4000DF4F288139814A815B81C858D0400F9439
:106C5000C24569837A838B839C83C457DF4F288125
:106C600039814A815B81CC58D040C701B6010F946D
:106C7000C24569AF7AAF8BAF9CAFC556DF4FB881C5
:106C8000CB59D040B11109C0C154DF4FE881CF5B6F
:106C9000D040EE2321F041E003C043E001C042E0D8
:106CA00000E020E0B101CE01C9960E947D536B0146
:106CB0007C019B01AC010F94814C81110C9408471D
:106CC000C058DF4F288139814A815B81C058D0404C
:106CD000C501B4010F9486492B013C0120E030E04E
:106CE00040EC50E40F94874920E030E040E85FE357
:106CF0000F9486490F94064C862F66E00F949D4CA6
:106D00000DE110E00C0F1D1FF4E09F9F000D111D01
:106D100011240C5F1F4F20E030E044EB52E4C058D8
:106D2000DF4F688179818A819B81C058D0400F9460
:106D3000C2452BED3FE049E450E40F94C24520E00A
:106D400030E044E353E40F94634ACC57DF4F688349
:106D500079838A839B83C458D0400F94604A9B01F7
:106D6000AC010F94C245A70196010F94C2459B0147
:106D7000AC01D8016D917D918D919C910F948749C3
:106D8000F8016083718382839383C301B2010F94FE
:106D9000064C862F66E00F949D4C0DE110E00C0F21
:106DA0001D1FF4E09F9F000D111D11240C5F1F4F4C
:106DB000CC57DF4F688179818A819B81C458D0404C
:106DC0000F94364C9B01AC010F94C245A70196016C
:106DD0000F94C2459B01AC01D8016D917D918D91BD
:106DE0009C910F948749F801608371838283938318
:106DF000ED96FFADED97FF5FED96FFAFED97C054B9
:106E0000DF4F2881C05CD0402F170CF0DDCE81E031
:106E1000E9969FADE9979827E9969FAFE997AE96D7
:106E2000AFADAE97A8309CF020E030E040E450E4F5
:106E3000AF966FADAF97E3967FADE397E7968FADD3
:106E4000E797E8969FADE8970F94C2450CC0AF96C0
:106E50006FADAF97E3967FADE397E7968FADE7977A
:106E6000E8969FADE8979B01AC01C501B4010F9472
:106E700087494B015C0151CEAE96BFADAE97B430A1
:106E8000C4F419821A821B821C8219AE1AAE1BAE80
:106E90001CAE29961CAE1DAE1EAE1FAE2997A101D9
:106EA000BE01675C7F4FCE018B5B9F4F0E949B5260
:106EB0002EC0AF962FADAF97E3963FADE397E79621
:106EC0004FADE797E8965FADE89760E070E080E847
:106ED0009FE30F94634A6B017C018E010F5D1F4F8E
:106EE000A7019601F80160817181828193810F94DD
:106EF000634AD8016D937D938D939D938D01AD96DB
:106F0000EEADFFADAD97EA17FB0751F7BACFC1550C
:106F1000DF4FE881CF5AD040E11107CC6D8D7E8DD7
:106F20008F8D98A19B01AC010F94C2456B017C0130
:106F3000CF51DF4FB880C15ED04001E010E0EDE1FD
:106F4000F0E0EC0FFD1F24E0B29EE00DF11D1124D6
:106F500060817181828193819B01AC010F94C24554
:106F60009B01AC01C701B6010F9487496B017C01FD
:106F70000F5F1F4FCE51DF4F8881C25ED040B80EE9
:106F800096E09B15E0F6B801110F880B990B0F9452
:106F900063459B01AC01C701B6010F94634A0F948E
:106FA000404C20E030E04AE754E40F94C2450F948F
:106FB000064C0F94634520E030E04AE754E40F9418
:106FC000634A2CEA35EC47E257E30F948749AF96C2
:106FD0006FAFAF97E3967FAFE397E7968FAFE797F3
:106FE000E8969FAFE897AF962FADAF97E3963FAD8A
:106FF000E397E7964FADE797E8965FADE897CB56F6
:10700000DF4F6881C559D040CA56DF4F7881C659D5
:10701000D040C956DF4F8881C759D040C856DF4F8E
:107020009881C859D0400F94FB4B181674F0C65481
:10703000DF4FA881CA5BD040CC56DF4FB881C4591E
:10704000D040AB1714F40C943942C555DF4F28815A
:1070500039814A815B81CB5AD040AF966FADAF97F3
:10706000E3967FADE397E7968FADE797E8969FAD00
:10707000E8970F94FB4B181614F00C943942AF9616
:107080002FADAF97E3963FADE397E7964FADE79708
:10709000E8965FADE897CE55DF4F6881C25AD04081
:1070A000CD55DF4F7881C35AD040CC55DF4F888112
:1070B000C45AD040CB55DF4F9881C55AD0400F9469
:1070C000FB4B18160CF080C08091500D9091510D23
:1070D000A091520DB091530DC352DF4F8883998315
:1070E000AA83BB83CD5DD0408091540D9091550D06
:1070F000A091560DB091570DCB52DF4F88839983E5
:10710000AA83BB83C55DD0408091580D9091590DE5
:10711000A0915A0DB0915B0DC353DF4F88839983C3
:10712000AA83BB83CD5CD04080914C0D90914D0DD6
:10713000A0914E0DB0914F0DCF53DF4F88839983AF
:10714000AA83BB83C15CD04080915C0D90915D0DA2
:10715000A0915E0DB0915F0DCB53DF4F8883998373
:10716000AA83BB83C55CD0408091400D9091410DB6
:10717000A091420DB091430DC753DF4F888399838F
:10718000AA83BB83C95CD0408091440D9091450D8A
:10719000A091460DB091470DC752DF4F8883998368
:1071A000AA83BB83C95DD0408091480D9091490D61
:1071B000A0914A0DB0914B0DCF52DF4F8883998338
:1071C000AA83BB83C15DD040FE01E35AFF4F8CE030
:1071D000DF01282F1D922A95E9F73C97DF011D92C8
:1071E0008A95E9F78090380D9090390DA0903A0D6E
:1071F000B0903B0DAE96BFADAE97B83084F026E6AA
:1072000036E646E65FE3C501B4010F94C2456093DC
:10721000380D7093390D80933A0D90933B0D20916A
:107220004C0D30914D0D40914E0D50914F0D609190
:10723000380D7091390D80913A0D90913B0D0F945E
:10724000634A2BEA3AEA4AE25FE30F94634A9B01FE
:10725000AC0160E070E080E89FE30F94634AC4589B
:10726000DF4F688379838A839B83CC57D0409CE12E
:10727000E92EF1012E2D11922A95E9F73E0185E4C0
:10728000680E711C2CE0F22ED301EF2D1D92EA95B1
:10729000E9F7AD96AEADBFADAD97EF2D1D92EA9576
:1072A000E9F78E01075C1F4F2AE037ED43E25CE30C
:1072B000B301C1010F9416312D853E854F85588944
:1072C0006D817E818F8198850F9487492D893E89B4
:1072D0004F89588D0F94874929893A894B895C8950
:1072E0000F948749298D3A8D4B8D5C8D0F9487497A
:1072F00029853A854B855C850F948749905820E015
:1073000030E040EC50E40F94634A9B01AC016AE02A
:1073100077ED83E29CE30F94634A20E030E040E4A1
:1073200050E40F94634ACC54DF4F688379838A8397
:107330009B83C45BD040D1011D92EA94E9F7F3012D
:107340002F2D11922A95E9F7AD96AEADBFADAD9751
:107350001D92FA94E9F7EA961FAF0EAFEA97610122
:1073600035E0F32EC055DF4F188219821A821B8236
:10737000C05BD040C058DF4F6882C058D040E72C77
:1073800019AE1AAE1BAE1CAE21961CAE1DAE1EAEC3
:107390001FAE219725961CAE1DAE1EAE1FAE2597C3
:1073A000EA96EEADFFADEA978AE097EDA3E2BCE383
:1073B00081939193A193B193EA96FFAFEEAFEA97D1
:1073C0008E01075C1F4F20E030E0A901C058DF4F5D
:1073D0006881C058D0407E2DC1010F9416318F2D89
:1073E00066E00F949D4CF10124E0929FE00DF11DA9
:1073F000112420E030E040EC50E464817581868106
:1074000097810F94634AC055DF4F288139814A81A3
:107410005B81C05BD0400F9487492B013C0120E089
:1074200030E040EC50E4D60118966D917D918D913D
:107430009C911B970F94634A9B01AC01C301B2015D
:107440000F948649C055DF4F688379838A839B8375
:10745000C05BD040F394F394B8E0CB0ED11CEBE0CA
:10746000FE128ECF8092380D9092390DA0923A0D77
:10747000B0923B0DAE96FFADAE97FF2309F493C7D4
:1074800014F5FF3F09F01EC3CD8CDE8CEF8CF8A005
:1074900080E00E94DC521092820D19821A821B82B7
:1074A0001C8219AE1AAE1BAE1CAEB101CE01C9963C
:1074B0000E946FD883E080932E0581E08093D804EA
:1074C00080932D0509C0AE962FADAE972130B1F156
:1074D000223009F456C0F6C280912D05882321F090
:1074E00080E00E941561F8CF11E010932E051092F4
:1074F000D8040E94D7C4A701960160919D057091A0
:107500009E0580919F059091A0050F9486499B014F
:10751000AC011093820D6091600D7091610D8091AE
:10752000620D9091630D0F9487496093600D709385
:10753000610D8093620D9093630D35C720E030E0BC
:1075400040E850E46D8D7E8D8F8D98A10F94C245DB
:1075500020E030E040E85EE30F94C245A1966CAFB6
:107560007DAF8EAF9FAFA197A5966CAF7DAF8EAF6D
:107570009FAFA597A9966CAF7DAF8EAF9FAFA99730
:1075800012C78D8D9E8DAF8DB8A1EC968CAF9DAF3F
:10759000AEAFBFAFEC97C854DF4F9881C85BD04007
:1075A000992309F434C189A19AA1ABA1BCA1C05807
:1075B000DF4F88839983AA83BB83C058D04020E0E3
:1075C00030E040E850E4BC01CD010F94C24520E01A
:1075D00030E040E85EE30F94C245CC57DF4F68834C
:1075E00079838A839B83C458D040C9A4DAA4EBA4CE
:1075F000FCA4A7019601C701B6010F94874920E0BA
:1076000030E040E85EE30F94C245C857DF4F68831F
:1076100079838A839B83C858D04089A89AA8ABA84D
:10762000BCA8A5019401C501B4010F94874920E0CD
:1076300030E040E85EE30F94C245C457DF4F6883F3
:1076400079838A839B83CC58D04020E030E040E8A7
:1076500050E4EC966CAD7DAD8EAD9FADEC970F9484
:10766000C24520E030E040E85EE30F94C2452B01C4
:107670003C01C857DF4F288139814A815B81C85856
:10768000D040CC57DF4F688179818A819B81C45873
:10769000D0400F948649C457DF4F288139814A81F1
:1076A0005B81CC58D0400F948649C458DF4F288165
:1076B00039814A815B81CC57D0400F94C245A301E8
:1076C00092010F948749A1966CAF7DAF8EAF9FAFAB
:1076D000A19720E030E040E850E4C701B6010F94E4
:1076E000C24520E030E040E85EE30F94C245C05759
:1076F000DF4F688379838A839B83C059D040C05809
:10770000DF4F288139814A815B81C058D040CA014E
:10771000B9010F94874920E030E040E85EE30F9420
:10772000C2456B017C019B01AC01C057DF4F6881F2
:1077300079818A819B81C059D0400F948649C45772
:10774000DF4F288139814A815B81CC58D0400F942A
:107750008649C458DF4F288139814A815B81CC57E3
:10776000D0400F94C245A30192010F948749A5967A
:107770006CAF7DAF8EAF9FAFA59720E030E040E8C3
:1077800050E4C501B4010F94C24520E030E040E868
:107790005EE30F94C2454B015C01C701B6019058EE
:1077A000C857DF4F288139814A815B81C858D04052
:1077B0000F948649A50194010F948749C458DF4F5F
:1077C000288139814A815B81CC57D0400F94C245D2
:1077D000A30192010F948749A9966CAF7DAF8EAF3C
:1077E0009FAFA997C057DF4F288139814A815B81BC
:1077F000C059D040CC57DF4F688179818A819B8105
:10780000C458D0400F948749A501940132C18DA975
:107810009EA9AFA9B8ADC058DF4F88839983AA83CA
:10782000BB83C058D0409C01AD01BC01CD010F9479
:10783000874920E030E040E85EE30F94C245CC5732
:10784000DF4F688379838A839B83C458D0408DA49B
:107850009EA4AFA4B8A820E030E040E850E4C50101
:10786000B4010F94C24520E030E040E85EE30F949D
:10787000C245C857DF4F688379838A839B83C85882
:10788000D040CDA0DEA0EFA0F8A4A7019601C701CB
:10789000B6010F94874920E030E040E85EE30F94A2
:1078A000C245C457DF4F688379838A839B83CC5852
:1078B000D04020E030E040E850E4EC966CAD7DAD87
:1078C0008EAD9FADEC970F94C24520E030E040E8CC
:1078D0005EE30F94C2452B013C01C857DF4F28815E
:1078E00039814A815B81C858D040CC57DF4F6881CD
:1078F00079818A819B81C458D0400F948649C457AE
:10790000DF4F288139814A815B81CC58D0400F9468
:107910008749C458DF4F288139814A815B81CC5720
:10792000D0400F94C245A30192010F948749A196BC
:107930006CAF7DAF8EAF9FAFA197A5019401C5013C
:10794000B4010F94874920E030E040E85EE30F94F3
:10795000C245C057DF4F688379838A839B83C059B0
:10796000D04020E030E040E850E4C058DF4F68816C
:1079700079818A819B81C058D0400F94C24520E014
:1079800030E040E85EE30F94C2454B015C019B018F
:10799000AC01C057DF4F688179818A819B81C059D2
:1079A000D0400F948649C457DF4F288139814A81DE
:1079B0005B81CC58D0400F948749C458DF4F288151
:1079C00039814A815B81CC57D0400F94C245A301D5
:1079D00092010F948749A5966CAF7DAF8EAF9FAF94
:1079E000A59720E030E040E850E4C701B6010F94CD
:1079F000C24520E030E040E85EE30F94C2456B01F1
:107A00007C01C057DF4F288139814A815B81C05991
:107A1000D040CC57DF4F688179818A819B81C458DF
:107A2000D0400F948749A70196010F948649C45806
:107A3000DF4F288139814A815B81CC57D0400F9438
:107A4000C245A30192010F948749A9966CAF7DAFFF
:107A50008EAF9FAFA997A5019401C857DF4F6881EA
:107A600079818A819B81C858D0400F948749A701AA
:107A700096010F9487496B017C0120E030E040E4DF
:107A800051E4EC966CAD7DAD8EAD9FADEC970F944F
:107A9000C24520E030E040E85EE30F94C2459B0120
:107AA000AC01C701B6010F948649CC54DF4F288141
:107AB00039814A815B81C45BD0400F94C2454B0140
:107AC0005C0188C489A19AA1ABA1BCA1EC968CAF42
:107AD0009DAFAEAFBFAFEC979C01AD01BC01CD0136
:107AE0000F94874920E030E040E85EE30F94C24500
:107AF000C554DF4F688379838A839B83CB5BD040F7
:107B000089A59AA5ABA5BCA5C058DF4F88839983EA
:107B1000AA83BB83C058D04020E030E040E85EE359
:107B2000BC01CD010F94C245CD51DF4F68837983ED
:107B30008A839B83C35ED04089A99AA9ABA9BCA9BB
:107B4000CC57DF4F88839983AA83BB83C458D04026
:107B500020E030E040E85EE3BC01CD010F94C24577
:107B60004B015C018DA59EA5AFA5B8A9C857DF4FF5
:107B700088839983AA83BB83C858D0409C01AD01F8
:107B8000BC01CD010F94874920E030E040E85EE37E
:107B90000F94C245C951DF4F688379838A839B83E1
:107BA000C75ED0408DA99EA9AFA9B8ADC457DF4F1D
:107BB00088839983AA83BB83CC58D04020E030E0EF
:107BC00040E85EE3BC01CD010F94C245C551DF4FD3
:107BD000688379838A839B83CB5ED0408DA19EA1ED
:107BE000AFA1B8A5C057DF4F88839983AA83BB8311
:107BF000C059D04020E030E040E85EE3BC01CD0158
:107C00000F94C2456B017C018D8D9E8DAF8DB8A107
:107C1000CA55DF4F88839983AA83BB83C65AD04055
:107C200020E030E040E850E4BC01CD010F94C245B3
:107C300020E030E040E85EE30F94C2452B013C01B8
:107C4000CD51DF4F288139814A815B81C35ED040AD
:107C5000C554DF4F688179818A819B81CB5BD0409D
:107C60000F948649A50194010F948649C951DF4FAD
:107C7000288139814A815B81C75ED0400F94864953
:107C8000C551DF4F288139814A815B81CB5ED0406D
:107C90000F948749A70196010F948749C458DF4F75
:107CA000288139814A815B81CC57D0400F94C245ED
:107CB000A30192010F948749A1966CAF7DAF8EAF5F
:107CC0009FAFA197C058DF4F288139814A815B81DE
:107CD000C058D040CA01B9010F94874920E030E074
:107CE00040E85EE30F94C245C151DF4F688379835A
:107CF0008A839B83CF5ED04020E030E040E85EE3A3
:107D0000EC966CAD7DAD8EAD9FADEC970F94C245FA
:107D1000CD50DF4F688379838A839B83C35FD040D4
:107D200020E030E040E85EE3C857DF4F68817981AA
:107D30008A819B81C858D0400F94C245C950DF4FFB
:107D4000688379838A839B83C75FD040C457DF4FA2
:107D5000288139814A815B81CC58D040CA01B90160
:107D60000F94874920E030E040E85EE30F94C2457D
:107D7000C550DF4F688379838A839B83CB5FD04074
:107D8000CD50DF4F288139814A815B81C35FD0406C
:107D9000C151DF4F688179818A819B81CF5ED0405C
:107DA0000F948649A50194010F948649C950DF4F6D
:107DB000288139814A815B81C75FD0400F94874910
:107DC000C550DF4F288139814A815B81CB5FD0402C
:107DD0000F948649A70196010F948749C458DF4F35
:107DE000288139814A815B81CC57D0400F94C245AC
:107DF000A30192010F948749A5966CAF7DAF8EAF1A
:107E00009FAFA597CC57DF4F288139814A815B818D
:107E1000C458D040CA01B9010F94874920E030E02E
:107E200040E85EE30F94C2454B015C01C057DF4F51
:107E3000288139814A815B81C059D040CA01B9018A
:107E40000F94874920E030E040E85EE30F94C2459C
:107E50006B017C01CD50DF4F688179818A819B81E4
:107E6000C35FD0409058CD51DF4F288139814A817E
:107E70005B81C35ED0400F948649A50194010F94A5
:107E80008749C950DF4F288139814A815B81C75FAB
:107E9000D0400F948749C551DF4F288139814A81ED
:107EA0005B81CB5ED0400F948749A70196010F9468
:107EB0008649C458DF4F288139814A815B81CC577C
:107EC000D0400F94C245A30192010F948749A9960F
:107ED0006CAF7DAF8EAF9FAFA997C151DF4F2881A7
:107EE00039814A815B81CF5ED040C554DF4F6881C4
:107EF00079818A819B81CB5BD0400F948749A50112
:107F000094010F948749C951DF4F288139814A81F3
:107F10005B81C75ED0400F948749C550DF4F2881F1
:107F200039814A815B81CB5FD0400F948749A7019B
:107F300096010F9487496B017C0120E030E040E41A
:107F400051E4CA55DF4F688179818A819B81C65A85
:107F5000D0400F94C24520E030E040E85EE30F944B
:107F6000C2459B01AC01C701B6010F948649CC54B0
:107F7000DF4F288139814A815B81C45BD0400F94F7
:107F8000C2454B015C01C854DF4F9881C85BD040AB
:107F9000992309F41FC2C055DF4F288139814A81D6
:107FA0005B81C05BD0406AE077ED83E29CE30F9495
:107FB000634A20E030E040E450E40F94634AC45840
:107FC000DF4F688379838A839B83CC57D04020E03E
:107FD00030E040E850E4C058DF4F688179818A8101
:107FE0009B81C058D0400F94C24520E030E040E86B
:107FF0005EE30F94C245C055DF4F688379838A835F
:108000009B83C05BD04020E030E040E850E4CC5798
:10801000DF4F688179818A819B81C458D0400F9459
:10802000C24520E030E040E85EE30F94C2452B01FA
:108030003C0120E030E040E850E4C457DF4F688165
:1080400079818A819B81CC58D0400F94C24520E031
:1080500030E040E85EE30F94C245CC54DF4F6883C4
:1080600079838A839B83C45BD04020E030E040E882
:1080700050E4C057DF4F688179818A819B81C05964
:10808000D0400F94C24520E030E040E85EE30F941A
:10809000C245C554DF4F688379838A839B83CB5B5A
:1080A000D04020E030E0A901CA55DF4F68817981D6
:1080B0008A819B81C65AD0400F94C24520E030E0AF
:1080C00040E85EE30F94C245CA55DF4F6883798369
:1080D0008A839B83C65AD04020E030E0A901EC9609
:1080E0006CAD7DAD8EAD9FADEC970F94C24520E099
:1080F00030E040E85EE30F94C245C055DF4F288171
:1081000039814A815B81C05BD0400F948649A301CD
:1081100092010F9487496B017C0120E030E0A901B6
:10812000C857DF4F688179818A819B81C858D040C8
:108130000F94C24520E030E040E85EE30F94C24572
:108140009B01AC01C701B6010F948749CC54DF4FA6
:10815000288139814A815B81C45BD0400F94864974
:10816000C554DF4F288139814A815B81CB5BD04088
:108170000F948749CA55DF4F288139814A815B8135
:10818000C65AD0400F948749C458DF4F288139819F
:108190004A815B81CC57D0400F94C24565966CAF45
:1081A0007DAF8EAF9FAF659720E030E040E850E4B0
:1081B000EC966CAD7DAD8EAD9FADEC970F94C24546
:1081C00020E030E040E85EE30F94C245EC966CAFEF
:1081D0007DAF8EAF9FAFEC9720E030E040E850E4F9
:1081E000C857DF4F688179818A819B81C858D04008
:1081F0000F94C24520E030E040E85EE30F94C245B2
:108200006B017C0120E030E0A901C058DF4F68819C
:1082100079818A819B81C058D0400F94C24520E06B
:1082200030E040E85EE30F94C245EC962CAD3DADE6
:108230004EAD5FADEC970F948749A30192010F9467
:108240008649A70196010F9487492B013C0120E044
:1082500030E0A901C457DF4F688179818A819B8111
:10826000CC58D0400F94C24520E030E040E85EE3B7
:108270000F94C2459B01AC01C301B2010F94874921
:10828000C554DF4F288139814A815B81CB5BD04067
:108290000F948649CA55DF4F288139814A815B8115
:1082A000C65AD0400F948749C458DF4F288139817E
:1082B0004A815B81CC57D0400F94C24569966CAF20
:1082C0007DAF8EAF9FAF699720E030E0A901CC571A
:1082D000DF4F688179818A819B81C458D0400F9497
:1082E000C24520E030E040E85EE30F94C2452B0138
:1082F0003C01EC962CAD3DAD4EAD5FADEC97C0555D
:10830000DF4F688179818A819B81C05BD0400F9467
:1083100086499B01AC01C301B2010F948749A701B3
:1083200096010F948649CC54DF4F288139814A81C8
:108330005B81C45BD0400F9487496B017C0120E0D6
:1083400030E0A901C057DF4F688179818A819B8124
:10835000C059D0400F94C24520E030E040E85EE3D1
:108360000F94C2459B01AC01C701B6010F94874928
:10837000CA55DF4F288139814A815B81C65AD04076
:108380000F948749C458DF4F288139814A815B8126
:10839000CC57D0400F94C2456D966CAF7DAF8EAF79
:1083A0009FAF6D9717C0812C912C5401CB56DF4F96
:1083B0001882C559D040CA56DF4F1882C659D040DE
:1083C000C956DF4F1882C759D040C856DF4F1882B0
:1083D000C859D0407E01ADE5EA0EF11C00E51DE074
:1083E000F70121913191419151917F01D8016D9116
:1083F0007D918D919C910F948749F80161937193C0
:10840000819391938F01FDE00C351F0749F7A5017A
:10841000940160914C0D70914D0D80914E0D909195
:108420004F0D0F94874960934C0D70934D0D8093C1
:108430004E0D90934F0D7E0121E5E20EF11C00E4FC
:108440001DE0D7012D913D914D915D917D01F80188
:1084500060817181828193810F948749D8016D93E6
:108460007D938D939D938D01BDE00C341B0749F7DF
:10847000A5C0AF962FADAF97E3963FADE397E796D4
:108480004FADE797E8965FADE897CB56DF4F688131
:10849000C559D040CA56DF4F7881C659D040C95619
:1084A000DF4F8881C759D040C856DF4F9881C859DF
:1084B000D0400F945D4518160CF480C0C352DF4FB6
:1084C00088819981AA81BB81CD5DD0408093500D78
:1084D0009093510DA093520DB093530DCB52DF4F9B
:1084E00088819981AA81BB81C55DD0408093540D5C
:1084F0009093550DA093560DB093570DC353DF4F76
:1085000088819981AA81BB81CD5CD0408093580D30
:108510009093590DA0935A0DB0935B0DCF53DF4F3D
:1085200088819981AA81BB81C15CD04080934C0D28
:1085300090934D0DA0934E0DB0934F0DCB53DF4F45
:1085400088819981AA81BB81C55CD04080935C0DF4
:1085500090935D0DA0935E0DB0935F0DC753DF4FF9
:1085600088819981AA81BB81C95CD0408093400DEC
:108570009093410DA093420DB093430DC752DF4F2E
:1085800088819981AA81BB81C95DD0408093440DC7
:108590009093450DA093460DB093470DCF52DF4FFA
:1085A00088819981AA81BB81C15DD0408093480DAB
:1085B0009093490DA0934A0DB0934B0DC756DF4FD2
:1085C0009881C959D040911148C00E944A6EAF9617
:1085D0002FADAF97E3963FADE397E7964FADE797A3
:1085E000E8965FADE897CE55DF4F6881C25AD0401C
:1085F000CD55DF4F7881C35AD040CC55DF4F8881AD
:10860000C45AD040CB55DF4F9881C55AD0400F9403
:10861000FB4B18160CF0C1C0AF96EFADAF97CE551F
:10862000DF4FE883C25AD040E396FFADE397CD55C4
:10863000DF4FF883C35AD040E7962FADE797CC556C
:10864000DF4F2883C45AD040E8968FADE897CB55CA
:10865000DF4F8883C55AD040A0C0C655DF4FA881E0
:10866000CA5AD040A11123C0C090580DD090590DC6
:10867000E0905A0DF0905B0DA090540DB090550D08
:108680000091560D1091570D6090500D7090510D46
:108690008090520D9090530D9301A401B501C80133
:1086A0000F945D4587FF45C05301840142C020E01F
:1086B00030E0A9016091400D7091410D8091420D13
:1086C0009091430D0F9487492091440D3091450DB1
:1086D0004091460D5091470D0F9487492091480DC8
:1086E0003091490D40914A0D50914B0D0F9487499F
:1086F00020E030E040E450E40F94634A4B015C0119
:1087000000E41DE08CE4E82E8DE0F82EA501940134
:10871000F80160817181828193810F948649D8012B
:108720006D937D938D939D938D01EA16FB0671F7F2
:108730009BCF9501A801B601C7010F945D4587FF46
:1087400002C0650178019601A70160915C0D7091EE
:108750005D0D80915E0D90915F0D0F948649609341
:108760005C0D70935D0D80935E0D90935F0D00E541
:108770001DE09601A701F8016081718182819381DA
:108780000F948649D8016D937D938D939D938D01B0
:10879000BDE00C351B0769F718CFC756DF4F98812E
:1087A000C959D040933009F060C0EDE6F7E08491FC
:1087B0008F010F5F1F4F882321F00E94EA5CF801B0
:1087C000F6CFBE01635E7F4F8BE697E00F945F3478
:1087D000C356DF4FA881CD59D040AA2331F1BE0145
:1087E0006F5D7F4F88E697E00F945F34BE01675D51
:1087F0007F4F85E697E00F945F34BE016F5C7F4F3B
:1088000082E697E00F945F34C656DF4FB881CA59AD
:10881000D040BB2331F18AE00E94EA5C8EE20E94E4
:10882000EA5C8DE00E94C3C107C0C656DF4FE881F5
:10883000CA59D040EE23A9F0BE01635D7F4F8FE59A
:1088400097E00F945F34BE016B5C7F4F8CE597E03F
:108850000F945F34BE016B5D7F4F89E597E00F9405
:108860005F348AE00E94EA5C0AC0C756DF4FF88195
:10887000C959D040F11103C0EAE2F8E0ADC1AF96AA
:108880002FADAF97E3963FADE397E7964FADE797F0
:10889000E8965FADE897CB56DF4F6881C559D04069
:1088A000CA56DF4F7881C659D040C956DF4F8881FC
:1088B000C759D040C856DF4F9881C859D0400F944F
:1088C0005D45181664F0C654DF4F2881CA5BD0405E
:1088D000CC56DF4F8881C459D0402817CCF0C555FD
:1088E000DF4F288139814A815B81CB5AD040AF96D6
:1088F0006FADAF97E3967FADE397E7968FADE797C0
:10890000E8969FADE8970F945D4518160CF4FDC0EE
:10891000EBE1F8E084918F010F5F1F4F882321F076
:108920000E94EA5CF801F6CF80E20E94C3C1AF96D4
:108930002FADAF97E3963FADE397E7964FADE7973F
:10894000E8965FADE897CB56DF4F6881C559D040B8
:10895000CA56DF4F7881C659D040C956DF4F88814B
:10896000C759D040C856DF4F9881C859D0400F949E
:108970005D4518167CF0C155DF4F9881CF5AD04025
:10898000911108C0AE96AFADAE97AA2319F0E4E0FE
:10899000F8E003C0E2E1F8E00AC084918F010F5FC4
:1089A0001F4F882329F10E94EA5CF801F6CF8491D9
:1089B0008F010F5F1F4F882321F00E94EA5CF801AE
:1089C000F6CF43E0CE55DF4F6881C25AD040CD5537
:1089D000DF4F7881C35AD040CC55DF4F8881C45ACD
:1089E000D040CB55DF4F9881C55AD0400E940A60D5
:1089F0008AE00E94EA5C64EF77E0C1010F94A6442C
:108A000020E030E040E85FE3CE55DF4F6881C25A96
:108A1000D040CD55DF4F7881C35AD040CC55DF4F81
:108A20008881C45AD040CB55DF4F9881C55AD04079
:108A30000F945D4587FF21C020E030E04AE754E411
:108A4000CE55DF4F6881C25AD040CD55DF4F788177
:108A5000C35AD040CC55DF4F8881C45AD040CB5543
:108A6000DF4F9881C55AD0400F94C2450F94064CF1
:108A70007F936F938DEE97E01AC0CE55DF4F6881DC
:108A8000C25AD040CD55DF4F7881C35AD040CC5523
:108A9000DF4F8881C45AD040CB55DF4F9881C55AEB
:108AA000D0400F94064C7F936F9386EE97E09F9390
:108AB0008F93CE0140969F938F930F94F7440F901E
:108AC0000F900F900F900F900F9060E0C1010E94E7
:108AD000098AC655DF4F6881CA5AD040C754DF4F54
:108AE0008881C95BD0400F949C34E8EBF7E0849117
:108AF0008F010F5F1F4F882321F00E94EA5CF8016D
:108B0000F6CF8AE00E94EA5CEEC0CC56DF4FB88117
:108B1000C459D040BF31C4F48B2F0B2E000C990BDD
:108B20009F93BF9387EA97E09F938F933F922F92F3
:108B30000F94F7440F900F900F900F900F900F909D
:108B40008E010F5F1F4F06C068E977E0C1010F94E7
:108B5000A644F6CFF80181918F01882319F00E9475
:108B6000EA5CF8CF80E20E94C3C1EFE8F7E08491AD
:108B70008F010F5F1F4F882321F00E94EA5CF801EC
:108B8000F6CF43E0AF966FADAF97E3967FADE39737
:108B9000E7968FADE797E8969FADE8970E940A6049
:108BA0008AE00E94EA5C60E0C1010E94098AC7561F
:108BB000DF4FF881C959D040F23008F494C0C6554F
:108BC000DF4F6881CA5AD040C754DF4F8881C95BE4
:108BD000D0400F949C3487C084918F010F5F1F4F4A
:108BE000882321F00E94EA5CF801F6CF83E20E941C
:108BF000C3C1E6E8F7E084918F010F5F1F4F882320
:108C000021F00E94EA5CF801F6CF43E0AF966FAD29
:108C1000AF97E3967FADE397E7968FADE797E8963A
:108C20009FADE8970E940A608AE00E94EA5C6AE2CF
:108C300078E0C1010F94A64461E877E0CE010C967C
:108C40000F94A64420E030E040E85FE3AF966FADBC
:108C5000AF97E3967FADE397E7968FADE797E896FA
:108C60009FADE8970F945D4587FF19C020E030E085
:108C70004AE754E4AF966FADAF97E3967FADE397C5
:108C8000E7968FADE797E8969FADE8970F94C245BA
:108C90000F94064C7F936F938AE797E012C0AF96CC
:108CA0006FADAF97E3967FADE397E7968FADE7970C
:108CB000E8969FADE8970F94064C7F936F9383E7F8
:108CC00097E09F938F93CE0140969F938F930F943D
:108CD000F7440F900F900F900F900F900F9060E05F
:108CE000C1010E94098A81E08093800D0E9456A4F0
:108CF00080917F0D8093800DAF962FADAF97E39657
:108D00003FADE397E7964FADE797E8965FADE897FD
:108D1000CB56DF4F6881C559D040CA56DF4F7881A6
:108D2000C659D040C956DF4F8881C759D040C85670
:108D3000DF4F9881C859D0400F94FB4B18163CF474
:108D4000CC56DF4F2881C459D0402F316CF0C65427
:108D5000DF4F8881CA5BD040CC56DF4F9881C45921
:108D6000D04089170CF44EC0C256DF4FE880CE5970
:108D7000D040C156DF4FF880CF59D040C056DF4FAA
:108D80000881C05AD040CF55DF4F1881C15AD0401A
:108D9000C555DF4F288139814A815B81CB5AD0404C
:108DA000AF966FADAF97E3967FADE397E7968FAD44
:108DB000E797E8969FADE8970F94FB4B181614F5CC
:108DC000AF969FADAF97C256DF4F9883CE59D04034
:108DD000E396AFADE397C156DF4FA883CF59D0409C
:108DE000E796BFADE797C056DF4FB883C05AD04073
:108DF000E896EFADE897CF55DF4FE883C15AD040F2
:108E00000C94F43280E00E94DC520E94635249C00C
:108E1000E6E3F8E084918F010F5F1F4F882391F301
:108E20000E94EA5CF801F6CFC555DF4F188219821F
:108E30001A821B82CB5AD0400C94B62FAE969FADAF
:108E4000AE979330A4F4AE968FADAE97813011F00B
:108E50000C946830C656DF4F1882CA59D040C356AA
:108E6000DF4F1882CD59D04010E00C94BE30A1E005
:108E7000C356DF4FA883CD59D04010E0B1E0C656AD
:108E8000DF4FB883CA59D0400C947330C456DF4FBB
:108E90001881CC59D040C356DF4F1882CD59D040ED
:108EA000EDCFCC5FDE4F0FB6F894DEBF0FBECDBF67
:108EB000DF91CF911F910F91FF90EF90DF90CF90B6
:108EC000BF90AF909F908F907F906F905F904F90EA
:108ED0003F902F9008958F929F92AF92BF92CF9222
:108EE000DF92EF92FF920F931F93CF93DF93CDB753
:108EF000DEB764970FB6F894DEBF0FBECDBFD62E97
:108F0000F72E8C018090020590900305A090040537
:108F1000B0900505A50194016091950570919605A5
:108F200080919705909198050F945D4581113DC002
:108F300020910605309107054091080550910905DB
:108F40006091990570919A0580919B0590919C057F
:108F50000F945D45811129C020910A0530910B05C0
:108F600040910C0550910D0560919D0570919E05F5
:108F700080919F059091A0050F945D45811115C0CA
:108F800020910E0530910F0540911005509111056B
:108F90006091A1057091A2058091A3059091A4050F
:108FA0000F945D45882309F46DC0E0902F0520E003
:108FB00030E0A9016D2D7F2DC8010F945D45811111
:108FC00008C0D0900102F0900202009103021091BB
:108FD00004026091520270915302072E000C880B1C
:108FE000990B0F9463452D2D3F2DA8010F94C24579
:108FF0002AE037ED43E25CE30F94C245698B7A8B3C
:109000008B8B9C8B1D861E861F86188A89829A826E
:10901000AB82BC828091060590910705A09108055E
:10902000B09109058D839E83AF83B88780910A052F
:1090300090910B05A0910C05B0910D0589879A8739
:10904000AB87BC87AE01475F5F4FBE016B5F7F4F51
:10905000CE0101960F94F729CE0101960E94E36795
:10906000CE010D966C018E010F5E1F4F2EE035E094
:109070004DEA55E069EA75E085EA95E00E94BAABF1
:109080000E94E05C64960FB6F894DEBF0FBECDBFC1
:10909000DF91CF911F910F91FF90EF90DF90CF90D4
:1090A000BF90AF909F908F9008952F923F924F92D4
:1090B0005F926F927F928F929F92AF92BF92CF9268
:1090C000DF92EF92FF920F931F93CF93DF93CDB771
:1090D000DEB72C970FB6F894DEBF0FBECDBF2B01C5
:1090E0003C0129833A834B835C8347015801F60195
:1090F000108181818C8792819B87038120E030E001
:10910000A901612F782F892F902F0F945D45811130
:109110000BC0E2EAFCE085919591A591B491382EBF
:10912000292EAD83BE8305C0312E2C84AB85AD8343
:109130000E83A3019201C301B2010F94C2456B01DA
:109140007C0129813A814B815C81CA01B9010F946C
:10915000C2459B01AC01C701B6010F94874920E0CD
:1091600030E442E556E40F945D4518160CF4ECC06B
:1091700020E030E0A901612F7C858B85902F0F9432
:109180005D4581110AC010910A02B0910B02BC87A3
:1091900080910C028B8700910D02809101029091C9
:1091A0000202A0910302B09104028F839887A987DD
:1091B000BA87812F9C85AB85B02F80930102909355
:1091C0000202A0930302B09304020E94D65CC090F6
:1091D0003502D0903602E0903702F0903802A701B5
:1091E000960160919D0570919E0580919F059091DB
:1091F000A0050F94FB4B18160CF04CC0A501940170
:10920000C701B6010F945D4587FF38C04092020543
:1092100050920305609204057092050589819A8138
:10922000AB81BC818093060590930705A093080548
:10923000B093090580920A0590920B05A0920C0547
:10924000B0920D0560E070E0CB012C960FB6F8945B
:10925000DEBF0FBECDBFDF91CF911F910F91FF9069
:10926000EF90DF90CF90BF90AF909F908F907F90C6
:109270006F905F904F903F902F902DCEC0920A0537
:10928000D0920B05E0920C05F0920D0560E070E0C5
:10929000CB0121DE20919D0530919E0540919F05D7
:1092A0005091A005C501B4010F94FB4B18166CF446
:1092B00080920A0590920B05A0920C05B0920D05C4
:1092C000632D722D8D819E8106DE409202055092A3
:1092D0000305609204057092050589819A81AB812E
:1092E000BC818093060590930705A0930805B09371
:1092F00009050E940A6920919D0530919E054091C3
:109300009F055091A005C501B4010F945D4587FFED
:109310000DC080920A0590920B05A0920C05B092A8
:109320000D05632D722D8D819E81D5DD0E94C6B9FC
:109330008F819885A985BA85809301029093020256
:10934000A0930302B09304022C960FB6F894DEBFEC
:109350000FBECDBFDF91CF911F910F91FF90EF9086
:10936000DF90CF90BF90AF909F908F907F906F9045
:109370005F904F903F902F9008959F92AF92BF9231
:10938000CF92DF92EF92FF920F931F93CF93DF93D1
:1093900087E5A82E82E0B82E02E015E0C5E9D5E009
:1093A0009DE0C92E9FE0D92E20E5E22E23E0F22E8B
:1093B000912CF50181915F010E947B5C882309F16A
:1093C0000E94485CF7012081211104C020915403C0
:1093D000222339F0288139814A815B810F948749A2
:1093E0000AC0F3E09F1639F0F601208131814281F5
:1093F00053810F948649F80160837183828393833C
:1094000009C088819981AA81BB81F80180839183F9
:10941000A283B38393940C5F1F4F2496F4E0CF0E86
:10942000D11C2FEFE21AF20A84E09812C2CF86E430
:109430000E94C45C8823C9F00E94485C20E030E0B0
:10944000A9010F94FB4B181684F40E94485C20E09D
:1094500030E040E752E40F94634A60930102709356
:1094600002028093030290930402DF91CF911F9137
:109470000F91FF90EF90DF90CF90BF90AF909F90B3
:1094800008952F923F924F925F926F927F929F9298
:10949000AF92BF92CF92DF92EF92FF920F931F9302
:1094A000CF93DF93CDB7DEB764970FB6F894DEBFE6
:1094B0000FBECDBF1A012B01922EF32EC82ED12C38
:1094C000F601E951F34FE491AA24A3941E160CF47B
:1094D000A12CBB24B39420E030E0A901C201B1016A
:1094E0000F94FB4B18160CF0B12CCC0CDD1CCC0CE3
:1094F000DD1CC6018B569A4F3C01FC011082118283
:10950000128213820E94CB5BF3012082318242825D
:109510005382E0902F0520E030E0A901B801892DA9
:109520009F2D0F945D4581110AC0F601E656F34F59
:1095300085919591A591B4918C019A2EFB2EC8012D
:10954000A92DBF2D898B9A8BAB8BBC8B80919D05F0
:1095500090919E05A0919F05B091A005409199051D
:1095600050919A0560919B0570919C05009195051D
:1095700010919605209197053091980509831A83DB
:109580002B833C834D835E836F83788789879A879B
:10959000AB87BC871D861E861F86188ACE010D9656
:1095A0006C018E010F5E1F4F21EA35E0AE01475F6F
:1095B0005F4FBE016B5F7F4F0C970E94BAAB0E945A
:1095C000C6B9AB100F94E02D64960FB6F894DEBFC9
:1095D0000FBECDBFDF91CF911F910F91FF90EF9004
:1095E000DF90CF90BF90AF909F907F906F905F90F3
:1095F0004F903F902F900895CF939091370D9817EB
:10960000B9F0C82F0E94C6B9C093370DC11109C067
:109610000E94A6648EEB94E00F94E8280E94FB75EC
:1096200004C085E995E00F94E828CF910C94C95BBC
:10963000CF91089580E0E0DFE2EEFFE080E090E08F
:10964000A0E8BFE380839183A283B3831482158251
:109650001682178210861186128613861486158646
:1096600016861786808B918BA28BB38B148A158AF2
:10967000168A178A108E118E128E138E148E158EE6
:10968000168E178E80A391A3A2A3B3A30895EF9281
:10969000FF921F93CF93DF93882329F0D0911D0F62
:1096A000D095D17001C0D0E0662339F010911D0F24
:1096B0001695117081E0182701C010E0442341F095
:1096C000C0911D0FC2FB882780F9C1E0C82701C0E7
:1096D000C0E0D11105C0111103C0CC2309F482C030
:1096E000E9E4FFE284917F019FEFE91AF90A811111
:1096F00003C0E5EBF9E004C00E94EA5CF701F2CF99
:1097000084917F019FEFE91AF90A882321F00E94D2
:10971000EA5CF701F5CFDD2369F0E3EBF9E0849132
:109720007F019FEFE91AF90A882321F00E94EA5C81
:10973000F701F5CF112369F0E1EBF9E084917F01A6
:109740009FEFE91AF90A882321F00E94EA5CF701E9
:10975000F5CFCC2319F0EFEAF9E003C0E7EAF9E02E
:109760000BC084917F019FEFE91AF90A8823B1F3B6
:109770000E94EA5CF701F5CF84917F019FEFE91A1F
:10978000F90A882321F00E94EA5CF701F5CFCC2387
:1097900019F041E253E002C04CE153E0112319F00B
:1097A00023E233E002C02CE133E0DD2319F085E24F
:1097B00093E002C08CE193E05F934F933F932F932C
:1097C0009F938F9385E999E09F938F931F920E94B7
:1097D000EC928DB79EB709960FB6F8949EBF0FBE58
:1097E0008DBFC1E08C2FDF91CF911F91FF90EF9043
:1097F00008952F923F924F925F926F927F928F9235
:109800009F92AF92BF92CF92DF92EF92FF920F930F
:109810001F93CF93DF93CDB7DEB7C456D1090FB6F0
:10982000F894DEBF0FBECDBF382E41E061E081E08D
:109830002EDF81112EC680914802882309F429C6A3
:109840009CDD82E50E94C45C882309F42CC10E943F
:10985000485C4B015C0120E030E0A9010F945D45BC
:10986000882309F4FEC52091950530919605409115
:10987000970550919805298F3A8F4B8F5C8F809177
:10988000990590919A05A0919B05B0919C058D8FAB
:109890009E8FAF8FB8A320910205309103054091B0
:1098A0000405509105052DA73EA74FA758AB809101
:1098B000060590910705A0910805B09109058DA3B3
:1098C0009EA3AFA3B8A7698D7A8D8B8D9C8D0F94C5
:1098D0005D4581110DC02DA13EA14FA158A56D8DF3
:1098E0007E8D8F8D98A10F945D45882309F4B9C5AD
:1098F000E32CF12C01E010E020E030E0A901C501EB
:10990000B4010F945D4587FD02C000E010E0E01651
:10991000F10649F420E030E040E85FE329AB3AABE0
:109920004BAB5CAB08C080E090E0A0E8BFEB89AB3C
:109930009AABABABBCAB298D3A8D4B8D5C8D6DA5D5
:109940007EA58FA598A90F94864969A77AA78BA7AA
:109950009CA72D8D3E8D4F8D58A16DA17EA18FA10D
:1099600098A50F9486496B017C0129A53AA54BA5C2
:109970005CA5CA01B9010F94C2452B013C01A701A6
:109980009601C701B6010F94C2459B01AC01C3010A
:10999000B2010F9487490F94404C69A37AA38BA31B
:1099A0009CA320E030E040E05FE30F94C2452B0130
:1099B0003C01A5019401C501B4010F94C2454B01BE
:1099C0005C01A3019201C301B2010F94C2459B0146
:1099D000AC01C501B4010F9486490F94404C9B0122
:1099E000AC0169A97AA98BA99CA90F94C2454B0126
:1099F0005C01C701B601905829A13AA14BA15CA115
:109A00000F94634AA50194010F94C2456B017C0138
:109A10002DA53EA54FA558A9698D7A8D8B8D9C8D5E
:109A20000F94874920E030E040E05FE30F94C245A7
:109A30009B01AC01C701B6010F948749298D3A8D6E
:109A40004B8D5C8D0F9486496B017C012DA13EA14D
:109A50004FA158A56D8D7E8D8F8D98A10F9487494C
:109A600020E030E040E05FE30F94C2452B013C0171
:109A700029A13AA14BA15CA169A57AA58BA59CA5BA
:109A80000F94634AA50194010F94C2459B01AC0158
:109A9000C301B2010F9487492D8D3E8D4F8D58A182
:109AA0000F94864914C089E40E94C45C882329F07D
:109AB0000E94485C6B017C0103C0C12CD12C760153
:109AC0008AE40E94C45C8823D9F00E94485C6DA798
:109AD0007EA78FA798AB20E030E0A901C701B601AF
:109AE0000F945D4581111AC020E030E0A9016DA5F9
:109AF0007EA58FA598A90F945D4581110FC0B1C4B3
:109B000020E030E0A901C701B6010F945D4588232C
:109B100009F4A7C41DA61EA61FA618AAA701960190
:109B20005058298F3A8F4B8F5C8F8DA59EA5AFA57E
:109B3000B8A9B0588D8F9E8FAF8FB8A3CA01B90155
:109B40000F94C2454B015C012D8D3E8D4F8D58A168
:109B5000CA01B9010F94C2459B01AC01C501B40112
:109B60000F9487490F94404C21966CAF7DAF8EAF18
:109B70009FAF2197209195053091960540919705CB
:109B8000509198052DA33EA34FA358A7C701B60136
:109B90000F9487492D966CAF7DAF8EAF9FAF2D97F9
:109BA0008091990590919A05A0919B05B0919C0593
:109BB00089A79AA7ABA7BCA79C01AD016DA57EA5FF
:109BC0008FA598A90F94874961966CAF7DAF8EAF32
:109BD0009FAF6197209102053091030540910405E4
:109BE0005091050529AB3AAB4BAB5CAB2D962CAD38
:109BF0003DAD4EAD5FAD2D9769A97AA98BA99CA902
:109C00000F9486496B017C018091060590910705B0
:109C1000A0910805B09109058DAB9EABAFABB8AF75
:109C200061962CAD3DAD4EAD5FAD6197BC01CD01F0
:109C30000F9486494B015C0120919D0530919E0552
:109C400040919F055091A00529AF3AAF4BAF5CAF53
:109C500060910A0570910B0580910C0590910D059E
:109C60000F94864969A37AA38BA39CA3A7019601AD
:109C7000698D7A8D8B8D9C8D0F94C2452B013C0193
:109C8000A50194016D8D7E8D8F8D98A10F94C24595
:109C90009B01AC01C301B2010F9487492B013C0128
:109CA000A5019401698D7A8D8B8D9C8D0F94C24591
:109CB0004B015C01A70196016D8D7E8D8F8D98A162
:109CC0000F94C2459B01AC01C501B4010F948649B4
:109CD000A30192010F94FA496B017C0120E030E06E
:109CE000A9010F945D4587FF0AC02BED3FE049ECC9
:109CF00050E4C701B6010F9487496B017C01332002
:109D000051F02BED3FE049EC50E4C701B6010F9450
:109D100086496B017C0120E030E0A901C701B60152
:109D20000F945D45811120C029A93AA94BA95CA9CE
:109D30006DA17EA18FA198A50F945D45811114C0DE
:109D40002DA93EA94FA958AD69A57AA58BA59CA5BB
:109D50000F945D45811108C08BEDC82E8FE0D82E81
:109D600089ECE82E80E4F82EA701960121966CADCF
:109D70007DAD8EAD9FAD21970F94C2454B015C0127
:109D800020E030E0A90169A17AA18BA19CA10F94E8
:109D90005D458823D9F0A5019401C501B4010F9454
:109DA000C2454B015C0129A13AA14BA15CA1CA01AA
:109DB000B9010F94C2459B01AC01C501B4010F94D8
:109DC00087490F94404C4B015C010DC020E030E00E
:109DD000A901C501B4010F94FB4B87FF04C0B7FA7A
:109DE000B094B7F8B0942FE632E143E85AE3C501E6
:109DF000B4010F945D4587FD4CC3C501B4010F94B8
:109E0000FC4A0F94D04A7AAB69AB672B21F481E00E
:109E100090E09AAB89AB4090A1055090A20560906C
:109E2000A3057090A405A9A9BAA9BD0180E090E09E
:109E30000F9461454B015C019B01AC01C701B60168
:109E40000F94634A6DA37EA38FA398A7A5019401E5
:109E500069A17AA18BA19CA10F94634AA1966CAFD2
:109E60007DAF8EAF9FAFA197A301920160910E05C8
:109E700070910F0580911005909111050F948649FE
:109E8000A50194010F94634AA5966CAF7DAF8EAF88
:109E90009FAFA5972DA13EA14FA158A5CA01B90119
:109EA0000F94C24520E030E040E05FE30F94C245EC
:109EB0009B01AC0160E070E080E89FE30F9486496D
:109EC00065966CAF7DAF8EAF9FAF659729AD3AAD0C
:109ED0004BAD5CAD29873A874B875C874D865E86A4
:109EE0006F86788A6091520270915302072E000C9F
:109EF000880B990B0F946345209101023091020267
:109F000040910302509104020F94C2452AE037EDBC
:109F100043E25CE30F94C24569966CAF7DAF8EAFB0
:109F20009FAF69970F94EF109B01AC0128533F4FEF
:109F30004F4F5F4F6D962CAF3DAF4EAF5FAF6D97FC
:109F400080911A1090911B10A0911C10B0911D10BF
:109F500021968CAF9DAFAEAFBFAF219720911E1061
:109F600030911F10409120105091211025962CAF58
:109F70003DAF4EAF5FAF2597809122109091231097
:109F8000A0912410B091251029968CAF9DAFAEAF53
:109F9000BFAF2997998D99A3AA8DA9A72B8C3C8C2B
:109FA00021E030E03EAB2DAB39E139AF49A95AA9E8
:109FB0008DA99EA94817590709F4BBC10E94E7F86B
:109FC0000F94EF10DC01CB016D962CAD3DAD4EAD85
:109FD0005FAD6D97821B930BA40BB50BB7FD11C042
:109FE0000F94EF109B01AC0128533F4F4F4F5F4F31
:109FF0006D962CAF3DAF4EAF5FAF6D9780E00E9486
:10A00000156139AD315039AF332309F444C02D8D7A
:10A010003E8D4F8D58A165966CAD7DAD8EAD9FADDB
:10A0200065970F94C2456B017C0129A139A5A10157
:10A030006DA17EA18FA198A50F94C245A70196019D
:10A040000F9487497B018C0129A139A5A10165964F
:10A050006CAD7DAD8EAD9FAD65970F94C2454B0144
:10A060005C012D8D3E8D4F8D58A16DA17EA18FA1DC
:10A0700098A50F94C2459B01AC01C501B4010F9492
:10A08000864969A379A71C01C701D8018D8F9E8FCE
:10A09000AF8FB8A350C04DA95EA9BA0180E090E08F
:10A0A0000F9461452DA13EA14FA158A50F94C24523
:10A0B0004B015C010F94604A6B017C01C501B40146
:10A0C0000F94364C4B015C01A7019601698D7A8D86
:10A0D0008B8D9C8D0F94C2452B013C01A5019401F1
:10A0E0006DA57EA58FA598A90F94C245A3019201E5
:10A0F0000F94874969A379A71C01A5019401698D73
:10A100007A8D8B8D9C8D0F94C2454B015C01A7010C
:10A1100096016DA57EA58FA598A90F94C2459B01B8
:10A12000AC01C501B4010F9486496D8F7E8F8F8F6E
:10A1300098A359E159AF29A139A5A1012D966CAD7C
:10A140007DAD8EAD9FAD2D970F94874969837A833E
:10A150008B839C832D8D3E8D4F8D58A161966CAD68
:10A160007DAD8EAD9FAD61970F9487496D837E83E2
:10A170008F839887A1962CAD3DAD4EAD5FADA19775
:10A1800069857A858B859C850F94874969877A874D
:10A190008B879C87A5962CAD3DAD4EAD5FADA59749
:10A1A0006D857E858F8598890F9487496D877E8719
:10A1B0008F87988B80913902882321F0CE010196F8
:10A1C0000E940576CE0101960E94E3671D8A1E8AD1
:10A1D0001F8A188E10912F0521962CAD3DAD4EADE6
:10A1E0005FAD21976091A5057091A6058091A705A7
:10A1F0009091A8050F9486492B013C0125962CAD22
:10A200003DAD4EAD5FAD25976091A9057091AA0552
:10A210008091AB059091AC050F9486494B015C0190
:10A2200029962CAD3DAD4EAD5FAD29976091AD0542
:10A230007091AE058091AF059091B0050F9486495D
:10A240006B017C01A3019201C301B2010F94C245CD
:10A250002B013C01A5019401C501B4010F94C24535
:10A260009B01AC01C301B2010F9487494B015C0112
:10A27000A7019601C701B6010F94C2459B01AC012D
:10A28000C501B4010F9487490F94404C9B01AC0168
:10A2900069966CAD7DAD8EAD9FAD69970F94C2454B
:10A2A000698B7A8B8B8B9C8BCE0145966C01E12E52
:10A2B0008E010F5E1F4F9E01235F3F4F4DEA55E019
:10A2C00069EA75E085EA95E00E94BAAB882389F1D6
:10A2D0002091A5053091A6054091A7055091A805AC
:10A2E00021962CAF3DAF4EAF5FAF21978091A9056E
:10A2F0009091AA05A091AB05B091AC0525968CAFC5
:10A300009DAFAEAFBFAF25972091AD053091AE05A3
:10A310004091AF055091B00529962CAF3DAF4EAF9F
:10A320005FAF29974DA95EA94F5F5F4F5EAB4DAB05
:10A330003DCE82E095E00E94E36721962CAD3DADD5
:10A340004EAD5FAD21976091A5057091A6058091F6
:10A35000A7059091A8050F9486492B013C012596ED
:10A360002CAD3DAD4EAD5FAD25976091A9057091C7
:10A37000AA058091AB059091AC050F9486494B01DD
:10A380005C0129962CAD3DAD4EAD5FAD2997609136
:10A39000AD057091AE058091AF059091B0050F9419
:10A3A00086496B017C01A3019201C301B2010F94A4
:10A3B000C2452B013C01A5019401C501B4010F94D4
:10A3C000C2459B01AC01C301B2010F9487494B0107
:10A3D0005C01A7019601C701B6010F94C2459B011C
:10A3E000AC01C501B4010F9487496B017C0120E0E9
:10A3F00030E0A9010F945D45882349F11D8A1E8A2A
:10A400001F8A188E10912F05C701B6010F94404C7A
:10A410009B01AC0169966CAD7DAD8EAD9FAD69972A
:10A420000F94C245698B7A8B8B8B9C8BCE014596A2
:10A430006C01E12E8E010F5E1F4F2EE035E04DEADC
:10A4400055E069EA75E085EA95E00E94BAAB80E1E3
:10A45000E2E0F5E0A5E9B5E001900D928A95E1F71B
:10A4600018C0E8E7F1E184918F010F5F1F4F882347
:10A4700021F00E94EA5CF801F6CFECEEF9E084915D
:10A480008F010F5F1F4F882321F00E94EA5CF801C3
:10A49000F6CFCC59DF4F0FB6F894DEBF0FBECDBF5D
:10A4A000DF91CF911F910F91FF90EF90DF90CF90B0
:10A4B000BF90AF909F908F907F906F905F904F90E4
:10A4C0003F902F9008958091570390915803A09149
:10A4D0005903B0915A038093010290930202A09312
:10A4E0000302B09304028091550390915603909318
:10A4F00053028093520208958091010290910202CA
:10A50000A0910302B09104028093570390935803E3
:10A51000A0935903B0935A03809152029091530231
:10A52000909356038093550384E690E090935302F2
:10A53000809352020895CF92DF92EF92FF920F9391
:10A540001F936A01E0909D05F0909E0500919F0584
:10A550001091A005FB012081318142815381FC01D2
:10A5600060817181828193810E9455481F910F9172
:10A57000FF90EF90DF90CF900895CF92DF92EF920F
:10A58000FF920F931F936B01FC01E080F180028129
:10A590001381E5E9F5E024813581468157816081A9
:10A5A0007181828193810E9455481F910F91FF9084
:10A5B000EF90DF90CF900895BF92CF92DF92EF920D
:10A5C000FF920F931F93CF93DF93CDB7DEB72897FA
:10A5D0000FB6F894DEBF0FBECDBF9091820D9817D5
:10A5E00009F47AC0B82E882309F453C080E090E0C3
:10A5F000A0E2B1E48D839E83AF83B887C090600DE5
:10A60000D090610DE090620DF090630D20E030E09D
:10A61000A901C701B6010F945D4587FF0CC0A701D2
:10A62000960160E070E080E291E40F9486496D83CA
:10A630007E838F83988720E030E040EA53E46D8189
:10A640007E818F8198850F94FB4B181644F480E02F
:10A6500090E0A0EAB3E48D839E83AF83B8872D8119
:10A660003E814F81588560919D0570919E05809136
:10A670009F059091A0050F945D4587FF0AC0198240
:10A680001A821B821C82BE016F5F7F4FCE0105962E
:10A6900074DF609195057091960580919705909172
:10A6A00098052091990530919A0540919B0550910C
:10A6B0009C0519821A821B821C82E0909D05F090F5
:10A6C0009E0500919F051091A005FE0131966F0136
:10A6D0000E945548B092820D80E028960FB6F894FB
:10A6E000DEBF0FBECDBFDF91CF911F910F91FF90C5
:10A6F000EF90DF90CF90BF9008952F923F924F92AE
:10A700005F926F927F928F929F92AF92BF92CF9201
:10A71000DF92EF92FF920F931F93CF93DF93CDB70A
:10A72000DEB7A4970FB6F894DEBF0FBECDBF1C01F5
:10A730007BA36AA3498F2CA3DC018D909D90AD90E3
:10A74000BC90FB014080518062807380A501940120
:10A75000C501B401002311F10F94C2456B017C01C6
:10A76000A3019201C301B2010F94C2459B01AC0148
:10A77000C701B6010F9487496B017C0120E030E4EA
:10A7800042E556E40F945D4518160CF418C220E01B
:10A7900030E94FE256E4C701B60114C00F94C24538
:10A7A0006B017C01A3019201C301B2010F94C24568
:10A7B0009B01AC01C701B6010F94874920E030E44A
:10A7C00042E556E40F945D4518160CF4F8C1D0909C
:10A7D0003502E0903602C090370210913802F091B5
:10A7E0009D05FA8F80919E058B8F90919F059C8F80
:10A7F000A091A005AD8F2F2F382F492F5A2F6D2DE7
:10A800007E2D8C2D912F0F94FB4B181624F0DA8E91
:10A81000EB8ECC8E1D8F8091010290910202A0914F
:10A820000302B09104028E8F9F8FA8A3B9A38091D9
:10A830000A0290910B02A0910C02B0910D0280933C
:10A84000010290930202A0930302B09304021982C2
:10A850001A821B821C82DE0111966D01EA8CFB8C30
:10A860000C8D1D8DA3019201C501B4010E945548B4
:10A8700081E0A2DE81111AC18091810D82FF11C099
:10A880002091600D3091610D4091620D5091630DEA
:10A8900060E070E080E090EC0F9486492B013C0171
:10A8A00006C0412C512C20E2622E21EC722E8090A9
:10A8B000600D9090610DA090620DB090630D20E04E
:10A8C00030E0A901C501B4010F945D4587FF0BC0BD
:10A8D000A501940160E070E080E791E40F9486495F
:10A8E0004B015C0106C0812C912C90E7A92E91E4CC
:10A8F000B92EA501940160919D0570919E058091EE
:10A900009F059091A0050F94FB4B18160CF04DC0BD
:10A910008D869E86AF86B88A812C912C88E4A82EDD
:10A9200082E4B82E89869A86AB86BC86BE01675FB4
:10A930007F4FCE010D9621DE1091880D1092880D6B
:10A940000E94A6648EEB94E00F94E8288091C604E0
:10A950009091C704A091C804B091C90480939D054B
:10A9600090939E05A0939F05B093A00512D712FF68
:10A970001CC089829A82AB82BC8220E030E040EA2F
:10A9800050E460919D0570919E0580919F05909186
:10A99000A0050F9487496D837E838F839887BE01BE
:10A9A0006F5F7F4FCE010596E8DD4D825E826F823C
:10A9B000788685E595E5A5E0B1E489839A83AB8344
:10A9C000BC83BE016F5F7F4FCE010596D6DD10912F
:10A9D000880D1092880D0E94A6648EEB94E00F946F
:10A9E000E8288091C6049091C704A091C804B09152
:10A9F000C90480939D0590939E05A0939F05B093F5
:10AA0000A005C7D612FF09C060919D0570919E05F3
:10AA100080919F059091A00504C060E070E080ECFB
:10AA20009FE72091600D3091610D4091620D509132
:10AA3000630D0F9487494B018C01898D82508230C0
:10AA400048F580E090E0A8E4B2E48D8B9E8BAF8B5C
:10AA5000B88F20919D0530919E0540919F055091A2
:10AA6000A005B98DB33029F060E070E080EA90E491
:10AA700004C060E070E088EC91E40F948749698B32
:10AA80007A8B8B8B9C8BBE016B5E7F4FCE01419688
:10AA900074DD07C0E98DE13021F480E08DDD8111A6
:10AAA00005C0FCA1F33008F459C008C09CA1933044
:10AAB00008F48AC0812C912C00EC1FE7E4EEF9E049
:10AAC00084915F019FEFA91AB90A882319F082D7F0
:10AAD000F501F6CF20910D0F30910E0F40910F0F21
:10AAE0005091100FD1016D917D918D919C910F949A
:10AAF000874943E00E940A60EFEDF9E084915F012D
:10AB0000BFEFAB1ABB0A882319F064D7F501F6CF63
:10AB10002091110F3091120F4091130F5091140F8B
:10AB2000EAA1FBA160817181828193810F948749A1
:10AB300043E00E940A60EAEDF9E084915F019FEF33
:10AB4000A91AB90A882319F045D7F501F6CF43E0D1
:10AB5000B401C8010E940A608AE03CD78E8D9F8DA7
:10AB6000A8A1B9A18093010290930202A0930302CD
:10AB7000B09304029401A801B401C8010F94814C60
:10AB8000882399F160E08BEC99E00E94CD89E8E799
:10AB9000F1E184917F019FEFE91AF90A882319F006
:10ABA00019D7F701F6CFEBEBF9E084917F01AFEF16
:10ABB000EA1AFA0A8823C9F00DD7F701F6CF812CDB
:10ABC000912C00EC1FE711C08E8D9F8DA8A1B9A11B
:10ABD0008093010290930202A0930302B0930402B7
:10ABE000812C912C00EC1FE7CDCFB401C801A496B5
:10ABF0000FB6F894DEBF0FBECDBFDF91CF911F918E
:10AC00000F91FF90EF90DF90CF90BF90AF909F900B
:10AC10008F907F906F905F904F903F902F9008950E
:10AC20002F923F924F925F926F927F928F929F925C
:10AC3000AF92BF92CF92DF92EF92FF920F931F934A
:10AC4000CF93DF93CDB7DEB72C970FB6F894DEBF66
:10AC50000FBECDBF94E0899F90011124F901E35804
:10AC6000F64F4591559165917491F901E95DFD4F5C
:10AC70004083518362837383823051F0F901E75737
:10AC8000F64F45915591659174917A018B0108C0F9
:10AC9000E0905C0DF0905D0D00915E0D10915F0DE8
:10ACA000F901E55EFD4FA701B8014083518362833E
:10ACB0007383823020F0823009F463C0ADC0A0906D
:10ACC0001F02B09020020091210210912202609098
:10ACD0001B0270901C0280901D0290901E0220901A
:10ACE0002B0230902C0240902D0250902E02C090EA
:10ACF0002702D0902802E0902902F0902A02A701B2
:10AD00009601B101C2010F945D4587FD02C061014A
:10AD1000720120E030E0A901C701B6010F94FB4B9E
:10AD200087FF04C0F7FAF094F7F8F094A7019601B2
:10AD3000B301C4010F94FB4B181614F063017401A6
:10AD4000A7019601B501C8010F94FB4B181614F02A
:10AD500065017801C092B604D092B704E092B804BD
:10AD6000F092B904A7019601C701B6010F94C2453C
:10AD70006093BA047093BB048093BC049093BD04A9
:10AD80004BC019821A821B821C821D821E821F8266
:10AD9000188619861A861B861C86CE0101960E948B
:10ADA000E3678090A5059090A605A090A705B090B8
:10ADB000A80580E090E0A8EEB2E48D839E83AF8387
:10ADC000B887CE0101960E94E3672091A5053091D6
:10ADD000A6054091A7055091A805C501B4010F949F
:10ADE00086494B015C0120E030E0A9010F94FB4B48
:10ADF00087FF04C0B7FAB094B7F8B094A5019401E6
:10AE0000B701C8010F9486496093350270933602EA
:10AE100080933702909338022C960FB6F894DEBFD9
:10AE20000FBECDBFDF91CF911F910F91FF90EF909B
:10AE3000DF90CF90BF90AF909F908F907F906F905A
:10AE40005F904F903F902F900895EF92FF920F9355
:10AE50001F93CF93DF937C0184E596D5D82F882369
:10AE600029F1F6D4C82F1816ECF4E9E4FFE2849136
:10AE70008F010F5F1F4F882319F0ACD5F801F7CF72
:10AE80008DE4A8D5B70180E090E04AE00E94855F9C
:10AE90006C2FCC0F770B8AE699E00E9408C28AE0FB
:10AEA00099D508C080930B0DD0E004C080912F0588
:10AEB00080930B0D8D2FDF91CF911F910F91FF90FC
:10AEC000EF9008959091870DE92FF0E0ED57F24F44
:10AED00080839F5F943018F49093870D02C0109286
:10AEE000870D80910A0F8F5F80930A0F0895089550
:10AEF00080E090E0089580915D0490915E04981741
:10AF000059F0E92FF0E0E352FC4F80819F5F9F777B
:10AF100090935E0490E008958FEF9FEF0895CF9394
:10AF2000FC0120812B33A1F020910A0F243080F402
:10AF3000C62FBC018091870DF0E68F9FC0011124C0
:10AF40008757924F0F944E4D8C2FBCDF81E001C08C
:10AF500080E0CF9108952F923F924F925F926F922F
:10AF60007F928F929F92AF92BF92CF92DF92EF9299
:10AF7000FF920F931F93CF93DF9300D000D0CDB7F4
:10AF8000DEB79A8389830F94EF10E981FA81C68036
:10AF9000D780E084F184C114D104E104F10409F004
:10AFA000ACC22485222309F469C332852150248749
:10AFB00021E0230F22874585241301C01286E981F1
:10AFC000FA8124E0329FE00DF11D1124C684D7845C
:10AFD000E088F188E981FA81C282D382E482F58235
:10AFE000DC01CB018C0D9D1DA11DB11D86839783B6
:10AFF000A087B18784819581892B09F43FC3FFB76E
:10B00000FD83F894E981FA81228033802101612C4B
:10B01000712C0481158180911302853221F08F3FBC
:10B0200009F068C205C0E0E8F5E224912E83DAC099
:10B0300085E280931302E0E8F5E284918E838F3FEE
:10B0400009F458C2823009F469C030F5882309F444
:10B050004CC0813009F0C6C010928000109281006F
:10B06000809181008860809381008091810081605F
:10B0700080938100E3EDF4E2E491F0E0EE0FFF1F36
:10B08000E658FB4D85919491E9E1F5E2E491E09376
:10B090006003E1E0EE8330C19E81943009F482C008
:10B0A00008F460C0953009F09DC010922001109204
:10B0B00021018091210188608093210180912101EB
:10B0C000816080932101E3EDF4E2E491F0E0EE0F82
:10B0D000FF1FE658FB4D85919491E9E1F5E2E4917B
:10B0E000E0935D0395E09E8307C114BC15BC84B555
:10B0F000826084BD85B5816085BDE3EDF4E2E491B5
:10B10000F0E0EE0FFF1FE658FB4D85919491E9E1C9
:10B11000F5E2E491E09361031E82ABC21092B000AD
:10B120001092B1008091B00082608093B000809155
:10B13000B10081608093B100E3EDF4E2E491F0E0CE
:10B14000EE0FFF1FE658FB4D859194919093720D81
:10B150008093710DE9E1F5E2E491E093730DF2E083
:10B16000FE8387C21092900010929100809191000E
:10B17000886080939100809191008160809391001C
:10B18000E3EDF4E2E491F0E0EE0FFF1FE658FB4D33
:10B1900085919491E9E1F5E2E491E0935F0323E086
:10B1A0002E83AAC01092A0001092A1008091A1004D
:10B1B00088608093A1008091A10081608093A100AC
:10B1C000E3EDF4E2E491F0E0EE0FFF1FE658FB4DF3
:10B1D00085919491E9E1F5E2E491E0935E0384E0E6
:10B1E0008E838AC0EE81E7FD85C161E085E20F9420
:10B1F000B30F8E818D7F09F083C04801A12CB12C43
:10B2000060E072E18AE790E0A50194010F94D04CD0
:10B2100029833A834B835C8369017A01F1E0CF1A79
:10B22000D108E108F1082FEFC216D104E104F104BE
:10B2300009F008F44EC060E472E48FE090E0A501EC
:10B2400094010F94D04C69017A0181E0C81AD108A9
:10B25000E108F1089E81923009F5EFEFCE16D10496
:10B26000E104F10409F008F4CBC160E970ED83E07A
:10B2700090E0A50194010F94D04C69017A01F1E0AE
:10B28000CF1AD108E108F1082FEFC216D104E1046A
:10B29000F10411F008F041C183E027C08FEFC81618
:10B2A000D104E104F104B9F0B0F068E478EE81E093
:10B2B00090E0A50194010F94D04C69017A0191E0CE
:10B2C000C91AD108E108F108EE81EE2309F49AC108
:10B2D00063C181E001C082E09E81911106C095B5F5
:10B2E000987F892B85BD7AC085E09091B100987FC9
:10B2F000892B8093B10072C061E085E20F94B30F97
:10B300004801A12CB12C60E072E18AE790E0A50130
:10B3100094010F94D04C69017A01E1E0CE1AD10872
:10B32000E108F108C114D104F1E0EF06F10488F05E
:10B3300068E478EE81E090E0A50194010F94D04C90
:10B3400069017A0181E0C81AD108E108F10883E0B7
:10B3500001C081E09E81913071F490918100987FCD
:10B36000892B80938100452846284728D9F52FEF5F
:10B370003FEFA90168C0EE81E33071F49091910034
:10B38000987F892B8093910045284628472851F5BE
:10B390002FEF3FEFA90179C0FE81F43071F4909155
:10B3A000A100987F892B8093A10045284628472833
:10B3B000C9F42FEF3FEFA9017AC02E81253071F437
:10B3C00090912101987F892B80932101452846285F
:10B3D000472841F42FEF3FEFA9017BC045284628BD
:10B3E000472869F0D801AA0FBB1F91010F94774934
:10B3F00028EE33E040E050E00F944B4903C02FEFBC
:10B400003FEFA9018E81823081F12CF4882361F015
:10B410008130C9F06FC09E81943009F448C0ACF10E
:10B42000953009F456C066C0C7BC209372033093B0
:10B430007303409374035093750380916E00826090
:10B4400080936E0057C0D0928900C09288002093EC
:10B450006E0330936F034093700350937103809198
:10B460006F00826080936F0045C0C092B30020934C
:10B47000740D3093750D4093760D5093770D809138
:10B48000700082608093700035C0D0929900C092A5
:10B49000980020936A0330936B0340936C0350939E
:10B4A0006D038091710082608093710023C0D092FF
:10B4B000A900C092A80020936603309367034093CD
:10B4C00068035093690380917200826080937200D8
:10B4D00011C0D0922901C0922801209362033093B9
:10B4E000630340936403509365038091730082600B
:10B4F00080937300ED81EFBFC1C0DC01CB018C19DB
:10B500009D09AE09BF09B7FDB9C04098E981FA812C
:10B510001682178210861186B1C068E478EE81E049
:10B5200090E0A50194010F94D04C69017A01F1E0FB
:10B53000CF1AD108E108F1082FEFC216D104E104B7
:10B54000F10441F138F164E274EF80E090E0A5018C
:10B5500094010F94D04C69017A01F1E0CF1AD1081F
:10B56000E108F1082FEFC216D104E104F10409F05B
:10B5700008F4BACE62E17AE780E090E0A501940198
:10B580000F94D04C69017A0181E0C81AD108E10812
:10B59000F10819C084E0A9CE2FEFC216D104E1044E
:10B5A000F10409F008F463C062E17AE780E090E01A
:10B5B000A50194010F94D04C69017A01F1E0CF1AF2
:10B5C000D108E108F1082FEFC216D104E104F1041B
:10B5D000A9F0A0F089819A81AB81BC812AE0B59560
:10B5E000A795979587952A95D1F76C017D01F1E094
:10B5F000CF1AD108E108F10887E077CE86E075CE52
:10B6000082E073CEEFEFCE16D104E104F10469F1CC
:10B6100060F162E17AE780E090E0A50194010F9487
:10B62000D04C69017A0181E0C81AD108E108F1081B
:10B630009FEFC916D104E104F104A9F0A0F08981BB
:10B640009A81AB81BC813AE0B595A795979587958E
:10B650003A95D1F76C017D01E1E0CE1AD108E108FD
:10B66000F10885E03CCE84E03ACE83E038CE84E039
:10B6700033CE61E085E20F94B30FBFCD26960FB6AF
:10B68000F894DEBF0FBECDBFDF91CF911F910F9118
:10B69000FF90EF90DF90CF90BF90AF909F908F90F2
:10B6A0007F906F905F904F903F902F900895CF9331
:10B6B000DF93EC0160E0CE0132DC811103C080E059
:10B6C000B4D5F8CFCE010E9475778823C1F3DF91FE
:10B6D000CF910895DF92EF92FF920F931F93CF9334
:10B6E000DF93CDB7DEB76E970FB6F894DEBF0FBE0F
:10B6F000CDBF6091F9047091FA046115710501F1F3
:10B700004DE150E0CE0101967C010F94CE441E8E97
:10B71000F7018F010E191F09D190DD2019F09AE071
:10B72000D912F7CFF701E00FF11F108260E0C701D7
:10B73000F6DB882329F0C7010E947577811109C0C3
:10B7400081E02091F9043091FA04232BA1F480E0E8
:10B7500012C0DD2049F00F5F1F4F8091F9049091D6
:10B76000FA04080F191F02C000E010E01093FA0459
:10B770000093F904E5CF6E960FB6F894DEBF0FBEC6
:10B78000CDBFDF91CF911F910F91FF90EF90DF9090
:10B7900008950C9446920F931F93CF93DF93CDB7E8
:10B7A000DEB72C970FB6F894DEBF0FBECDBFE5E92C
:10B7B000F5E080859185A285B385448155816681B8
:10B7C0007781008111812281338109831A832B8340
:10B7D0003C834D835E836F83788789879A87AB87A5
:10B7E000BC8721EA35E0AE01475F5F4FBE016B5F6A
:10B7F0007F4FCE0101960E94EAC22C960FB6F894B4
:10B80000DEBF0FBECDBFDF91CF911F910F91089585
:10B8100080915B0390915C03009731F04AE050E027
:10B8200060E070E00D94944360E070E0CB01089517
:10B8300080915B0390915C03009731F04AE050E007
:10B8400060E070E00D94694260E070E0CB01089523
:10B85000EFDF97FD0AC0ECDF6F3F710581059105B1
:10B8600009F02CF4E5DF862F089580E008958FEF2E
:10B87000089580915B0390915C03892B31F0E8DFA0
:10B8800091E0811103C090E001C091E0892F0895FB
:10B890000F931F93CF9380915B0390915C0300976C
:10B8A000F1F0FC018F01C1912C2F2F7D89F0C5345F
:10B8B00011F0C536B9F7F801108260E070E00F941E
:10B8C0001641F801C083562F472F382F292F0BC060
:10B8D00060E070E0CF911F910F910D94164150E000
:10B8E00040E030E020E0652F742F832F922FCF911E
:10B8F0001F910F91089581548A3108F042C0E82FBA
:10B90000F0E040919C1350919D1360919E137091B3
:10B910009F1304C076956795579547958A95D2F7FA
:10B92000842F817040FF2FC0EE57FC4E90819923E9
:10B9300009F1E091FC04F091FD04E90FF11D908103
:10B9400020ED290F2A3098F09E3211F491810CC01D
:10B950009D3211F09B3271F4918120ED290F2A3034
:10B9600030F09E3239F4928190539A3018F42E2F91
:10B970009F2F02C020E090E020935B0390935C0334
:10B98000089580E008950895B6DF882341F081E0AE
:10B9900020915B0330915C03232B09F480E0089530
:10B9A000FC01238121110C94D46F089580E1E5E915
:10B9B000F5E0A2E0B5E001900D928A95E1F70895D7
:10B9C00080E1E2E0F5E0A5E9B5E001900D928A950D
:10B9D000E1F708959091C00095FFFCCF8093C600D9
:10B9E00008953F924F925F926F927F928F929F92B3
:10B9F000AF92BF92CF92DF92EF92FF920F931F937D
:10BA0000CF93DF931F92CDB7DEB764DE81116AC298
:10BA100080910A0F843008F047C06DDAAC0197FFBF
:10BA20007CC142C08E3409F0D9C10115110509F459
:10BA3000D5C162E37BE0C8010F94DD447C01892B12
:10BA400009F48EC16EE470E0C80104960F943A4D7B
:10BA5000009709F485C14AE050E060E070E001968B
:10BA60000F94694260937603709377038093780311
:10BA7000909379038090BE079090BF07A090C00775
:10BA8000B090C1072FEF821A920AA20AB20A681573
:10BA900079058A059B0509F465C1EF2809F062C1A3
:10BAA0008FEF9AE00E949D9080915A10882309F4AC
:10BAB00019C280910A0F811102C01092DC03EE249A
:10BAC000E3944091FA125091FB126091FC12709134
:10BAD000FD128091F6129091F712A091F812B09198
:10BAE000F912481759076A077B0708F4E12C00E0B0
:10BAF00010E09924939480E6882E97E3A92E9BE08A
:10BB0000B92E2DE8322E80910A0F843008F0EAC158
:10BB1000E110E8C18091DC038111E4C180915112F0
:10BB200090915212A0915312B09154128093FA1234
:10BB30009093FB12A093FC12B093FD1241E050E0F1
:10BB4000BE016F5F7F4F89E492E10E94C47201974A
:10BB500019F4898190E002C08FEF9FEFF82E40909A
:10BB6000FA125090FB126090FC127090FD124091FE
:10BB7000F6125091F7126091F8127091F912EE24BA
:10BB8000E394441655066606770608F4E12C44163D
:10BB9000550666067706B0F4019609F46AC08AE095
:10BBA000F81609F489C09DE0F91609F485C023E26E
:10BBB000F21619F08AE3F81296C08091DB03811126
:10BBC00092C06FC00E94C6B989E492E10E94D46F0E
:10BBD00080916412882359F1815080936412389EB9
:10BBE000C001112441E061E087599D4E0E94EC8E16
:10BBF000E091641294E0E99FF0011124EB59FD4EAD
:10BC000040815181628173814093FA125093FB12FB
:10BC10006093FC127093FD1289E492E10F94AF1FC0
:10BC200080915B108823A9F090925A1012C0109254
:10BC30005A100E9404BA0E9404F60E947EF56D33E9
:10BC400071058105910528F0B092FA04A092F904DB
:10BC500041DD80915A10811128C0EAE4FBE0849113
:10BC60006F012FEFC21AD20A8823D9F0B3DEF60192
:10BC7000F6CFE8E7F1E184916F019FEFC91AD90A85
:10BC8000882319F0A7DEF601F6CFEBE3FBE0849101
:10BC90006F012FEFC21AD20A882319F09BDEF6013A
:10BCA000F6CF83E2F81208C005C023E2F21217C1F2
:10BCB00000E010E09092DC031092DB030115110507
:10BCC00019F40E94E7F80CC08091870D889E000D42
:10BCD000111D1124F801E757F24F108280E0F2D8CD
:10BCE00000E010E010CF0F35110508F00CCF9BE3FA
:10BCF000F91202C09092DB038091DB03811103CF24
:10BD00008091870DF801889EE00DF11D1124E75701
:10BD1000F24FF0820F5F1F4FF6CE982F2091BC0795
:10BD20003091BD078A3019F09D3009F0A7C01092FC
:10BD3000DA032115310519F40E94E7F869CEF901FB
:10BD4000E658FC4F10821092BD071092BC070AE71C
:10BD500013E0F8018191803209F064CE8F01F9CFB0
:10BD6000C80179CE6AE270E0C8010F94724D9C015F
:10BD7000009701F1982F901BF12C992339F09150E5
:10BD8000F801E90FF11D8081F826F7CF4AE050E075
:10BD900060E070E0C90101960F946942CF2CD12C6C
:10BDA000E12CF12C6C157D058E059F0531F080EEA0
:10BDB0009AE078CE86EB9AE075CE809176039091EA
:10BDC0007703A0917803B09179038093BE07909395
:10BDD000BF07A093C007B093C10707C08091581058
:10BDE000882319F08CE89AE05DCE80914802811199
:10BDF00022C067E470E0C8010F943A4D0097D9F073
:10BE00004AE050E060E070E001960F9469426430CF
:10BE1000710588F4E5E1FAE084917F019FEFE91A6A
:10BE2000F90A882319F0D6DDF701F6CF60E08BE040
:10BE30009AE00E94CD8967E273E0C8010F94454DF6
:10BE4000892B21F410921A0210922D056CE273E0F6
:10BE5000C8010F94454D892B19F482E09AE095D1E1
:10BE600061E373E0C8010F94454D892B11F40E94E2
:10BE7000C5CE61E08AE793E052D8CACD2F353105AF
:10BE80000CF0C6CD9C35B9F436D897FDC1CD2091C4
:10BE9000DA032111BDCD2091BC073091BD07A90166
:10BEA0004F5F5F4F5093BD074093BC07F901E658C1
:10BEB000FC4F8083ADCD9B3319F481E08093DA038E
:10BEC0008091DA038111A4CDC90101969093BD0739
:10BED0008093BC07F901E658FC4F408399CD10923E
:10BEE000DB03EFCE0F90DF91CF911F910F91FF9069
:10BEF000EF90DF90CF90BF90AF909F908F907F900A
:10BF00006F905F904F903F9008958F929F92AF9265
:10BF1000BF92EF92FF920F931F93CF93DF93CDB712
:10BF2000DEB7A0970FB6F894DEBF0FBECDBF611588
:10BF300071058105910589F100E0842E912CA12CD9
:10BF4000B12C102FEE24E394F12CEC0EFD1EE00E2C
:10BF5000F11C07FDFA94A50194010F944B49F701D8
:10BF60006083B901CA010F5F6115710581059105F3
:10BF700041F71F3F21F1E1E0F0E0EC0FFD1FE10F81
:10BF8000F11D17FDFA9580818A3010F097E301C00A
:10BF900090E3890F1FDD1150ECCF80E3A0960FB620
:10BFA000F894DEBF0FBECDBFDF91CF911F910F91EF
:10BFB000FF90EF90BF90AF909F908F900BCDA09689
:10BFC0000FB6F894DEBF0FBECDBFDF91CF911F91AA
:10BFD0000F91FF90EF90BF90AF909F908F9008953A
:10BFE000CF92DF92EF92FF926B017C0197FF0AC024
:10BFF0008DE2F0DCF094E094D094C094C11CD11C8C
:10C00000E11CF11C4AE0C701B601FF90EF90DF9000
:10C01000CF907BCF8F929F92AF92BF92CF92DF92C1
:10C02000EF92FF92CF936B017C01B42E20E030E0C1
:10C03000A9010F945D4587FF06C08DE2CBDCF7FABE
:10C04000F094F7F8F094C0E060E070E080E09FE3E7
:10C05000CB1541F02DEC3CEC4CEC5DE30F94C2456C
:10C06000CF5FF6CF9B01AC01C701B6010F948749A2
:10C070006B017C010F94D04A4B015C014AE045DF23
:10C08000CC2379F1C501B4010F9461459B01AC014A
:10C09000C701B6010F9486496B017C018EE29ADCE0
:10C0A00020E030E040E251E4C701B6010F94C24500
:10C0B0004B015C010F94CB4A6B01770FEE08FF0830
:10C0C000C701B6018DDFC701B6010F9463459B011F
:10C0D000AC01C501B4010F9486496B017C01C150CC
:10C0E000F9F6CF91FF90EF90DF90CF90BF90AF9097
:10C0F0009F908F9008951F920F920FB60F92112468
:10C100000BB60F922F938F939F93EF93FF932091F2
:10C110005E04E0915D0481E08E0F8F779091C60000
:10C12000281729F0F0E0E352FC4F9083E82FE093CA
:10C130005D04FF91EF919F918F912F910F900BBE16
:10C140000F900FBE0F901F90189521E033E0FC0177
:10C1500031832083049624CC5F9A8091810D8E7F59
:10C160008093810D8A9A8091810D8D7F8093810DBE
:10C170008091080180958170809306018091810DE6
:10C180008B7F8093810D129A08958C01E8E7F1E18D
:10C190008491EF012196882319F01CDCFE01F8CF71
:10C1A000EDE6FCE08491EF012196882319F012DC82
:10C1B000FE01F8CF0E9419F6CFDF0E946A8D61E080
:10C1C000C8010E94CD890E94D1C460E080E00F9434
:10C1D000C80364E181E395E00E9484C562E080E0E9
:10C1E0000F94C8038EE59CE00F94A90363E080E000
:10C1F0000F94C80381E59CE00F94A9032FEF8BE413
:10C200009DE1215080409040E1F700C00000F8948B
:10C210002FEF84E39CE0215080409040E1F700C084
:10C2200000000E9419F6A895FECF2F923F924F92E0
:10C230005F926F927F928F929F92AF92BF92CF92B6
:10C24000DF92EF92FF920F931F93CF93DF9300D073
:10C250001F92CDB7DEB7182F0E94318A0F94EF10CE
:10C260006B017C0100910002002309F475C08091EC
:10C270002E05882309F470C04091A0045091A104B8
:10C280006091A2047091A30446015701841A950A93
:10C29000A60AB70AB7FC72C0833041F134F481308A
:10C2A0000CF45AC0E9E4FFE206C0843009F054C03F
:10C2B000E9E4FFE237C084919F012F5F3F4F3B834A
:10C2C0002A83882321F086DBEA81FB81F4CFE3ED2A
:10C2D000FBE08491AF014F5F5F4F5B834A8388230C
:10C2E00009F43AC077DBEA81FB81F3CFE9E4FFE2AE
:10C2F00084919F012F5F3F4F3B832A83882321F046
:10C3000069DBEA81FB81F4CFECEBFBE08491AF01C8
:10C310004F5F5F4F5B834A838823F1F05BDBEA81E9
:10C32000FB81F4CF84919F012F5F3F4F3B832A8392
:10C33000882321F04FDBEA81FB81F4CFE4EAFBE0C4
:10C340008491AF014F5F5F4F5B834A83882321F065
:10C3500041DBEA81FB81F4CF202F30E0A8EEB3E08F
:10C360000F947749C60ED71EE81EF91EC092A0048E
:10C37000D092A104E092A204F092A30480910A0F4B
:10C38000843008F42EDB0F94EF10809067049090B7
:10C390006804A0906904B0906A0481149104A10417
:10C3A000B10479F1C0906304D0906404E090650416
:10C3B000F0906604C80CD91CEA1CFB1C4B015C0104
:10C3C0008C189D08AE08BF08B7FC1BC0E8E7F1E178
:10C3D00084919F012F5F3F4F3B832A83882321F065
:10C3E000F9DAEA81FB81F4CF6091FC047091FD04DD
:10C3F00087E19CE00E9421C28AE0ECDA8EE09CE0BA
:10C4000084C0C0905F04D0906004E0906104F0901C
:10C410006204C114D104E104F10409F441C0309173
:10C42000E00F2091E10F321749F06093630470939D
:10C430006404809365049093660432C02091C40F15
:10C4400021112EC011112CC00091630410916404BD
:10C4500020916504309166040C0D1D1D2E1D3F1D9D
:10C46000DC01CB01801B910BA20BB30BB7FD18C0F5
:10C470005F9A8091810D8E7F8093810D8A9A809141
:10C48000810D8D7F8093810D809108018095817051
:10C49000809306018091810D8B7F8093810D129A8C
:10C4A0008091B4049091B504909902C0019604C0A3
:10C4B000181619062CF401979093B5048093B404D0
:10C4C0008091B4049091B5048E3E9240FCF0E8E770
:10C4D000F1E18491AF014F5F5F4F5B834A83882313
:10C4E00021F078DAEA81FB81F4CFEEEEFBE0849173
:10C4F0009F012F5F3F4F3B832A83882321F06ADA15
:10C50000EA81FB81F4CF85EE9BE03FDE0F94EF10D4
:10C510000091A8041091A9042091AA043091AB04C1
:10C520004B015C01801A910AA20AB30AB7FC4AC007
:10C530008B019C010C53164F2F4F3F4F0093A804C3
:10C540001093A9042093AA043093AB044F9BDEC13F
:10C550007A9BDCC12091060120FFD8C120910A0DF1
:10C560002111D4C1029BD2C10091A4041091A50451
:10C570002091A6043091A70401151105210531056C
:10C5800099F0DC01CB01801B910BA20BB30B805601
:10C590009A4EA109B1098827B7FD83959927AA2743
:10C5A000BB27682F619501C060E0262F30E08091A5
:10C5B000020161118095807180930001B90187E0CB
:10C5C0000F94EF0F9091E00F8091E10F9817A1F079
:10C5D000E091E10F2DE4E29FF0011124EB5CF74FB5
:10C5E00060818091E10F9091E00F981302C0698300
:10C5F00006C08F5F8F70F7CF80907F1389829980FC
:10C60000992049F10F94EF100091B0041091B104FA
:10C610002091B2043091B304DC01CB010115110566
:10C620002105310579F48C599F4FAF4FBF4F80934F
:10C63000B0049093B104A093B204B093B3042FEF6D
:10C64000298311C0801B910BA20BB30BB7FF0BC04A
:10C650003FEF398308C01092B0041092B1041092D9
:10C66000B2041092B3048980682D70E089E00F94C1
:10C67000EF0F80912C0F882309F4F9C00091440238
:10C6800010914502909046029C82A0904702AA8297
:10C690006091DF047091E0046E5F7F4F072E000C05
:10C6A000880B990B0F9463459801492D5A2D0F94CF
:10C6B0005D4587FDDCC0F090E10F212C312CE12C91
:10C6C00019828091E00F8F1509F462C08F2D90E0E0
:10C6D0003DE4B32EB89EF001B99EF00D1124E25155
:10C6E000F84F458956896789708D452B462B472B16
:10C6F00081F4418D528D638D748D452B462B472BD4
:10C7000041F4458D568D678D70A1452B462B472BE7
:10C71000D1F12DE4C22EC89E9001C99E300D112486
:10C72000A9014251584F6A01FA01618172818381E6
:10C7300094810F94404C4B015C01F60161A172A100
:10C7400083A194A10F9461452B013C01F60165A1E1
:10C7500076A187A190A50F9461459B01AC01C3010F
:10C76000B2010F94634AA50194010F94C2455B0185
:10C770006C0191014E2D59810F94FB4B18161CF43E
:10C780001501EC2CD98281E08F0D8F70F82E99CF96
:10C7900020913C0230913D0240913E0250913F0277
:10C7A000B1018E2D99810F94C24598014C815A8117
:10C7B0000F9487496B017C019B01AC01B8018C810E
:10C7C0009A810F94FB4B1816ACF000914002109127
:10C7D0004102809042028C82909043029A8298019A
:10C7E000A401B601C7010F94FB4B18161CF086017B
:10C7F000EC82FA82C090AC04D090AD04E090AE041C
:10C80000F090AF0498014C815A81C701B6010F9492
:10C81000FB4B1816D4F420E037ED43EA5CE3B80193
:10C820008C819A810F94C2454B015C0128E431EE62
:10C830004AE75FE3C701B6010F94C245A501940121
:10C840000F9487498B018C839A83C801AC81BA818C
:10C850008093AC049093AD04A093AE04B093AF0466
:10C86000B801CD010F94CB4ACB010E946E890E9482
:10C87000E7F88AE390E10E94AB57A0906F04A98289
:10C88000AA2009F44CC00F94EF1000916B04109192
:10C890006C0420916D0430916E04DC01CB01801B8F
:10C8A000910BA20BB30BB7FD3AC00F94EF106B01C5
:10C8B0007C01B9802B2D30E0A8EEB3E00F947749CE
:10C8C000C60ED71EE81EF91EC0926B04D0926C04EF
:10C8D000E0926D04F0926E040E9408CB8AE00F9003
:10C8E0000F900F900F90DF91CF911F910F91FF90BC
:10C8F000EF90DF90CF90BF90AF909F908F907F9000
:10C900006F905F904F903F902F9064C86093A40405
:10C910007093A5048093A6049093A70425CE0F904E
:10C920000F900F900F90DF91CF911F910F91FF907B
:10C93000EF90DF90CF90BF90AF909F908F907F90BF
:10C940006F905F904F903F902F9008954F925F921D
:10C950006F927F928F929F92AF92BF92CF92DF920F
:10C96000EF92FF92CF93DF93CDB7DEB7E4970FB688
:10C97000F894DEBF0FBECDBF82E00E94D7B96987B1
:10C980007A878B879C8781E00E94D7B92B013C0175
:10C9900080E00E94D7B96D8F7E8F8F8F98A3A0E71C
:10C9A000B4E08D919D910D90BC91A02D89A39AA387
:10C9B000ABA3BCA39C01AD01609178047091790494
:10C9C00080917A0490917B040F9486494B015C011D
:10C9D0008091740490917504A0917604B0917704CD
:10C9E0008DA39EA3AFA3B8A79C01AD0160917C0469
:10C9F00070917D0480917E0490917F040F9486490C
:10CA00006B017C012D8D3E8D4F8D58A1C301B2016C
:10CA10000F94864969837A838B839C83A501940153
:10CA2000C501B4010F94C2452B013C01A701960139
:10CA3000C701B6010F94C2459B01AC01C301B2010D
:10CA40000F9487492B013C0129813A814B815C81FC
:10CA5000CA01B9010F94C2459B01AC01C301B201E7
:10CA60000F9487496DA77EA78FA798AB0F94404C72
:10CA70009B01AC0160E070E080E89FE30F94634AA3
:10CA80006D837E838F8398879B01AC01C501B401C0
:10CA90000F94C245698B7A8B8B8B9C8B2D813E8149
:10CAA0004F815885C701B6010F94C2456D8B7E8BAF
:10CAB0008F8B988F2D813E814F81588569817A8136
:10CAC0008B819C810F94C245698F7A8F8B8F9C8F4D
:10CAD00029A13AA14BA15CA16091800470918104CD
:10CAE00080918204909183040F9486494B015C01EC
:10CAF0002DA13EA14FA158A5609184047091850499
:10CB000080918604909187040F9486496B017C0183
:10CB10002D8D3E8D4F8D58A169857A858B859C859D
:10CB20000F9486496D877E878F87988BA501940126
:10CB300069897A898B899C890F94C2452B013C01B4
:10CB4000A70196016D897E898F89988D0F94C245C2
:10CB50009B01AC01C301B2010F9487492B013C0139
:10CB60002D853E854F855889698D7A8D8B8D9C8D5D
:10CB70000F94C2459B01AC01C301B2010F948749D8
:10CB800069837A838B839C839B01AC0169897A8951
:10CB90008B899C890F94C2459B01AC01C501B401EE
:10CBA0000F94864969877A878B879C8729813A8188
:10CBB0004B815C816D897E898F89988D0F94C245E8
:10CBC0009B01AC01C701B6010F9486494B015C0182
:10CBD00029813A814B815C81698D7A8D8B8D9C8D09
:10CBE0000F94C2459B01AC016D857E858F85988928
:10CBF0000F9486496B017C0129853A854B855C85BC
:10CC0000CA01B9010F94C2452B013C01A501940151
:10CC1000C501B4010F94C2459B01AC01C301B2012F
:10CC20000F9487492B013C01A7019601C701B6016A
:10CC30000F94C2459B01AC01C301B2010F94874917
:10CC400069AB7AAB8BAB9CAB0F94404C9B01AC01B6
:10CC500060E070E080E89FE30F94634A2B013C01A1
:10CC60009B01AC0169857A858B859C850F94C245B3
:10CC700069877A878B879C87A3019201C501B401DC
:10CC80000F94C2456D877E878F87988BA301920191
:10CC9000C701B6010F94C24569A77AA78BA79CA7C5
:10CCA000A8E8B4E0CD90DD90ED90FC9020918C044C
:10CCB00030918D0440918E0450918F04C701B601CC
:10CCC0000F9486492DA53EA54FA558A90F948749D5
:10CCD0002D813E814F8158850F94C24520E030E080
:10CCE00040E05FE30F94C2456D837E838F83988716
:10CCF00020919004309191044091920450919304BA
:10CD0000C701B6010F9486494B015C0129813A8124
:10CD10004B815C81CA01B9010F94C2459B01AC01F2
:10CD2000C501B4010F94874929A93AA94BA95CA967
:10CD30000F94874920E030E040E05FE30F94C24564
:10CD40004B015C012D813E814F81588569817A813B
:10CD50008B819C810F94C2459B01AC01C501B4013C
:10CD60000F948649A30192010F94C2454B015C01C7
:10CD70002D813E814F815885CA01B9010F94C2456A
:10CD80002B013C01A5019401C501B4010F94C245DA
:10CD90009B01AC01C301B2010F9487499B01AC0117
:10CDA000C701B6010F9486490F94404C69837A837A
:10CDB0008B839C832D813E814F81588569897A8937
:10CDC0008B899C890F94C24529A13AA14BA15CA1F2
:10CDD0000F9487496B017C01A501940169857A85CF
:10CDE0008B859C850F94C2459B01AC01C701B601A0
:10CDF0000F9487496B017C0129A53AA54BA55CA539
:10CE00006D897E898F89988D0F94C2452B013C01D5
:10CE10002D853E854F855889698D7A8D8B8D9C8DAA
:10CE20000F94C2459B01AC01C301B2010F94864926
:10CE300029813A814B815C810F94C2459B01AC01F1
:10CE4000C701B6010F948649EEEBF4E0608371836D
:10CE5000828393832D813E814F8158856D897E89A0
:10CE60008F89988D0F94C2452DA13EA14FA158A541
:10CE70000F9487496B017C01A50194016D857E8526
:10CE80008F8598890F94C2459B01AC01C701B601FB
:10CE90000F9487496B017C0129853A854B855C8518
:10CEA000698D7A8D8B8D9C8D0F94C2452B013C0131
:10CEB00029A53AA54BA55CA569897A898B899C89A6
:10CEC0000F94C2459B01AC01C301B2010F94864986
:10CED00029813A814B815C810F94C2459B01AC0151
:10CEE000C701B6010F9486496093C2047093C304CE
:10CEF0008093C4049093C5042D813E814F81588551
:10CF0000698D7A8D8B8D9C8D0F94C2452D8D3E8DB4
:10CF10004F8D58A10F9487496B017C01A5019401A5
:10CF200069A57AA58BA59CA50F94C2459B01AC0170
:10CF3000C701B6010F9487496B017C012D853E85A1
:10CF40004F85588969897A898B899C890F94C24554
:10CF50004B015C0129853A854B855C856D897E890D
:10CF60008F89988D0F94C2459B01AC01C501B40116
:10CF70000F94864929813A814B815C810F94C24587
:10CF80009B01AC01C701B6010F9486496093C604AA
:10CF90007093C7048093C8049093C904E4960FB6B5
:10CFA000F894DEBF0FBECDBFDF91CF91FF90EF9021
:10CFB000DF90CF90BF90AF909F908F907F906F90B9
:10CFC0005F904F9008952F923F924F925F926F9291
:10CFD0007F928F929F92AF92BF92CF92DF92EF9209
:10CFE000FF920F931F93CF93DF9300D000D0CDB764
:10CFF000DEB79E838D83DC011896CD90DD90ED9099
:10D00000FC901B9700E714E02D913D914D915C91B0
:10D01000F80160817181828193810F9486492B018F
:10D020003C01AD81BE8114968D919D910D90BC9176
:10D03000A02D89839A83AB83BC839C01AD01F80149
:10D0400064817581868197810F9486494B015C01CB
:10D0500088E8282E84E0382EA3019201C301B20192
:10D060000F94C2452B013C01A5019401C501B401F7
:10D070000F94C2459B01AC01C301B2010F948749D3
:10D080009B01AC01D1016D917D918D919C910F948B
:10D0900086490F94404C9B01AC01C701B6010F9427
:10D0A0008749E5EAF5E06083718382839383AD81EC
:10D0B000BE812D913D914D915C91F8016085718506
:10D0C000828593850F9486494B015C0129813A81C1
:10D0D0004B815C81D8011C966D917D918D919C91C5
:10D0E0001F970F9486492B013C01A5019401C501AE
:10D0F000B4010F94C2454B015C01A3019201C3012D
:10D10000B2010F94C2459B01AC01C501B4010F945B
:10D1100087499B01AC01F10164817581868197810A
:10D120000F9486490F94404C9B01AC01C701B60196
:10D130000F9487496093A9057093AA058093AB0566
:10D140009093AC05AD81BE812D913D914D915C9147
:10D15000F80160897189828993890F9486494B010E
:10D160005C01AD81BE8114962D913D914D915C91F4
:10D170001797F80164897589868997890F9486497C
:10D180002B013C01A5019401C501B4010F94C245D6
:10D190004B015C01A3019201C301B2010F94C2458E
:10D1A0009B01AC01C501B4010F9487499B01AC01FF
:10D1B000D10118966D917D918D919C911B970F9443
:10D1C00086490F94404C9B01AC01C701B6010F94F6
:10D1D00087496093AD057093AE058093AF0590933A
:10D1E000B00526960FB6F894DEBF0FBECDBFDF9117
:10D1F000CF911F910F91FF90EF90DF90CF90BF9054
:10D20000AF909F908F907F906F905F904F903F90E6
:10D210002F9008952F923F924F925F926F927F923C
:10D220008F929F92AF92BF92CF92DF92EF92FF9236
:10D230000F931F93CF93DF93CDB7DEB7C854D109B7
:10D240000FB6F894DEBF0FBECDBF809139028823A0
:10D2500021F082E095E00E9405768091C40783FD6D
:10D26000A5C0C0900E05D0900F05E0901005F0907D
:10D2700011052091A1053091A2054091A30550917F
:10D28000A405C701B6010F945D45882309F48EC03B
:10D2900080912205811131C0609123057091240590
:10D2A00080912505909126050F94CB4A2091070285
:10D2B000309108026217730704F5C092A105D0925D
:10D2C000A205E092A305F092A405E9E4FFE28491AF
:10D2D0008F010F5F1F4F882321F00E94EA5CF80145
:10D2E000F6CFE9E8FBE084918F010F5F1F4F8823A1
:10D2F00021F00E94EA5CF801F6CF80900E05909034
:10D300000F05A0901005B09011052091A105309156
:10D31000A2054091A3055091A405C501B4010F9445
:10D3200086496B017C0120E030E0A9010F94FB4BA2
:10D3300087FF04C0F7FAF094F7F8F094E0912F0516
:10D3400084E0E89FF0011124E45BFD4F20813181EE
:10D3500042815381C701B6010F94C24520E030E0FD
:10D3600046E154E40F94FB4B181604F58092A10596
:10D370009092A205A092A305B092A405E9E4FFE271
:10D3800084918F010F5F1F4F882321F00E94EA5C78
:10D39000F801F6CFEAE6FBE084918F010F5F1F4FA3
:10D3A000882321F00E94EA5CF801F6CF60915202D6
:10D3B00070915302072E000C880B990B0F94634554
:10D3C0002091010230910202409103025091040227
:10D3D0000F94C2452AE037ED43E25CE30F94C24567
:10D3E00069AF7AAF8BAF9CAF69A77AA78BA79CA7D1
:10D3F0008090020590900305A0900405B09005056B
:10D40000209195053091960540919705509198058A
:10D41000C501B4010F9486492B013C01C09006055B
:10D42000D0900705E0900805F09009052091990536
:10D4300030919A0540919B0550919C05C701B6011A
:10D440000F94864969AB7AAB8BAB9CAB20E030E0A4
:10D45000A901C301B2010F945D4581113AC020E0DA
:10D4600030E0A90169A97AA98BA99CA90F945D450F
:10D4700081112FC010912F05198A1A8A1B8A1C8AC4
:10D4800089829A82AB82BC82CD82DE82EF82F8866C
:10D4900080910A0590910B05A0910C05B0910D05A6
:10D4A00089879A87AB87BC87AE01475F5F4FBE0114
:10D4B0006B5F7F4FCE0101960F94F729CE01019645
:10D4C00082DDDE0151966D01E12E8E01075D1F4F59
:10D4D000BBC3A5019401C501B4010F94C2454B0122
:10D4E0005C01A7019601C701B6010F94C2459B01DB
:10D4F000AC01C501B4010F94874920E030E442E556
:10D5000056E40F945D4518160CF4AAC320919D05AE
:10D5100030919E0540919F055091A00560910A05AC
:10D5200070910B0580910C0590910D050F94864923
:10D530006DAB7EAB8FAB98AF2091A1053091A2056A
:10D540004091A3055091A40560910E0570910F05BF
:10D5500080911005909111050F9486496DA77EA7C3
:10D560008FA798ABA3019201C301B2010F94C245EA
:10D570006B017C0129A93AA94BA95CA9CA01B9018F
:10D580000F94C2459B01AC01C701B6010F948749B6
:10D590006B017C012DA93EA94FA958ADCA01B90163
:10D5A0000F94C2459B01AC01C701B6010F94874996
:10D5B0000F94404C6B017C012DEB37E346E855E3BB
:10D5C0000F945D4587FF13C020E030E0A9016DA5F1
:10D5D0007EA58FA598A90F94FB4BCDA4DEA4EFA444
:10D5E000F8A887FF04C0F7FAF094F7F8F0942DEB51
:10D5F00037E346E855E3C701B6010F945D4587FD63
:10D600002FC329AD3AAD4BAD5CADC701B6010F9448
:10D61000634A2091BC0F3091BD0F4091BE0F5091D5
:10D62000BF0F0F94C2450F94D04A1B01672B19F40A
:10D6300022242394312CB10180E090E00F946145C5
:10D640009B01AC0160E070E080E89FE30F94634AC7
:10D650004B015C019B01AC01C301B2010F94C245B7
:10D66000698B7A8B8B8B9C8BA501940169A97AA914
:10D670008BA99CA90F94C2456D8B7E8B8F8B988F45
:10D68000A50194016DA97EA98FA998AD0F94C245FB
:10D69000698F7A8F8B8F9C8FA50194016DA57EA5D4
:10D6A0008FA598A90F94C2456D8F7E8F8F8F98A3F9
:10D6B000A5019401C701B6010F94C2459B01AC01BD
:10D6C00060E070E080E89FE30F94634A29AD3AADD3
:10D6D0004BAD5CAD0F94C24525966CAF7DAF8EAF60
:10D6E0009FAF259780911A1090911B10A0911C104C
:10D6F000B0911D108DAB9EABAFABB8AF80911E103B
:10D7000090911F10A0912010B091211089AF9AAF75
:10D71000ABAFBCAF8091221090912310A091241048
:10D72000B091251021968CAF9DAFAEAFBFAF2197C2
:10D7300080E1E5E9F5E0DE01119601900D928A9510
:10D74000E1F791E0291A310809F4FFC180919804AA
:10D75000811113C00F94EF10DC01CB0188539F4F50
:10D76000AF4FBF4F8093940490939504A093960479
:10D77000B0939704A1E0A09398040E94E7F80F9457
:10D78000EF1000919404109195042091960430912B
:10D790009704DC01CB01801B910BA20BB30BB7FDEF
:10D7A00013C00F94EF10DC01CB0188539F4FAF4F94
:10D7B000BF4F8093940490939504A0939604B093E4
:10D7C000970480E00E9415617E01B1E1EB0EF11C2F
:10D7D0008E010F5F1F4F6701F70121913191419138
:10D7E00051917F01D8016D917D918D919C910F9404
:10D7F0008749F80161937193819391938F01CE16BC
:10D80000DF0651F789859A85AB85BC858DA79EA7D4
:10D81000AFA7B8ABC980DA80EB80FC80A701960186
:10D8200060917004709171048091720490917304FE
:10D830000F9486492B013C018D819E81AF81B88573
:10D8400089AB9AABABABBCAB9C01AD0160917404EE
:10D850007091750480917604909177040F948649B5
:10D860004B015C01A3019201C301B2010F94C245B7
:10D870002B013C01A5019401C501B4010F94C245DF
:10D880009B01AC01C301B2010F9487499B01AC011C
:10D89000609188047091890480918A0490918B042E
:10D8A0000F9486490F94404C9B01AC016DA57EA559
:10D8B0008FA598A90F94874929966CAF7DAF8EAF3D
:10D8C0009FAF29976093A5057093A6058093A70540
:10D8D0009093A805A701960160917804709179044E
:10D8E00080917A0490917B040F9486492B013C012E
:10D8F00029A93AA94BA95CA960917C0470917D0487
:10D9000080917E0490917F040F9486494B015C01C5
:10D91000A3019201C301B2010F94C2452B013C0146
:10D92000A5019401C501B4010F94C2459B01AC014E
:10D93000C301B2010F9487499B01AC0160918C0433
:10D9400070918D0480918E0490918F040F9486497C
:10D950000F94404C9B01AC016DA57EA58FA598A9A5
:10D960000F9487494B015C016093A9057093AA0548
:10D970008093AB059093AC05A7019601609180045C
:10D980007091810480918204909183040F94864960
:10D990006B017C0129A93AA94BA95CA96091840477
:10D9A0007091850480918604909187040F94864934
:10D9B0002B013C01A7019601C701B6010F94C24596
:10D9C0006B017C01A3019201C301B2010F94C24516
:10D9D0009B01AC01C701B6010F9487499B01AC01C3
:10D9E00060919004709191048091920490919304BD
:10D9F0000F9486490F94404C9B01AC016DA57EA508
:10DA00008FA598A90F9487496B017C016093AD05A0
:10DA10007093AE058093AF059093B0051DA21EA232
:10DA20001FA218A610912F052DA93EA94FA958ADE8
:10DA300029966CAD7DAD8EAD9FAD29970F9486492B
:10DA40002B013C0129AD3AAD4BAD5CADC501B40134
:10DA50000F9486494B015C0121962CAD3DAD4EAD36
:10DA60005FAD2197C701B6010F9486496B017C0118
:10DA7000A3019201C301B2010F94C2452B013C01E5
:10DA8000A5019401C501B4010F94C2459B01AC01ED
:10DA9000C301B2010F9487494B015C01A7019601B4
:10DAA000C701B6010F94C2459B01AC01C501B40189
:10DAB0000F9487490F94404C9B01AC0125966CADA7
:10DAC0007DAD8EAD9FAD25970F94C24569A37AA316
:10DAD0008BA39CA3DE0195966D01E12E8E010F5D57
:10DAE0001F4F9E01235F3F4F4DEA55E069EA75E005
:10DAF00085EA95E00E94BAAB882339F18091A505AB
:10DB00009091A605A091A705B091A8058DAB9EABFD
:10DB1000AFABB8AF8091A9059091AA05A091AB05D4
:10DB2000B091AC0589AF9AAFABAFBCAF8091AD05FA
:10DB30009091AE05A091AF05B091B00521968CAF44
:10DB40009DAFAEAFBFAF2197FCCD82E095E03BDA51
:10DB50002DA93EA94FA958AD6091A5057091A605C4
:10DB60008091A7059091A8050F9486492B013C014F
:10DB700029AD3AAD4BAD5CAD6091A9057091AA0598
:10DB80008091AB059091AC050F9486494B015C01E7
:10DB900021962CAD3DAD4EAD5FAD21976091AD05A9
:10DBA0007091AE058091AF059091B0050F948649B4
:10DBB0006B017C01A3019201C301B2010F94C24524
:10DBC0002B013C01A5019401C501B4010F94C2458C
:10DBD0009B01AC01C301B2010F9487494B015C0169
:10DBE000A7019601C701B6010F94C2459B01AC0184
:10DBF000C501B4010F9487496B017C0120E030E03E
:10DC0000A9010F945D45882349F11DA21EA21FA200
:10DC100018A610912F05C701B6010F94404C9B0127
:10DC2000AC0125966CAD7DAD8EAD9FAD25970F9463
:10DC3000C24569A37AA38BA39CA3DE0195966D01CF
:10DC4000E12E8E010F5D1F4F2EE035E04DEA55E0CD
:10DC500069EA75E085EA95E00E94BAAB0E94E05C53
:10DC6000C85BDF4F0FB6F894DEBF0FBECDBFDF91AC
:10DC7000CF911F910F91FF90EF90DF90CF90BF90C9
:10DC8000AF909F908F907F906F905F904F903F905C
:10DC90002F9008954F925F926F927F928F929F92F2
:10DCA000AF92BF92CF92DF92EF92FF920F931F93AA
:10DCB000CF93DF9300E41DE020E030E042E553E441
:10DCC000F80160817181828193810F9487492BEDE6
:10DCD0003FE049E450E40F94C24520E030E044E3E3
:10DCE00053E40F94634A4B015C010F94604A2B018B
:10DCF0003C0120E030E0A90160914C0D70914D0D88
:10DD000080914E0D90914F0D0F9487496B017C01CE
:10DD1000C0E7D4E09B01AC01C301B2010F94C2453E
:10DD2000688379838A839B83C501B4010F94364C41
:10DD30009B01AC01C701B6010F94C2456C837D8382
:10DD40008E839F8320E030E045EA53E4F80164814C
:10DD50007581868197810F9487492BED3FE049E4D7
:10DD600050E40F94C24520E030E044E353E40F94C4
:10DD7000634A4B015C010F94604A9B01AC01C701EF
:10DD8000B6010F94C245688779878A879B87C5014A
:10DD9000B4010F94364C9B01AC01C701B6010F943E
:10DDA000C2456C877D878E879F8720E030E044EBFB
:10DDB00052E4F80160857185828593850F948749C7
:10DDC0002BED3FE049E450E40F94C24520E030E001
:10DDD00044E353E40F94634A4B015C010F94604A9F
:10DDE0009B01AC01C701B6010F94C245688B798BCA
:10DDF0008A8B9B8BC501B4010F94364C9B01AC01FF
:10DE0000C701B6010F94C2456C8B7D8B8E8B9F8BA7
:10DE100020E030E0A90160913C0D70913D0D8091B2
:10DE20003E0D90913F0D0F9487499B01AC010F94DB
:10DE3000C245E8E8F4E0608371838283938364835E
:10DE4000758386839783608771878287938782E053
:10DE50000E94105610921D0FDF91CF911F910F91CC
:10DE6000FF90EF90DF90CF90BF90AF909F908F90FA
:10DE70007F906F905F904F900895CF93DF93E091E4
:10DE8000090FF0E0ED57F24F8081882381F0E7E63B
:10DE9000FBE08491EF012196882321F00E94EA5C47
:10DEA000FE01F7CF8AE0DF91CF910C94EA5CDF911D
:10DEB000CF910895CF93DF9380915D0480935E04AA
:10DEC000EEE5FBE08491EF012196882321F00E948A
:10DED000EA5CFE01F7CF8091BE079091BF07A09149
:10DEE000C007B091C107BC01CD016F5F7F4F8F4F5D
:10DEF0009F4F0E94F05F8AE00E94EA5CDF91CF9121
:10DF0000BCCF0F931F93CF93DF93FC012381222378
:10DF100011F080E044C08B01EC01FB018789803166
:10DF200039F18032B1F783E08B83F801428D538D54
:10DF3000648D758D4D8B5E8B6F8B788F9E012F5E00
:10DF40003F4FC8010F94AF1E882319F31A8F098F12
:10DF500081E08983188619861A861B861C821D8299
:10DF60001E821F82188A1C861D861E861F8617C069
:10DF700082E08B831D8A1E8A1F8A188EFB01808D8A
:10DF8000918DA0E0B0E025E0880F991FAA1FBB1F6C
:10DF90002A95D1F7898B9A8BAB8BBC8BD7CFDF912E
:10DFA000CF911F910F910895CF93DF93EC010F94C0
:10DFB0007D1F1B82DF91CF910895CF93DF93EC01FA
:10DFC00041E0611101C040E06C857D858E859F85B3
:10DFD0000F94661D882341F0888920E2829FC0014A
:10DFE00011248F549A4F02C080E090E0DF91CF91CE
:10DFF0000895CF93DF93EB01FC012381211102C02F
:10E0000080E027C02250223020F48FE288831982DA
:10E010001FC060E0D2DF009799F3FC0190E080E040
:10E020002EE23081303269F0883029F4DE01A90F08
:10E03000B11D2C939F5FDE01A90FB11D30813C9370
:10E040009F5F8F5F31968B3061F7C90FD11D1882AA
:10E0500081E0DF91CF9108953F924F925F926F924E
:10E060007F928F929F92AF92BF92CF92DF92EF9268
:10E07000FF920F931F93CF93DF93CDB7DEB72C970B
:10E080000FB6F894DEBF0FBECDBF5C01DC01599620
:10E090008D909C905A97F40181859285A385B485D3
:10E0A0009C01AD012F5F3F4F4F4F5F4F29873A874C
:10E0B0004B875C87D5011496CD90DD90ED90FC9058
:10E0C0001797C114D104E104F10439F0BFEFCB1A62
:10E0D000DB0AEB0AFB0A312C07C0F401C080D180B7
:10E0E000E280F38033243394260137011D821E829F
:10E0F0001F821886F40181859285A385B4852D81C0
:10E100003E814F815885281739074A075B0708F079
:10E1100064C089859A85AB85BC858C159D05AE0547
:10E12000BF0550F482E0C82ED12CE12CF12C92E0F6
:10E13000492E512C612C712C9E012F5F3F4FB7014E
:10E14000A601C4010F942F1E882309F446C08981BB
:10E150009A81AB81BC81892B8A2B8B2B41F02601C4
:10E1600037019FEF491A590A690A790A05C0C41490
:10E17000D504E604F70491F02D813E814F81588546
:10E180002F5F3F4F4F4F5F4F2D833E834F83588705
:10E190003FEFC31AD30AE30AF30AACCF0FEF1FEF26
:10E1A0002FEF3FE0B301A201C4010F949E1DF82E92
:10E1B000882399F0D50114964D915D916D917C91D4
:10E1C0001797411551056105710549F093018201C9
:10E1D000C4010F949E1D811102C0F12C29C0D501EC
:10E1E00014964D925D926D927C921797332051F068
:10E1F000D301C2010196A11DB11DF4018083918359
:10E20000A283B383F50185899689A789B08D892B6F
:10E210008A2B8B2B69F4D50155964D925D926D92A8
:10E220007C92589711968C911197806811968C93D7
:10E230008F2D2C960FB6F894DEBF0FBECDBFDF91A9
:10E24000CF911F910F91FF90EF90DF90CF90BF90F3
:10E25000AF909F908F907F906F905F904F903F9086
:10E26000089540E050E0BA010D94AF1F61E0FC0159
:10E2700080810C9432E38EBD0DB407FEFDCF08956E
:10E280008FEF8EBD0DB407FEFDCF8EB508950F93B1
:10E290001F93CF93DF93EB010F94EF108B01F0DF0F
:10E2A0008F3F49F00F94EF10601B710B6C177D07C7
:10E2B000B0F380E001C081E0DF91CF911F910F9119
:10E2C00008958F929F92AF92BF92EF92FF921F9309
:10E2D000CF93DF93EC01162F49015A019A81892FC0
:10E2E000806A86958CBD90FD03C081E0963009F46C
:10E2F00080E08DBD60E088810E9432E36CE271E0D5
:10E30000CE01C5DF812F8064B6DF88E1E82EF12CD5
:10E31000D501C4010E2C04C0B695A7959795879595
:10E320000A94D2F7A8DF88E0E81AF10888EFE81627
:10E330008FEFF80669F7112391F0183011F487E890
:10E3400001C08FEF98DF1C3009F49ADF10E098DFEE
:10E350008B8387FF07C01F3F29F01F5FF8CF85E938
:10E360008ADFF4CFDF91CF911F91FF90EF90BF90A4
:10E37000AF909F908F9008950F931F93CF93DF934B
:10E38000EC0189018C81833039F089E0440F551FFD
:10E39000661F771F8A95D1F79A01AB0168E1CE011C
:10E3A00090DF882311F086E02CC08EEF8EBDF8013F
:10E3B000C8019E5F0DB407FEFDCF20812EBD0DB4B8
:10E3C00007FEFDCF21812EBD32968E179F0791F754
:10E3D0000DB407FEFDCF8FEF4EDF8FEF4CDF50DF28
:10E3E0008B838F71853029F083E18983CE013EDFF5
:10E3F00009C068E572E0CE014ADF182F811106C01E
:10E4000087E18983CE0132DF10E00FC020E030E0E9
:10E41000A9016DE0CE0155DF811103C031DF8823F2
:10E4200011F086E1EECFCE0121DF812FDF91CF9178
:10E430001F910F9108952F923F924F925F926F928A
:10E440007F928F929F92AF92BF92CF92DF92EF9284
:10E45000FF920F931F93CF93DF93EC012A013B01AF
:10E4600069018C81833039F059E0440C551C661CDD
:10E47000771C5A95D1F743E0342E22242A94560172
:10E4800081E0A81A8EEFB80A4601EEEF9E1AA301AA
:10E49000920161E1CE0115DF882319F0F4E0F983E0
:10E4A00052C00F94EF108B01EBDE8B838F3F51F442
:10E4B0000F94EF10601B710B6D327140A8F381E176
:10E4C00089833DC08E3F19F0EFE0E98338C02EBC50
:10E4D000D601F6010DB407FEFDCF8EB581932EBC9B
:10E4E000AE16BF06B9F70DB407FEFDCF8EB5F50128
:10E4F0008083E12CF12C8D91EF2DFF27E827EE0F83
:10E50000FF1FE651F34F85919491FE2CEE24E826EF
:10E51000F926A815B90579F7B3DE082F10E0102FFA
:10E520000027AEDE082B0E151F0519F0F0E2F98367
:10E5300006C0CE019BDE8FEF9EDE81E012C0CE01D1
:10E5400095DE8FEF98DECE0191DE3A94332041F0D4
:10E5500020E030E0A9016CE0CE01B3DE198297CF54
:10E5600080E0DF91CF911F910F91FF90EF90DF90AE
:10E57000CF90BF90AF909F908F907F906F905F9063
:10E580004F903F902F9008952F923F924F925F921D
:10E590006F927F928F929F92AF92BF92CF92DF92B3
:10E5A000EF92FF920F931F93CF93DF9300D01F92B0
:10E5B000CDB7DEB79C838B834B015A01DC011396E8
:10E5C0008C91811103C08FEF9FEFEAC0EB81FC813A
:10E5D000818180FFF8CFAB81BC8151960D911D9157
:10E5E0002D913C91549718964D915D916D917C9130
:10E5F0001B97C501A0E0B0E068017901C41AD50AF3
:10E60000E60AF70AC816D906EA06FB0618F4580106
:10E61000A41AB50A75018B819C8104969A8389831B
:10E62000612C42E0742EE114F10409F48BC0AB813B
:10E63000BC8118964D915D916D917C911B976A01FB
:10E64000B1E0DB22EB81FC812381818D928D1A0167
:10E650002B0139E056944794379427943A95D1F793
:10E66000223061F4FC01828D938DA48DB58DBC01A7
:10E67000CD01620D731D841D951D4AC0DC011496E9
:10E680001C9111501221C114D10401F511111EC0A9
:10E69000452B462B472B59F4EB81FC8185899689C4
:10E6A000A789B08D84839583A683B7830FC0AB8180
:10E6B000BC8114964D915D916D917C911797298144
:10E6C0003A810F942F1E882309F47DCFEB81FC81C2
:10E6D000218D328D84819581A681B7810297A10910
:10E6E000B109F901058404C0880F991FAA1FBB1F37
:10E6F0000A94D2F74685578560897189840F951FE2
:10E70000A61FB71FBC01CD01610F711D811D911D99
:10E7100093012C193D0987012E153F0508F4890145
:10E720000115F2E01F0771F52091B1073091B20792
:10E730004091B3075091B407621773078407950798
:10E7400019F420C0C5012CC09401AB01BC0180911B
:10E75000BA079091BB076FDE882309F434CF800E8F
:10E76000911EEB81FC8180859185A285B385800F08
:10E77000911FA11DB11D80879187A287B387E01AE1
:10E78000F10A51CF40E00F94661D882309F41BCF96
:10E79000B6016F547A4FA801C4010F94134DDFCF17
:10E7A0000F900F900F900F90DF91CF911F910F91CD
:10E7B000FF90EF90DF90CF90BF90AF909F908F90A1
:10E7C0007F906F905F904F903F902F9008954F9261
:10E7D0005F926F927F929F92AF92BF92CF92DF92A1
:10E7E000EF92FF920F931F93CF93DF931F92CDB7BA
:10E7F000DEB78C017B015A01C22EDB0159968D9147
:10E800009C915A97F801928F818FCB012ADD912C30
:10E81000F70180859185A285B385418952896389F5
:10E82000748984179507A607B70708F05FC025E02D
:10E83000B695A795979587952A95D1F7F82FFF70EC
:10E84000DF2ED70113968C91823008F45EC041E030
:10E8500050E0BE016F5F7F4FC70196DE019719F44C
:10E86000898190E002C08FEF9FEF019609F44DC0BF
:10E87000F70180859185A285B3854F96A11DB11DB5
:10E8800080879187A287B387F0E2DF9EB0011124D1
:10E890006F547A4F61157105C1F1DB018C918823AA
:10E8A00019F0853EC1F469C191100EC08091B10785
:10E8B0009091B207A091B307B091B407F801848793
:10E8C0009587A687B787D08ADB018C91882361F072
:10E8D000992493949DCF4BE050E0C5010F94064DD1
:10E8E000892B09F095CF13C0992493948C2D8274B1
:10E8F000823459F4992009F48AC0F801D08861E083
:10E90000C8015BDB009709F00BC180E039C1C7FC8F
:10E91000FCCFF0E2DF9EA00111249A012F543A4F60
:10E92000D9011B968C91817121F08C2D827109F097
:10E930006AC08091B1079091B207A091B307B091DE
:10E94000B407F80184879587A687B787D08ACA015C
:10E950008F549A4F7C01DC0154964D915C915597F0
:10E9600060E070E0DA0199278827858B968BA78B6A
:10E97000B08FF701428D538D60E070E0482B592B2A
:10E980006A2B7B2BD80155964D935D936D937C93A9
:10E990005897F9018385887161F4F701848D958D0D
:10E9A000A68DB78DF801818B928BA38BB48B81E000
:10E9B00010C0803141F598012F5E3F4FD801599624
:10E9C0008D919C915A970F94AF1E8823E1F084E0BB
:10E9D000F80183838C2D8F70D80111968C93119739
:10E9E000F801148215821682178218961D921D92C4
:10E9F0001D921C921B97C4FEB3C0C8010F94A304C0
:10EA00008111AEC082CFD80113961C927ECFD70160
:10EA100013968C911397823009F477CF51968D918C
:10EA20009D910D90BC91A02D803E9F4FAF41B105AF
:10EA300008F06BCFC70110DB882309F466CF0F9471
:10EA4000261D882309F461CFD70159962D913C9159
:10EA50005A9714968D919D910D90BC91A02D02977F
:10EA6000A109B109F901058404C0880F991FAA1FE3
:10EA7000BB1F0A94D2F74684578460887188480E79
:10EA8000591E6A1E7B1E81E08093B9074092B10730
:10EA90005092B2076092B3077092B40780E092E0A0
:10EAA000E1EBF5E0DF019C011D9221503040E1F7E0
:10EAB000DD24D394D7015996ED91FC915A97848126
:10EAC000D81690F421EB35E0B301A2014D0D511D94
:10EAD000611D711D8091BA079091BB074DDC8823A1
:10EAE00009F413CFD394E6CF80E092E0A0E0B0E049
:10EAF000058404C0880F991FAA1FBB1F0A94D2F770
:10EB0000F7014189528963897489840F951FA61F73
:10EB1000B71F818B928BA38BB48B81EB95E0D12CAB
:10EB200020E2DC011D922A95E9F72BE0F501DC01DA
:10EB300001900D922A95E1F721E238E2FC01318B38
:10EB4000208B40E058E057874687338B228B318FEC
:10EB5000208F578B468B0F94261D8111DACED5CE90
:10EB6000C5FE09C0F8014189528963897489C801C9
:10EB70000F94AF1F05C081E003C09110A9CE96CEBF
:10EB80000F90DF91CF911F910F91FF90EF90DF9049
:10EB9000CF90BF90AF909F907F906F905F904F907D
:10EBA00008958091810D8770873069F48FE40E9409
:10EBB000C45C882319F00E94395C03C08FE40E9472
:10EBC0007B5C811117C00E94C6B980E00E94FC4A9C
:10EBD0000E947C5281E08093800D0E9456A4809117
:10EBE0007F0D8093800D0E94635283E08093090221
:10EBF0000C9480D408958CE0EEEBF4E0A5E9B5E048
:10EC000001900D928A95E1F708954F925F926F926D
:10EC10007F928F929F92AF92BF92CF92DF92EF92AC
:10EC2000FF92CF93DF93EC0188809980AA80BB800C
:10EC3000CC80DD80EE80FF80A5019401C501B40188
:10EC40000F94C2452B013C01A7019601C701B601F3
:10EC50000F94C2459B01AC01C301B2010F948749D7
:10EC60002B013C012091BA043091BB044091BC04BB
:10EC70005091BD040F94FB4B181634F5C301B2013B
:10EC80000F94404C9B01AC016091B6047091B704A5
:10EC90008091B8049091B9040F94634A2B013C0110
:10ECA0009B01AC01C501B4010F94C245688379830F
:10ECB0008A839B83A3019201C701B6010F94C245C9
:10ECC0006C837D838E839F83C0902F02D09030020F
:10ECD000E0903102F0903202A701960168857985B3
:10ECE0008A859B850F945D4587FF04C0C886D986B9
:10ECF000EA86FB86C0902302D0902402E090250291
:10ED0000F0902602A7019601688579858A859B8502
:10ED10000F94FB4B181624F4C886D986EA86FB8626
:10ED2000DF91CF91FF90EF90DF90CF90BF90AF90A9
:10ED30009F908F907F906F905F904F9008954F922B
:10ED40005F926F927F928F929F92AF92BF92DF926B
:10ED5000EF92FF920F931F93CF93DF93D82EC82F7C
:10ED6000D0E0FE01E951F34F64917E01EE0CFF1CEF
:10ED7000EE0CFF1CF701E552F34F4590559065905E
:10ED80007490062E000C770B880B990B0F9463453B
:10ED90004B015C0120E030E040EC5FE3C301B201D5
:10EDA0000F94C245A50194010F94C245AB01BC016B
:10EDB00000E010E098018D2D0E94414AF701E153D7
:10EDC000F34F2591359145915491C501B4010F94AC
:10EDD000C2454B015C0120E030E0A9010F945D4584
:10EDE000882309F447C000E010E09801B501A401B0
:10EDF00070588D2D0E94414AFE01E453F34F6491F7
:10EE0000611117C0E9E4FFE28491EF0121968823A4
:10EE100021F00E94EA5CFE01F7CFEAEAFCE084916F
:10EE2000EF012196882321F00E94EA5CFE01F7CFD2
:10EE30006AE0F701E656F34F45905590659074905F
:10EE400070E080E090E00F9463459B01AC01C3014A
:10EE5000B2010F94634A2B013C01A5019401C50145
:10EE6000B4010F948749AB01BC01930182018D2D40
:10EE70000E94414AF701E05BF24F80809180A280BE
:10EE8000B38020E030E0A901C501B4010F945D45D5
:10EE90001816DCF0F701E252F84F20E030E040EEC7
:10EEA00050E460817181828193810F94C2459B01FE
:10EEB000AC01C501B4010F948649AB01BC0100E06F
:10EEC00010E098018D2D0E94414ADF91CF911F9152
:10EED0000F91FF90EF90DF90BF90AF909F908F9039
:10EEE0007F906F905F904F9008950F931F93CF93F3
:10EEF000DF938C01E9E4FFE28491EF0121968823FE
:10EF000021F00E94EA5CFE01F7CFB8018DE89CE099
:10EF10000E9421C282E20E94EA5C8AE00E94EA5CCE
:10EF200081E0DF91CF911F910F9108952F923F9231
:10EF30004F925F926F927F928F929F92AF92BF9209
:10EF4000CF92DF92EF92FF920F931F93CF93DF93B5
:10EF5000CDB7DEB7C254D1090FB6F894DEBF0FBEED
:10EF6000CDBF4C015B016A01322E19821C821C8EBE
:10EF70001F8E6115710511F410E0A4C0FC0183819E
:10EF80008111FACFFA0180818F3209F099C0F50121
:10EF900083818250823010F485010CC0F501618DAF
:10EFA000728DCE014C960E94816F882329F38E01C9
:10EFB000045E1F4FC6016C010196F60120812F32BD
:10EFC000D1F3CE0101967C013C012E019CE1490E5A
:10EFD000511C2396EFAE23972F2C9BE09150E7E333
:10EFE000F0E0EC0FFD1FE90FF11D80E2808391112D
:10EFF000F5CF960147E0D9018D91882369F18F32D1
:10F0000059F18E3239F44A3009F4B6CF98E04AE02B
:10F010009D01F1CFEAEEFEE02491222321F031960A
:10F020008213FACFA9CF491708F4A6CF813208F48A
:10F03000A3CF8F3709F4A0CF21E0290FE7E3F0E059
:10F04000EC0FFD1FE90FF11D9FE9980F9A3108F4AD
:10F0500080528083922FDCCF8FA9803209F48CCF2D
:10F060006901F90180812F5F3F4F8F32C9F38823F7
:10F07000F1F021E0AE01495C5F4FB801C701A7DBA9
:10F08000882309F479CF0A151B0519F0C8010E94DD
:10F09000D46F6E147F0441F023969FAD2397822D89
:10F0A0008701E92EF82E99CF942D852DF9CF232DA8
:10F0B000AE01495C5F4FB801C40189DB182F02C063
:10F0C0008B017FCFCE014C960E94D05CCE01019681
:10F0D0000E94D05C812FCE5BDF4F0FB6F894DEBF6D
:10F0E0000FBECDBFDF91CF911F910F91FF90EF9099
:10F0F000DF90CF90BF90AF909F908F907F906F9058
:10F100005F904F903F902F900895CF93DF938B3B6C
:10F110009240B1F0E8E7F1E18491EF012196882374
:10F1200021F00E94EA5CFE01F7CFEAEFFEE0849155
:10F13000EF012196882331F00E94EA5CFE01F7CFAF
:10F1400080E001C081E0DF91CF9108952F923F923E
:10F150004F925F926F927F928F929F92AF92BF92E7
:10F16000CF92DF92EF92FF920F931F93CF93DF9393
:10F17000CDB7DEB7C157D1090FB6F894DEBF0FBEC9
:10F18000CDBF8DB69EB6A3961FAE1EAEA39784E6E6
:10F1900090E0A5969FAF8EAFA59701E09E012F59F5
:10F1A0003F4F44E050E0BE01695A7F4FCE018D5978
:10F1B0009F4F0F94CD1B9E012F593F4F42E050E0CF
:10F1C000BE016B597F4FCE018D599F4F0F94CD1BC0
:10F1D00043E050E0BE01695A7F4F87ED92E00F9403
:10F1E000554D892B09F43CC06B968FAD6B978823E6
:10F1F00039F08FE368968FAF689769961FAE69976D
:10F20000E9E4FFE284918F010F5F1F4F811103C07A
:10F21000EDEBFFE004C00E94EA5CF801F3CF8491BB
:10F220008F010F5F1F4F882321F00E94EA5CF801D5
:10F23000F6CFBE01695A7F4F84EB9FE00E9421C246
:10F24000E6EAFFE084918F010F5F1F4F882321F0D2
:10F250000E94EA5CF801F6CF81E08093CA046BC596
:10F260002DB63EB667961CAE1DAE1EAE1FAE67979E
:10F27000A3961FAE1EAEA39701E09E012F593F4FEC
:10F2800041E050E0BE0164597F4FCE018D599F4F40
:10F290000F94CD1B80E1EBE5F2E0DE019196019049
:10F2A0000D928A95E1F780E1EBE6F2E0DE015196FE
:10F2B00001900D928A95E1F780E1EBE7F2E0DE0143
:10F2C000119601900D928A95E1F7AD964FADAD97ED
:10F2D00050E04D5F5F4F440F551F440F551F2DB732
:10F2E0003EB7241B350B0FB6F8943EBF0FBE2DBFA3
:10F2F0008DB79EB701963C0100E09E012F593F4F0C
:10F30000BC01CE018D599F4F0F94CD1B9E012F59EB
:10F310003F4F44E050E060EC7FE0CE018D599F4FBD
:10F320000F94CD1BAD96AFACAD97B12C93E0A90E69
:10F33000B11CAA0CBB1CAA0CBB1CEDB7FEB7EA198A
:10F34000FB090FB6F894FEBF0FBEEDBF2DB73EB759
:10F350002F5F3F4F79018DB79EB78A199B090FB672
:10F36000F8949EBF0FBE8DBFEDB7FEB731966F010B
:10F370009E012F593F4FA501B701CE018D599F4FD7
:10F380000F94CD1B9E012F593F4FA501B601CE0111
:10F390008D599F4F0F94CD1B8091BB0F882309F48B
:10F3A000A4C000E09E012F593F4F44E050E061E3CC
:10F3B00073E1CE018D599F4F0F94CD1B9E012F59A4
:10F3C0003F4F44E050E069E275E0CE018D599F4F18
:10F3D0000F94CD1B9E012F593F4F44E050E06DE24A
:10F3E00073E1CE018D599F4F0F94CD1B9E012F5974
:10F3F0003F4F44E050E069E073E1CE018D599F4FEB
:10F400000F94CD1B9E012F593F4F44E050E065E023
:10F4100073E1CE018D599F4F0F94CD1B9E012F5943
:10F420003F4F40E150E065E373E1CE018D599F4FBE
:10F430000F94CD1B9E012F593F4F44E050E0BE0179
:10F440006D5A7F4FCE018D599F4F0F94CD1B9E015A
:10F450002F593F4F4CE050E0BE01635C7F4FCE011F
:10F460008D599F4F0F94CD1B9E012F593F4F44E064
:10F4700050E0BE016D5A7F4FCE018D599F4F0F94C2
:10F48000CD1B9E012F593F4F44E050E0BE016D5A05
:10F490007F4FCE018D599F4F0F94CD1B01E09E01F0
:10F4A0002F593F4F41E050E0BE0165597F4FCE01DB
:10F4B0008D599F4F0F94CD1B9E012F593F4F41E017
:10F4C00050E0BE0166597F4FCE018D599F4F0F947A
:10F4D000CD1BAC968FADAC97AB96CFACAB978C9D5C
:10F4E00060011124E12CF12C7CC0AD968FADAD975D
:10F4F00090E002962DE033E1E0963FAF2EAFE0972B
:10F50000B601AE014F5F5F4F25E8A22E25E0B22E77
:10F51000D7017E0131E1E30EF11C3DE1C32E33E161
:10F52000D32EE2967FAE6EAEE2978E010F5D1F4F37
:10F5300020E030E0821793072CF0E296EEADFFADAD
:10F54000E29701C0F8014080518062807380F6012B
:10F5500041925192619271926F018217930734F038
:10F560004D905D906D907C90139705C0F7014080A1
:10F57000518062807380F501419251926192719243
:10F580005F018217930714F0FB0101C0FA0140806C
:10F59000518062807380E096EEADFFADE0974192BE
:10F5A000519261927192E096FFAFEEAFE0972F5FBC
:10F5B0003F4F6C5F7F4F4C5F5F4F1496F4E0EF0E50
:10F5C000F11CE296EEADFFADE2973496E296FFAF06
:10F5D000EEAFE2970C5F1F4F2430310509F0AACF40
:10F5E000E0CE00E09E012F593F4F44E050E0EC1484
:10F5F000FD0461F0BE016D5A7F4FCE018D599F4FC2
:10F600000F94CD1BFFEFEF1AFF0AEBCF60E67DE012
:10F61000CE018D599F4F0F94CD1B9E012F593F4F07
:10F6200044E250E062EE7FE0CE018D599F4F0F948F
:10F63000CD1B01E09E012F593F4F41E050E0BE013C
:10F6400067597F4FCE018D599F4F0F94CD1B9E015F
:10F650002F593F4F41E050E0BE0168597F4FCE0126
:10F660008D599F4F0F94CD1B00E09E012F593F4FA6
:10F6700044E050E0BE01675B7F4FCE018D599F4F44
:10F680000F94CD1B9E012F593F4F44E050E0BE0127
:10F690006F5C7F4FCE018D599F4F0F94CD1BAA9663
:10F6A0008FADAA97A996CFACA9978C9D6001112424
:10F6B000E12CF12C00E09E012F593F4FCE14DF04C6
:10F6C00071F044E050E0BE016D5A7F4FCE018D597C
:10F6D0009F4F0F94CD1B2FEFE21AF20AEBCF41E0C0
:10F6E00050E0BE0163597F4FCE018D599F4F0F945B
:10F6F000CD1B9E012F593F4F41E050E0BE0169599B
:10F700007F4FCE018D599F4F0F94CD1B9E012F59D6
:10F710003F4F44E050E06CE57DE0CE018D599F4FB6
:10F720000F94CD1B9E012F593F4F4CE050E060E5F8
:10F730007DE0CE018D599F4F0F94CD1B9E012F5917
:10F740003F4F44E050E06CE47DE0CE018D599F4F87
:10F750000F94CD1B9E012F593F4F44E050E06CE3C6
:10F760007DE0CE018D599F4F0F94CD1B9E012F59E7
:10F770003F4F44E050E06CEB7FE0CE018D599F4F4E
:10F780000F94CD1B9E012F593F4F44E050E068E39A
:10F790007DE0CE018D599F4F0F94CD1B9E012F59B7
:10F7A0003F4F4CE050E060E47DE0CE018D599F4F2B
:10F7B0000F94CD1B9E012F593F4F44E050E061E371
:10F7C0007FE0CE018D599F4F0F94CD1B9E012F5985
:10F7D0003F4F44E050E06DE27FE0CE018D599F4FF6
:10F7E0000F94CD1B9E012F593F4F44E050E065E33D
:10F7F0007FE0CE018D599F4F0F94CD1B10E000E0AC
:10F800009E012F593F4F44E050E0BE016D5A7F4F9B
:10F81000CE018D599F4F0F94CD1B111110C06796CB
:10F82000CCACDDACEEACFFAC679720E030E84BE34E
:10F8300055E4C701B6010F945D45811103C084E012
:10F84000F82E33C08091BB0F811108C0C092200FE9
:10F85000D092210FE092220FF092230F00E09E0140
:10F860002F593F4F44E050E068E27FE0CE018D59D0
:10F870009F4F0F94CD1B9E012F593F4F44E050E006
:10F8800064E27FE0CE018D599F4F0F94CD1B9E0106
:10F890002F593F4F44E050E0BE016D5A7F4FCE01DB
:10F8A0008D599F4F0F94CD1B12C0FA94FF2079F011
:10F8B00000E09E012F593F4F44E050E0BE016D5AD9
:10F8C0007F4FCE018D599F4F0F94CD1BEECF1F5F01
:10F8D000153009F094CF00E09E012F593F4F42E0D0
:10F8E00050E0BE01615A7F4FCE018D599F4F0F945A
:10F8F000CD1B9E012F593F4F44E050E0BE016D5A91
:10F900007F4FCE018D599F4F0F94CD1B6796CCAC86
:10F91000DDACEEACFFAC679720E030E84BE355E49C
:10F92000C701B6010F945D45882329F18091BB0F73
:10F93000811108C0C092580FD092590FE0925A0F0F
:10F94000F0925B0F00E09E012F593F4F44E050E0E2
:10F9500064E57FE0CE018D599F4F0F94CD1B9E0132
:10F960002F593F4F44E050E060E57FE0CE018D59D4
:10F970009F4F0F94CD1B00E09E012F593F4F42E057
:10F9800050E0BE01635A7F4FCE018D599F4F0F94B7
:10F99000CD1B9E012F593F4F41E050E0BE016359FE
:10F9A0007F4FCE018D599F4F0F94CD1B19E0115001
:10F9B00000E09E012F593F4F112359F044E050E0E1
:10F9C000BE016D5A7F4FCE018D599F4F0F94CD1BB5
:10F9D000EECF41E050E060E77DE0CE018D599F4FD2
:10F9E0000F94CD1B10E000E09E012F593F4F44E0E3
:10F9F00050E0BE016D5A7F4FCE018D599F4F0F943D
:10FA0000CD1B8091BB0F811110C011110EC06796E4
:10FA10008CAD9DADAEADBFAD679780936C0D9093EF
:10FA20006D0DA0936E0DB0936F0D1F5F1530D9F65D
:10FA30001CE0115011F41CE00FC000E09E012F5992
:10FA40003F4F42E050E0BE01655A7F4FCE018D59D5
:10FA50009F4F0F94CD1BEDCF115000E09E012F5909
:10FA60003F4F112359F044E050E0BE01615B7F4FEE
:10FA7000CE018D599F4F0F94CD1BEECF46E050E045
:10FA8000BE01675B7F4FCE018D599F4F0F94CD1BF9
:10FA90009E012F593F4F44E050E0BE016D5A7F4F09
:10FAA000CE018D599F4F0F94CD1B9E012F593F4F73
:10FAB0004CE050E0BE016F5C7F4FCE018D599F4FEF
:10FAC0000F94CD1B1CE1115011F414E00FC000E0A5
:10FAD0009E012F593F4F44E050E0BE016D5A7F4FC9
:10FAE000CE018D599F4F0F94CD1BEDCF115079F062
:10FAF00000E09E012F593F4F44E050E0BE016D5A97
:10FB00007F4FCE018D599F4F0F94CD1BEFCF10E04B
:10FB100000E09E012F593F4F44E050E0BE016D5A76
:10FB20007F4FCE018D599F4F0F94CD1B8091BB0FFE
:10FB3000811110C011110EC067968CAD9DADAEAD98
:10FB4000BFAD67978093680D9093690DA0936A0D80
:10FB5000B0936B0D1F5F1530D9F610E000E09E01E9
:10FB60002F593F4F44E050E0BE016D5A7F4FCE0108
:10FB70008D599F4F0F94CD1B8091BB0F811110C0E9
:10FB800011110EC067968CAD9DADAEADBFAD679740
:10FB90008093640D9093650DA093660DB093670DEF
:10FBA0001F5F1530D9F6A5968EAD9FADA5978456EB
:10FBB0009109ABDA8093CA04882301F1E9E4FFE2FA
:10FBC00084918F010F5F1F4F882321F00E94EA5C10
:10FBD000F801F6CFA5966EAD7FADA5976456710975
:10FBE0008EE99FE00E9408C26BEB72E086E99FE01D
:10FBF0000E9408C28AE00E94EA5C8EC0A3962EADE5
:10FC00003FADA397A7968EAD9FADA797281739074D
:10FC100009F447C081E08093CA04E8E7F1E18491E8
:10FC20008F010F5F1F4F811103C0E6E7FFE004C0A3
:10FC30000E94EA5CF801F3CF84918F010F5F1F4FA0
:10FC4000882321F00E94EA5CF801F6CFA7966EADFA
:10FC50007FADA79780E090E04AE00E94855FE1E7F2
:10FC6000FFE084918F010F5F1F4F882321F00E94D6
:10FC7000EA5CF801F6CFA3966EAD7FADA39780E066
:10FC800090E04AE00E94855FE1E6FFE084918F0109
:10FC90000F5F1F4F882309F43FC00E94EA5CF80100
:10FCA000F5CF8091BB0F811141C0E9E4FFE284915F
:10FCB0008F010F5F1F4F811103C007ED12E004C0D9
:10FCC0000E94EA5CF801F3CFF80181918F0188234B
:10FCD00019F00E94EA5CF8CFA5966EAD7FADA597AE
:10FCE0006456710984E49FE00E9408C2A3964EAD59
:10FCF0005FADA39760E070E087E39FE00E94CEC114
:10FD0000E4E3FFE084918F010F5F1F4F882321F010
:10FD10000E94EA5CF801F6CF8091BB0F811106C00A
:10FD20008091CA04811102C00F948E1C0FB6F89402
:10FD30003EBE0FBE2DBE8091BB0F811102C00E943E
:10FD40008FFC9091CA0481E089270FB6F8949EBE7B
:10FD50000FBE8DBECF58DF4F0FB6F894DEBF0FBE7B
:10FD6000CDBFDF91CF911F910F91FF90EF90DF906A
:10FD7000CF90BF90AF909F908F907F906F905F904B
:10FD80004F903F902F9008958F929F92AF92BF9285
:10FD9000CF92DF92EF92FF920F931F93CF93DF9357
:10FDA000CDB7DEB7C65AD1090FB6F894DEBF0FBE85
:10FDB000CDBFCF57DF4F188219821A821B82C158DC
:10FDC000D0408091360390913703A0913803B091D1
:10FDD0003903CB57DF4F88839983AA83BB83C558E8
:10FDE000D040C956DF4F19821882C759D04084E6E7
:10FDF00090E0C756DF4F99838883C959D04010924D
:10FE0000CA049E0129563F4F44E050E0BE016B57A3
:10FE10007F4FCE0187569F4F0F941A1CC756DF4F56
:10FE200088819981C959D0400296C756DF4F99837E
:10FE30008883C959D040C956DF4F19821882C759E3
:10FE4000D04081E0C156DF4F8883CF59D0409E011A
:10FE500029563F4F41E050E0BE0161567F4FCE0131
:10FE600087569F4F0F941A1C9E0129563F4F40E121
:10FE700050E06DE173E1CE0187569F4F0F941A1C3D
:10FE80009E0129563F4F44E050E060EC7FE0CE01F8
:10FE900087569F4F0F941A1C9E0129563F4F40E1F1
:10FEA00050E065E875E0CE0187569F4F0F941A1C0D
:10FEB0009E0129563F4F40E150E06DE073E1CE01D5
:10FEC00087569F4F0F941A1C9E0129563F4F44E0BE
:10FED00050E061E373E1CE0187569F4F0F941A1CE7
:10FEE0009E0129563F4F44E050E069E275E0CE01A3
:10FEF00087569F4F0F941A1C9E0129563F4F44E08E
:10FF000050E06DE273E1CE0187569F4F0F941A1CAB
:10FF10009E0129563F4F44E050E069E073E1CE0175
:10FF200087569F4F0F941A1C9E0129563F4F44E05D
:10FF300050E065E073E1CE0187569F4F0F941A1C85
:10FF40009E0129563F4F40E150E065E373E1CE0149
:10FF500087569F4F0F941A1C8AE097EDA3EABCE3E3
:10FF6000CF57DF4F88839983AA83BB83C158D04082
:10FF70009E0129563F4F44E050E0BE016F577F4F2E
:10FF8000CE0187569F4F0F941A1CBE016D597F4FAB
:10FF90008CE0FB0111928A95E9F79E0129563F4FAB
:10FFA0004CE050E0CE0187569F4F0F941A1C80E022
:10FFB00090E0A0E2B1E4C757DF4F88839983AA831A
:10FFC000BB83C958D0409E0129563F4F44E050E0C2
:10FFD000BE0167577F4FCE0187569F4F0F941A1C63
:10FFE000CF57DF4F188219821A821B82C158D04026
:10FFF00083E0C056DF4F8883C05AD040CF55DF4FD3
:020000021000EC
:100000008883C15AD0409E0129563F4F44E050E0BA
:10001000BE016F577F4FCE0187569F4F0F941A1C1A
:100020009E0129563F4F41E050E0BE0160567F4F90
:10003000CE0187569F4F0F941A1C9E0129563F4FA1
:1000400041E050E0BE016F557F4FCE0187569F4F74
:100050000F941A1C1AE011509E0129563F4F44E09C
:1000600050E0112349F0BE016F577F4FCE018756F4
:100070009F4F0F941A1CEFCF60E67DE0CE018756AC
:100080009F4F0F941A1C9E0129563F4F44E250E0A7
:1000900062EE7FE0CE0187569F4F0F941A1C83E0DB
:1000A000CE55DF4F8883C25AD040CD55DF4F88836D
:1000B000C35AD040C357DF4F188219821A821B825D
:1000C000CD58D040CF56DF4F188219821A821B823A
:1000D000C159D040CF57DF4F188219821A821B8234
:1000E000C158D0409E0129563F4F41E050E0BE012B
:1000F0006E557F4FCE0187569F4F0F941A1C9E015D
:1001000029563F4F41E050E0BE016D557F4FCE0173
:1001100087569F4F0F941A1C9E0129563F4F44E06B
:1001200050E0BE016F567F4FCE0187569F4F0F9410
:100130001A1C9E0129563F4F44E050E0BE01635710
:100140007F4FCE0187569F4F0F941A1C0AE010E094
:100150000150110971F09E0129563F4F44E050E0D3
:10016000BE016F577F4FCE0187569F4F0F941A1CC9
:10017000EFCFCC55DF4F1882C45AD0408FEFCB550C
:10018000DF4F8883C55AD0409E0129563F4F41E03A
:1001900050E0BE016C557F4FCE0187569F4F0F94A4
:1001A0001A1C9E0129563F4F41E050E0BE016B559D
:1001B0007F4FCE0187569F4F0F941A1C9E012956E0
:1001C0003F4F44E050E06CE57DE0CE0187569F4F05
:1001D0000F941A1C9E0129563F4F4CE050E060E5F9
:1001E0007DE0CE0187569F4F0F941A1C9E01295621
:1001F0003F4F44E050E06CE47DE0CE0187569F4FD6
:100200000F941A1C9E0129563F4F44E050E06CE3C6
:100210007DE0CE0187569F4F0F941A1C9E012956F0
:100220003F4F44E050E06CEB7FE0CE0187569F4F9C
:100230000F941A1C9E0129563F4F44E050E068E39A
:100240007DE0CE0187569F4F0F941A1C9E012956C0
:100250003F4F4CE050E060E47DE0CE0187569F4F79
:100260000F941A1C9E0129563F4F44E050E061E371
:100270007FE0CE0187569F4F0F941A1C9E0129568E
:100280003F4F44E050E06DE27FE0CE0187569F4F44
:100290000F941A1C9E0129563F4F44E050E065E33D
:1002A0007FE0CE0187569F4F0F941A1C10E0C12C9F
:1002B00080E8D82E8BE3E82E85E4F82E812C912C53
:1002C00090E8A92E9FE3B92E11113AC09E0129563C
:1002D0003F4F44E050E060E27FE0CE0187569F4F01
:1002E0000F941A1C9E0129563F4F44E050E068E2EB
:1002F0007FE0CE0187569F4F0F941A1C9E0129560E
:100300003F4F44E050E064E27FE0CE0187569F4FCC
:100310000F941A1CCF57DF4F88829982AA82BB8222
:10032000C158D0409E0129563F4F44E050E0BE01E5
:100330006F577F4FCE0187569F4F0F941A1C2EC0C8
:10034000CF57DF4FC882D982EA82FB82C158D040A2
:100350009E0129563F4F44E050E0BE016F577F4F4A
:10036000CE0187569F4F0F941A1CCF57DF4F18822C
:1003700019821A821B82C158D04004E0015071F0EA
:100380009E0129563F4F44E050E0BE016F577F4F1A
:10039000CE0187569F4F0F941A1CF0CF1F5F153068
:1003A00009F092CF84E190E0C556DF4F99838883AE
:1003B000CB59D0409E0129563F4F42E050E0BE014C
:1003C00065567F4FCE0187569F4F0F941A1C9E0192
:1003D00029563F4F44E050E068E57FE0CE01875664
:1003E0009F4F0F941A1C9E0129563F4F44E050E046
:1003F00064E57FE0CE0187569F4F0F941A1C9E0143
:1004000029563F4F44E050E060E57FE0CE0187563B
:100410009F4F0F941A1C80E290E0C356DF4F9983E0
:100420008883CD59D0409E0129563F4F42E050E08D
:10043000BE0163567F4FCE0187569F4F0F941A1C03
:10044000CA55DF4F1882C65AD04080E2EBE8F2E08E
:10045000DE019D9601900D928A95E1F79E01295645
:100460003F4F41E050E0BE016A557F4FCE018756B5
:100470009F4F0F941A1C9E0129563F4F40E250E0B7
:10048000BE01635D7F4FCE0187569F4F0F941A1CAC
:100490009E0129563F4F41E050E060E77DE0CE01EC
:1004A00087569F4F0F941A1C10E0111110C08091B5
:1004B0006C0D90916D0DA0916E0DB0916F0DCF5799
:1004C000DF4F88839983AA83BB83C158D0409E01A4
:1004D00029563F4F44E050E0BE016F577F4FCE0199
:1004E00087569F4F0F941A1C1F5F1530F1F6BE01FF
:1004F000635B7F4F86E1FB0111928A95E9F79E01CC
:1005000029563F4F46E150E0CE0187569F4F0F944A
:100510001A1C8CE2EBEAF2E0DE01119601900D92DA
:100520008A95E1F79E0129563F4F4CE250E0BE010B
:100530006F5F7F4FCE0187569F4F0F941A1CBE01ED
:1005400065587F4F86E0FB0111928A95E9F79E017D
:1005500029563F4F46E050E0CE0187569F4F0F94FB
:100560001A1CCF57DF4F188219821A821B82C1587A
:10057000D0409E0129563F4F44E050E0BE016F57E6
:100580007F4FCE0187569F4F0F941A1CBE016159B1
:100590007F4F8CE0FB0111928A95E9F79E01295665
:1005A0003F4F4CE050E0CE0187569F4F0F941A1CEE
:1005B000CF57DF4F188219821A821B82C158D04050
:1005C0001CE1115071F09E0129563F4F44E050E06C
:1005D000BE016F577F4FCE0187569F4F0F941A1C55
:1005E000F0CFCF57DF4F188219821A821B82C15871
:1005F000D04014E0115071F09E0129563F4F44E065
:1006000050E0BE016F577F4FCE0187569F4F0F942A
:100610001A1CF0CF10E0111110C08091680D90915C
:10062000690DA0916A0DB0916B0DCF57DF4F888394
:100630009983AA83BB83C158D0409E0129563F4F5E
:1006400044E050E0BE016F577F4FCE0187569F4F69
:100650000F941A1C1F5F1530F1F610E0111110C035
:100660008091640D9091650DA091660DB091670D1C
:10067000CF57DF4F88839983AA83BB83C158D0406B
:100680009E0129563F4F44E050E0BE016F577F4F17
:10069000CE0187569F4F0F941A1C1F5F1530F1F63D
:1006A0008091CA04811167C0C756DF4FE880F98086
:1006B000C959D040F4E6EF1AF108C956DF4F8881D6
:1006C0009981C759D040CB56DF4F99838883C5594C
:1006D000D04084E690E0C756DF4F99838883C9599C
:1006E000D0409E0129563F4F44E050E067ED72E054
:1006F000CE0187569F4F0F941A1C9E0129563F4FDB
:1007000042E050E0BE016B567F4FCE0187569F4FAF
:100710000F941A1CE9E4FFE284918F010F5F1F4FD1
:10072000882321F00E94EA5CF801F6CFB70182E24B
:100730009FE00E9408C2CB56DF4F48815981C559BE
:10074000D04060E070E085E19FE00E94CEC1E2E130
:10075000FFE084918F010F5F1F4F882321F00E94DB
:10076000EA5CF801F6CFC7010E9485789091CA042F
:10077000892B8093CA049091CA0481E08927CA55C5
:10078000DF4F0FB6F894DEBF0FBECDBFDF91CF9124
:100790001F910F91FF90EF90DF90CF90BF90AF909F
:1007A0009F908F900895CF92DF92EF92FF920F93D8
:1007B0001F93CF93DF9300D01F92CDB7DEB781E0B8
:1007C0008093060280916A1390916B13A0916C1331
:1007D000B0916D13B7FF08C010926A1310926B139B
:1007E00010926C1310926D1380916E1390916F1391
:1007F000A0917013B091711340916A1350916B13D3
:1008000060916C1370916D1384179507A607B70755
:1008100044F480936A1390936B13A0936C13B0937A
:100820006D1380910902882379F140916A135091E8
:100830006B1360916C1370916D1380917213909192
:100840007313A0917413B09175136A017B01C80EE4
:10085000D91EEA1EFB1EC701B6010F94614520E0B8
:1008600030E048EC52E40F94C24569837A838B836D
:100870009C83CE0101960F940D14BC0180917813D6
:10088000909179130E94B4C510915B1311110AC0A5
:1008900080917A13882309F442C080910902882349
:1008A00009F43DC040916A1350916B1360916C1331
:1008B00070916D138091721390917313A0917413C2
:1008C000B09175136A017B01C80ED91EEA1EFB1E8A
:1008D000C701B6010F94614520E030E048EC52E4D6
:1008E0000F94C2450F94D04AE0917613F09177139C
:1008F000309721F06083718382839383E0917B132F
:10090000F0917C13309731F080917A13811101C0FE
:100910001111199580915B1381110E94D7C4109217
:100920005B130F900F900F900F90DF91CF911F915D
:100930000F91FF90EF90DF90CF900895CF92DF92CC
:10094000EF92FF920F931F93CF93DF9300D01F92EC
:10095000CDB7DEB781E08093060280916A13909153
:100960006B13A0916C13B0916D13B7FF08C0109278
:100970006A1310926B1310926C1310926D13809186
:100980006E1390916F13A0917013B09171134091F9
:100990006A1350916B1360916C1370916D138417EF
:1009A0009507A607B70744F480936A1390936B13D7
:1009B000A0936C13B0936D1380910902882379F191
:1009C00040916A1350916B1360916C1370916D1389
:1009D0008091721390917313A0917413B091751359
:1009E0006A017B01C80ED91EEA1EFB1EC701B601B3
:1009F0000F94634520E030E048EC52E40F94C24588
:100A000069837A838B839C83CE0101960F940D14A6
:100A1000BC0180917813909179130E94B4C5109114
:100A20005B13111109C080917A13882309F43FC028
:100A3000809109028823D9F140916A1350916B1378
:100A400060916C1370916D13809172139091731378
:100A5000A0917413B09175136A017B01C80ED91E61
:100A6000EA1EFB1EC701B6010F94634520E030E08B
:100A700048EC52E40F94C245E0917613F09177135D
:100A8000309721F06083718382839383E0917B139D
:100A9000F0917C13309731F080917A13811101C06D
:100AA0001111199580915B1381110E94D7C4109286
:100AB0005B130F900F900F900F90DF91CF911F91CC
:100AC0000F91FF90EF90DF90CF900895CF92DF923B
:100AD000EF92FF920F931F93CF93DF9300D01F925B
:100AE000CDB7DEB781E08093060280916A139091C2
:100AF0006B13A0916C13B0916D13B7FF08C01092E7
:100B00006A1310926B1310926C1310926D138091F4
:100B10006E1390916F13A0917013B0917113409167
:100B20006A1350916B1360916C1370916D1384175D
:100B30009507A607B70744F480936A1390936B1345
:100B4000A0936C13B0936D1380910902882379F1FF
:100B500040916A1350916B1360916C1370916D13F7
:100B60008091721390917313A0917413B0917513C7
:100B70006A017B01C80ED91EEA1EFB1EC701B60121
:100B80000F9463452AE037ED43E25CE30F94C245DE
:100B900069837A838B839C83CE0101960F94AB1279
:100BA000BC0180917813909179130E94B4C5109183
:100BB0005B13111109C080917A13882309F43FC097
:100BC000809109028823D9F140916A1350916B13E7
:100BD00060916C1370916D138091721390917313E7
:100BE000A0917413B09175136A017B01C80ED91ED0
:100BF000EA1EFB1EC701B6010F9463452AE037EDDC
:100C000043E25CE30F94C245E0917613F0917713D1
:100C1000309721F06083718382839383E0917B130B
:100C2000F0917C13309731F080917A13811101C0DB
:100C30001111199580915B1381110E94D7C41092F4
:100C40005B130F900F900F900F90DF91CF911F913A
:100C50000F91FF90EF90DF90CF900895CF92DF92A9
:100C6000EF92FF920F931F93CF93DF9300D01F92C9
:100C7000CDB7DEB781E08093060280916A13909130
:100C80006B13A0916C13B0916D13B7FF08C0109255
:100C90006A1310926B1310926C1310926D13809163
:100CA0006E1390916F13A0917013B09171134091D6
:100CB0006A1350916B1360916C1370916D138417CC
:100CC0009507A607B70744F480936A1390936B13B4
:100CD000A0936C13B0936D1380910902882379F16E
:100CE00040916A1350916B1360916C1370916D1366
:100CF0008091721390917313A0917413B091751336
:100D00006A017B01C80ED91EEA1EFB1EC701B6018F
:100D10000F9463452AE037ED43E25CE30F94C2454C
:100D200069837A838B839C83CE0101960F946C1325
:100D3000BC0180917813909179130E94B4C51091F1
:100D40005B13111109C080917A13882309F43FC005
:100D5000809109028823D9F140916A1350916B1355
:100D600060916C1370916D13809172139091731355
:100D7000A0917413B09175136A017B01C80ED91E3E
:100D8000EA1EFB1EC701B6010F9463452AE037ED4A
:100D900043E25CE30F94C245E0917613F091771340
:100DA000309721F06083718382839383E0917B137A
:100DB000F0917C13309731F080917A13811101C04A
:100DC0001111199580915B1381110E94D7C4109263
:100DD0005B130F900F900F900F90DF91CF911F91A9
:100DE0000F91FF90EF90DF90CF900895CF92DF9218
:100DF000EF92FF920F931F93CF93DF9300D01F9238
:100E0000CDB7DEB781E08093060280916A1390919E
:100E10006B13A0916C13B0916D13B7FF08C01092C3
:100E20006A1310926B1310926C1310926D138091D1
:100E30006E1390916F13A0917013B0917113409144
:100E40006A1350916B1360916C1370916D1384173A
:100E50009507A607B70744F480936A1390936B1322
:100E6000A0936C13B0936D1380910902882379F1DC
:100E700040916A1350916B1360916C1370916D13D4
:100E80008091721390917313A0917413B0917513A4
:100E90006A017B01C80ED91EEA1EFB1EC701B601FE
:100EA0000F9463452FE632E143E85AE30F94C245BD
:100EB00069837A838B839C83CE0101960F946F2E76
:100EC000BC0180917813909179130E94B4C5109160
:100ED0005B13111109C080917A13882309F43FC074
:100EE000809109028823D9F140916A1350916B13C4
:100EF00060916C1370916D138091721390917313C4
:100F0000A0917413B09175136A017B01C80ED91EAC
:100F1000EA1EFB1EC701B6010F9463452FE632E1BE
:100F200043E85AE30F94C245E0917613F0917713AA
:100F3000309721F06083718382839383E0917B13E8
:100F4000F0917C13309731F080917A13811101C0B8
:100F50001111199580915B1381110E94D7C41092D1
:100F60005B130F900F900F900F90DF91CF911F9117
:100F70000F91FF90EF90DF90CF900895CF92DF9286
:100F8000EF92FF920F931F93CF93DF9300D01F92A6
:100F9000CDB7DEB781E08093060280916A1390910D
:100FA0006B13A0916C13B0916D13B7FF08C0109232
:100FB0006A1310926B1310926C1310926D13809140
:100FC0006E1390916F13A0917013B09171134091B3
:100FD0006A1350916B1360916C1370916D138417A9
:100FE0009507A607B70744F480936A1390936B1391
:100FF000A0936C13B0936D1380910902882379F14B
:1010000040916A1350916B1360916C1370916D1342
:101010008091721390917313A0917413B091751312
:101020006A017B01C80ED91EEA1EFB1EC701B6016C
:101030000F9463452AE037ED43E25CE30F94C24529
:1010400069837A838B839C83CE0101960F943D152F
:10105000BC0180917813909179130E94B4C51091CE
:101060005B13111109C080917A13882309F43FC0E2
:10107000809109028823D9F140916A1350916B1332
:1010800060916C1370916D13809172139091731332
:10109000A0917413B09175136A017B01C80ED91E1B
:1010A000EA1EFB1EC701B6010F9463452AE037ED27
:1010B00043E25CE30F94C245E0917613F09177131D
:1010C000309721F06083718382839383E0917B1357
:1010D000F0917C13309731F080917A13811101C027
:1010E0001111199580915B1381110E94D7C4109240
:1010F0005B130F900F900F900F90DF91CF911F9186
:101100000F91FF90EF90DF90CF900895CF92DF92F4
:10111000EF92FF920F931F93CF9381E0809306028B
:1011200080916A1390916B13A0916C13B0916D1321
:10113000B7FF08C010926A1310926B1310926C13D1
:1011400010926D1380916E1390916F13A091701394
:10115000B091711340916A1350916B1360916C13AD
:1011600070916D1384179507A607B70744F4809311
:101170006A1390936B13A0936C13B0936D138091CB
:1011800009028823E1F140916A1350916B13609139
:101190006C1370916D138091721390917313A091E1
:1011A0007413B09175138A019B01080F191F2A1F30
:1011B0003B1FC901B8010F9463456B017C0120E01E
:1011C00030E0A9010F945D4587FD05C020E030E0C7
:1011D00040E05FE304C020E030E040E05FEBC701A7
:1011E000B6010F9487490F94CB4ACB010F94871611
:1011F000BC0180917813909179130E94B4C5C0917D
:101200005B13C11108C080917A138823C9F18091C2
:1012100009028823A9F140916A1350916B136091E0
:101220006C1370916D138091721390917313A09150
:101230007413B09175138A019B01080F191F2A1F9F
:101240003B1FC901B8010F946345E0917613F091FB
:101250007713309721F06083718382839383E091C9
:101260007B13F0917C13309731F080917A138111C8
:1012700001C0C111199580915B1381110E94D7C4DF
:1012800010925B13CF911F910F91FF90EF90DF9021
:10129000CF900895CF92DF92EF92FF926B017C0185
:1012A00083E3C816D104E104F10470F082E3C81AA4
:1012B000D108E108F10862E370E080E090E00F946B
:1012C000B7100E94E7F8ECCFC701B6010F94B71032
:1012D000FF90EF90DF90CF900C94E7F89093E004AC
:1012E0008093DF0480E00C940BF40F931F930F9412
:1012F000EF100091F5041091F6042091F70430915D
:10130000F804DC01CB01801B910BA20BB30BB7FDE2
:101310000CC086B186FB992790F981E08927349B20
:101320008260329B84608093F4048091F404817025
:101330009091F40491FD82609091F304891751F12A
:101340008130A9F028F0823041F0833059F020C07C
:10135000913089F09230A9F01BC0992361F093304D
:1013600081F016C0913069F0923091F404C0992355
:1013700041F0933069F49091F20420910602921B9F
:1013800005C02091F20490910602920F9093F2040E
:101390008093F3041F910F9108950F931F93CF93A0
:1013A000DF938C0167FF03C01092740560E08091A9
:1013B000740590E0262F062E000C330B28173907F2
:1013C0001CF160937405C8010F94AD44800F911F08
:1013D000EC01C01BD10BC334D1053CF00197FC01DB
:1013E0002491207C2038D1F3F3CFDD27AE01B80162
:1013F00081E395E00F94CE44CF5CDA4F188283E00E
:101400008093090210923005DF91CF911F910F91C7
:101410000895CF93DF932091740521111FC0FC0123
:1014200001900020E9F73197EF01C81BD90BC334B5
:10143000D1052CF02291207C2038E1F3F5CFBC01BE
:10144000DD27AE0181E395E00F94634DCF5CDA4F69
:10145000188283E08093090210923005DF91CF91CA
:1014600008954F925F926F927F928F929F92AF9268
:10147000BF92CF92DF92EF92FF920F931F93CF9381
:10148000DF9300D01F92CDB7DEB78091D3048111D6
:101490001EC0009105020F3FD1F00F94EF10C090D5
:1014A000CF04D090D004E090D104F090D204DC01BD
:1014B000CB018C199D09AE09BF09B7FD08C0809109
:1014C000E00F9091E10F8F5F8F7089130EC20DDFD7
:1014D0008091F40482FF43C08091F104811141C0E6
:1014E00091E09093F10420912D05211103C080918A
:1014F000DE04892780935B1310922D0583E080938F
:1015000009021092F4040F94EF10DC01CB018C500F
:101510009E4FAF4FBF4F8093F5049093F604A09376
:10152000F704B093F80488E893E19C838B8382E00E
:1015300090E09A838983BE016D5F7F4FCE01019653
:1015400071D716E0115069F08AE390E10E94AB5721
:1015500062E070E080E090E00F94B710F3CF10925B
:10156000F10480910901817091E098271091F004B5
:10157000191729F19093F00481110FC264EF71E003
:1015800080E090E087DE0BD6123009F002C21092A4
:10159000AC108BE1E1EBF0E1A0EDB0E101900D9238
:1015A0008A95E1F78091AF109091B0109093CF1091
:1015B0008093CE1083E0809309020E94EDC50F94C2
:1015C000EF106B017C018091EC049091ED04A091EF
:1015D000EE04B091EF04A7019601281B390B4A0BCA
:1015E0005B0B57FD0EC2D701C6018C599F4FAF4F01
:1015F000BF4F8093EC049093ED04A093EE04B0935E
:10160000EF048091F204082E000C990B97FF03C0A1
:1016100091958195910984302CF480915B1381110F
:1016200094C0A4C08091DD04882309F467C0809130
:10163000F2048090D9049090DA04A090DB04B0907A
:10164000DC0481149104A104B10409F44AC0082EF9
:10165000000C990B97FF03C0919581959109682F14
:1016600087FF02C063E0680F65956595062E000C44
:10167000770B880B990B0F9463452B013C01C70135
:10168000B601681979098A099B090F9461459B0184
:10169000AC01C301B2010F94634A20E030E04AE795
:1016A00054E40F94C2454B015C0120E030E040E27D
:1016B00053E40F94FB4B87FF0FC020E030E046E976
:1016C00052E4C501B4010F94FB4B87FD0AC02AE028
:1016D00030E040E050E009C024E630E040E050E077
:1016E00004C021E030E040E050E0C092D904D09244
:1016F000DA04E092DB04F092DC0404C021E030E084
:1017000040E050E0A091F2040A2E000CBB0B0F94B5
:10171000F44C24E030E040E050E00F94D04C809155
:101720006A1390916B13A0916C13B0916D13820F9B
:10173000931FA41FB51F80936A1390936B13A093FC
:101740006C13B0936D131092F204D701C601805A46
:101750009541AF4FBF4F8093E8049093E904A09365
:10176000EA04B093EB0481E08093090220915502D2
:101770003091560245EC253F340741F480915402E4
:10178000882309F416C18150809354022E50314EA3
:1017900071F48091601390916113891740F49091D6
:1017A0005402992309F415C19150909354028091E9
:1017B0006F00282F227081FF05C080916F008D7F00
:1017C00080936F008091D4049091D504A091D604A9
:1017D000B091D704222329F020916F00226020933A
:1017E0006F0020910902222309F449C04AE0B6950E
:1017F000A795979587954A95D1F70097E1E0AE07B1
:10180000B10520F08FEF9FEFA0E0B0E096958795AF
:10181000009739F04091E6045091E70448175907C2
:1018200070F5223050F0243028F0243031F410923A
:10183000090203C081E080930902E0915502F09112
:101840005602199510925B138090E6049090E7047D
:10185000A12CB12C0F94EF10DC01CB018C199D0948
:10186000AE09BF0988169906AA06BB0640F40F9474
:10187000EF106C197D097093E7046093E604809182
:10188000550290915602855F954C21F08091D804C5
:10189000882379F020E6C20E2AEED21EE11CF11C4C
:1018A000C092E804D092E904E092EA04F092EB04DA
:1018B0000FC08091E8049091E904A091EA04B091EE
:1018C000EB04C81AD90AEA0AFB0AF7FE0E94D1C43F
:1018D00080910902813031F0833009F092C00F9479
:1018E000D9038FC0109209028CC0C0900102D09021
:1018F0000202E0900302F090040234E0030280014F
:101900001124F801E552FD4F20E030E040E752E4B9
:1019100060817181828193810F94634A6093010297
:101920007093020280930302909304020E94D65C9B
:101930000E5F1A4F2091CB043091CC044091CD041E
:101940005091CE04F80160817181828193810F945E
:101950008749F80160837183828393831092CB045B
:101960001092CC041092CD041092CE048FEF80938D
:10197000050281E08093D3040E940A691092D30487
:10198000C0920102D0920202E0920302F09204029D
:101990009ECD60E083EE9FE00AC010925A10109234
:1019A0005B10123009F406CE60E086ED9FE0F5DCB6
:1019B00001CE89E0809354028091E6049091E7047F
:1019C00001979093E7048093E60481E080930902F5
:1019D000DDCE96E09093540291E0909309028F5FE0
:1019E00080936013D701C601805A9541AF4FBF4F16
:1019F0008093E8049093E904A093EA04B093EB0485
:101A0000D6CE0F900F900F900F90DF91CF911F9136
:101A10000F91FF90EF90DF90CF90BF90AF909F908D
:101A20008F907F906F905F904F900895CF92DF924C
:101A3000EF92FF920F931F930F94EF100091E20427
:101A40001091E3042091E4043091E5046B017C01E2
:101A5000C01AD10AE20AF30AF7FC13C02091E1048C
:101A600020952093E104DC01CB018A549C4FAF4FB9
:101A7000BF4F8093E2049093E304A093E404B093F7
:101A8000E50481E09091E104911101C080E01F9193
:101A90000F91FF90EF90DF90CF900895FC0180E0D0
:101AA00090E02491222339F02491207C203809F001
:101AB00001963196F6CF0895FC0120E030E0919137
:101AC000992331F0907C9038D1F32F5F3F4FF7CFBF
:101AD000C90108950E94EDC53E98469A3C98449AE3
:101AE0003A98429AEAE0F1E080818E7F808380918B
:101AF0000B01809581708093090182E08093F0044E
:101B0000F4DB1092F2040895CF93DF93EC010E946E
:101B10008EC440E050E0BA01CE01DF91CF910C9429
:101B2000AEC48F929F92AF92BF92CF92DF92EF920C
:101B3000FF921F93CF93DF93C82F82E292E190939D
:101B4000BB078093BA0710923E1282E090E0A0E0BB
:101B5000B0E08093271290932812A0932912B0939B
:101B60002A121092B9071092B5071092B607109278
:101B7000B7071092B8078FEF9FEFDC018093B10792
:101B80009093B207A093B307B093B407CC2379F135
:101B9000C53008F0F8C040E060E070E0CB010F9481
:101BA000661D882309F4EFC020E1C29FC001112403
:101BB0008F559A4FFC01E254FE4F20812F7709F098
:101BC000E2C03C9640815181628173814436510567
:101BD0006105710508F4D7C03497C080D180E280D8
:101BE000F380C114D104E104F10421F4CCC0C12C70
:101BF000D12C760140E0C701B6010F94661D182F65
:101C0000882309F4C0C08091BC059091BD05811561
